:020000040800F2
:100000000000012065290008351D0008371D000883
:10001000391D00083B1D00083D1D000800000000C0
:100020000000000000000000000000003F1D00086C
:10003000411D000800000000431D0008451D000888
:10004000AD290008AD290008AD2900084D1D0008A4
:10005000AD2900085D1D00085F1D0008691D00082E
:10006000AD290008731D00087D1D0008AD2900089A
:10007000AD290008AD290008AD290008891D000838
:10008000AD290008AD290008AD290008AD290008F8
:10009000991D0008AD290008AD290008AD29000808
:1000A000AD290008AD290008AD290008AD290008D8
:1000B000AD290008AD290008A91D0008AD290008D8
:1000C000AD290008AD290008AD290008AD290008B8
:1000D000AD290008B91D0008AD290008C91D000898
:1000E000AD290008D91D0008AD290008AD29000878
:1000F000AD290008AD290008AD290008AD29000888
:10010000AD290008AD290008AD290008AD29000877
:10011000AD290008AD290008AD290008AD29000867
:10012000AD290008AD290008AD290008AD29000857
:1001300000000000000000000000000000000000BF
:1001400000000000000000000000000000000000AF
:10015000000000000000000000000000000000009F
:10016000000000000000000000000000000000008F
:10017000000000000000000000000000000000007F
:10018000000000000000000000000000000000006F
:10019000000000000000000000000000000000005F
:1001A000000000000000000000000000000000004F
:1001B000000000000000000000000000000000003F
:1001C000000000000000000000000000000000002F
:1001D000000000000000000000000000000000001F
:0401E0005FF8E0F1F3
:1001E80081F0004102E000BF83F0004330B54FEAE0
:1001F80041044FEA430594EA050F08BF90EA020F4D
:100208001FBF54EA000C55EA020C7FEA645C7FEADF
:10021800655C00F0E2804FEA5454D4EB5555B8BF02
:100228006D420CDD2C4480EA020281EA030382EA73
:10023800000083EA010180EA020281EA0303362D05
:1002480088BF30BD11F0004F4FEA01314FF4801CD8
:100258004CEA113102D0404261EB410113F0004FEA
:100268004FEA03334CEA133302D0524263EB4303A1
:1002780094EA050F00F0A780A4F10104D5F1200E3F
:100288000DDB02FA0EFC22FA05F2801841F100019A
:1002980003FA0EF2801843FA05F359410EE0A5F16E
:1002A80020050EF1200E012A03FA0EFC28BF4CF09F
:1002B800020C43FA05F3C01851EBE37101F0004555
:1002C80007D54FF0000EDCF1000C7EEB00006EEB62
:1002D8000101B1F5801F1BD3B1F5001F0CD34908EC
:1002E8005FEA30004FEA3C0C04F101044FEA445243
:1002F80012F5800F80F09A80BCF1004F08BF5FEACA
:10030800500C50F1000041EB045141EA050130BDA9
:100318005FEA4C0C404141EB0101013C28BFB1F5BB
:10032800801FE9D291F0000F04BF01460020B1FA06
:1003380081F308BF2033A3F10B03B3F120020CDAD9
:100348000C3208DD02F1140CC2F10C0201FA0CF0B7
:1003580021FA02F10CE002F11402D8BFC2F1200C1C
:1003680001FA02F120FA0CFCDCBF41EA0C019040D2
:10037800E41AA2BF01EB0451294330BD6FEA04041B
:100388001F3C1CDA0C340EDC04F11404C4F1200206
:1003980020FA04F001FA02F340EA030021FA04F318
:1003A80045EA030130BDC4F10C04C4F1200220FA6F
:1003B80002F001FA04F340EA0300294630BD21FAAD
:1003C80004F0294630BD94F0000F83F4801306BF73
:1003D80081F480110134013D4EE77FEA645C18BF67
:1003E8007FEA655C29D094EA050F08BF90EA020FFE
:1003F80005D054EA000C04BF1946104630BD91EAF6
:10040800030F1EBF0021002030BD5FEA545C05D1F8
:100418004000494128BF41F0004130BD14F5800437
:100428003CBF01F5801130BD01F0004545F0FE41AB
:1004380041F470014FF0000030BD7FEA645C1ABFE0
:10044800194610467FEA655C1CBF0B46024650EA17
:10045800013406BF52EA033591EA030F41F4002143
:1004680030BD00BF90F0000F04BF0021704730B5C9
:100478004FF4806404F132044FF000054FF000019E
:1004880050E700BF90F0000F04BF0021704730B55F
:100498004FF4806404F1320410F0004548BF404234
:1004A8004FF000013EE700BF42004FEAE2014FEA89
:1004B80031014FEA02701FBF12F07F4393F07F4F64
:1004C80081F06051704732F07F4208BF704793F067
:1004D8007F4F04BF41F40021704730B54FF460747A
:1004E80001F0004521F000411CE700BF50EA01027D
:1004F80008BF704730B54FF000050AE050EA010226
:1005080008BF704730B511F0004502D5404261EB95
:1005180041014FF4806404F132045FEA915C3FF4D6
:10052800D8AE4FF003025FEADC0C18BF03325FEA73
:10053800DC0C18BF033202EBDC02C2F1200300FA24
:1005480003FC20FA02F001FA03FE40EA0E0021FA49
:1005580002F11444BDE600BF4FF0FF3C06E000BFC7
:100568004FF0010C02E000BF4FF0010C4DF804CD34
:100578004FEA410C7FEA6C5C4FEA430C18BF7FEAF4
:100588006C5C1BD001B050EA410C0CBF52EA430C22
:1005980091EA030F02BF90EA020F0020704710F1A2
:1005A800000F91EA030F58BF994208BF90422CBF31
:1005B800D8176FEAE37040F0010070474FEA410C2A
:1005C8007FEA6C5C02D150EA013C07D14FEA430C48
:1005D8007FEA6C5CD6D152EA033CD3D05DF8040BB9
:1005E800704700BF8446104662468C4619466346EB
:1005F80000E000BF01B5FFF7B7FF002848BF10F1C2
:10060800000F01BD4DF808EDFFF7F4FF0CBF012006
:1006180000205DF808FB00BF4DF808EDFFF7EAFF82
:1006280034BF012000205DF808FB00BF4DF808ED3D
:10063800FFF7E0FF94BF012000205DF808FB00BF32
:100648004DF808EDFFF7CEFF94BF012000205DF8BC
:1006580008FB00BF4DF808EDFFF7C4FF34BF0120C9
:1006680000205DF808FB00BF4FEA410C7FEA6C5C94
:1006780002D150EA013C0AD14FEA430C7FEA6C5C94
:1006880002D152EA033C02D14FF0000070474FF00C
:10069800010070474FEA410212F5001215D211D538
:1006A8006FF47873B3EB625212D94FEAC12343F067
:1006B800004343EA505311F0004F23FA02F018BFE9
:1006C800404270474FF00000704750EA013005D1B2
:1006D80011F0004008BF6FF0004070474FF0000075
:1006E800704700BF4FEA4102B2F1E04324BFB3F5BF
:1006F800001CDCF1FE5C0DD901F0004C4FEAC00291
:100708004CEA5070B2F1004F40EB830008BF20F074
:100718000100704711F0804F21D113F13872BCBF2E
:1007280001F00040704741F480114FEA5252C2F183
:100738001802C2F1200C10FA0CF320FA02F018BFCC
:1007480040F001004FEAC1234FEAD32303FA0CFC1F
:1007580040EA0C0023FA02F34FEA4303CCE77FEAAE
:10076800625307D150EA01331EBF4FF0FE4040F4F8
:100778004000704701F0004040F0FE4040F40000A7
:10078800704700BF80F0004002E000BF81F00041E8
:1007980042001FBF5FEA410392EA030F7FEA226C1F
:1007A8007FEA236C6AD04FEA1262D2EB1363C1BFAF
:1007B800D218414048404140B8BF5B42192B88BF1E
:1007C800704710F0004F40F4000020F07F4018BF41
:1007D800404211F0004F41F4000121F07F4118BF61
:1007E800494292EA030F3FD0A2F1010241FA03FC09
:1007F80010EB0C00C3F1200301FA03F100F00043F1
:1008080002D5494260EB4000B0F5000F13D3B0F1B8
:10081800807F06D340084FEA310102F10102FE2A27
:1008280051D2B1F1004F40EBC25008BF20F0010097
:1008380040EA03007047490040EB0000013A28BF36
:10084800B0F5000FEDD2B0FA80FCACF1080CB2EBB9
:100858000C0200FA0CF0AABF00EBC2505242184337
:10086800BCBFD0401843704792F0000F81F40001DC
:1008780006BF80F400000132013BB5E74FEA4103AF
:100888007FEA226C18BF7FEA236C21D092EA030F1B
:1008980004D092F0000F08BF0846704790EA010F95
:1008A8001CBF0020704712F07F4F04D1400028BFC2
:1008B80040F00040704712F100723CBF00F50000A4
:1008C800704700F0004343F0FE4040F400007047DA
:1008D8007FEA226216BF08467FEA23630146420286
:1008E80006BF5FEA412390EA010F40F48000704799
:1008F8004FF0000304E000BF10F0004348BF40423F
:100908005FEA000C08BF704743F0964301464FF07A
:1009180000001CE050EA010208BF70474FF00003D6
:100928000AE000BF50EA010208BF704711F0004317
:1009380002D5404261EB41015FEA010C02BF8446E7
:100948000146002043F0B64308BFA3F18053A3F546
:100958000003BCFA8CF2083AA3EBC25310DB01FA8D
:1009680002FC634400FA02FCC2F12002BCF1004F11
:1009780020FA02F243EB020008BF20F001007047A2
:1009880002F1200201FA02FCC2F1200250EA4C00F6
:1009980021FA02F243EB020008BF20EADC7070473C
:1009A8004FF0FF0C1CEAD0521EBF1CEAD15392EA4A
:1009B8000C0F93EA0C0F6FD01A4480EA010C400226
:1009C80018BF5FEA41211ED04FF0006343EA501080
:1009D80043EA5111A0FB01310CF00040B1F5000FC2
:1009E8003EBF490041EAD3715B0040EA010062F171
:1009F8007F02FD2A1DD8B3F1004F40EBC25008BF5B
:100A080020F00100704790F0000F0CF0004C08BF78
:100A180049024CEA502040EA51207F3AC2BFD2F145
:100A2800FF0340EAC250704740F400004FF0000353
:100A3800013A5DDC12F1190FDCBF00F0004070478D
:100A4800C2F10002410021FA02F1C2F1200200FACB
:100A580002FC5FEA310040F1000053EA4C0308BF92
:100A680020EADC70704792F0000F00F0004C02BFE3
:100A7800400010F4000F013AF9D040EA0C0093F05E
:100A8800000F01F0004C02BF490011F4000F013BB8
:100A9800F9D041EA0C018FE70CEAD15392EA0C0F26
:100AA80018BF93EA0C0F0AD030F0004C18BF31F091
:100AB800004CD8D180EA010000F00040704790F067
:100AC800000F17BF90F0004F084691F0000F91F00B
:100AD800004F14D092EA0C0F01D142020FD193EAD1
:100AE8000C0F03D14B0218BF084608D180EA010059
:100AF80000F0004040F0FE4040F40000704740F035
:100B0800FE4040F4400070474FF0FF0C1CEAD05202
:100B18001EBF1CEAD15392EA0C0F93EA0C0F69D05E
:100B2800A2EB030280EA010C49024FEA402037D0C9
:100B38004FF0805343EA111143EA10130CF00040C0
:100B48008B4238BF5B0042F17D024FF4000C8B42B0
:100B580024BF5B1A40EA0C00B3EB510F24BFA3EB90
:100B6800510340EA5C00B3EB910F24BFA3EB910360
:100B780040EA9C00B3EBD10F24BFA3EBD10340EABA
:100B8800DC001B0118BF5FEA1C1CE0D1FD2A3FF600
:100B980050AF8B4240EBC25008BF20F001007047B5
:100BA8000CF0004C4CEA50207F32C2BFD2F1FF0358
:100BB80040EAC250704740F400004FF00003013A89
:100BC80037E792F0000F00F0004C02BF400010F42D
:100BD800000F013AF9D040EA0C0093F0000F01F041
:100BE800004C02BF490011F4000F013BF9D041EA63
:100BF8000C0195E70CEAD15392EA0C0F08D1420296
:100C08007FF47DAF93EA0C0F7FF470AF084676E768
:100C180093EA0C0F04D14B023FF44CAF08466EE741
:100C280030F0004C18BF31F0004CCAD130F000420F
:100C38007FF45CAF31F000437FF43CAF5FE700BF67
:100C48004FF0FF3C06E000BF4FF0010C02E000BF90
:100C58004FF0010C4DF804CD4FEA40024FEA410332
:100C68007FEA226C18BF7FEA236C11D001B052EAE8
:100C7800530C18BF90EA010F58BFB2EB030088BFAE
:100C8800C81738BF6FEAE17018BF40F0010070471D
:100C98007FEA226C02D15FEA402C05D17FEA236CFF
:100CA800E4D15FEA412CE1D05DF8040B704700BF46
:100CB800844608466146FFE70FB5FFF7C9FF0028DD
:100CC80048BF10F1000F0FBD4DF808EDFFF7F4FF16
:100CD8000CBF012000205DF808FB00BF4DF808EDAF
:100CE800FFF7EAFF34BF012000205DF808FB00BFD2
:100CF8004DF808EDFFF7E0FF94BF012000205DF8F4
:100D080008FB00BF4DF808EDFFF7D2FF94BF0120A4
:100D180000205DF808FB00BF4DF808EDFFF7C8FF9D
:100D280034BF012000205DF808FB00BF80EA010CF9
:100D38001CF0030F37D110F0030C20F0030021F052
:100D4800030150F8042B08BF51F8043B0ED08CF077
:100D5800030C6FF07F434FEACC0C23FA0CFC51F8DC
:100D6800043B42EA0C0243EA0C0300BFA2F1013C37
:100D78009A4201BF2CEA020C1CF0803F50F8042B69
:100D880051F8043BF2D04FEA02604FEA12220128E0
:100D980028BFB0EB036F08BF1B0AF4D003F0FF03B2
:100DA800000EC01A704710F0030F0AD010F8012B7C
:100DB80011F8013B012A28BF9A42F4D0A2EB0300A4
:100DC80070474DF8045D50F8042B01F0030521F03D
:100DD800030151F8043B022D26D04DD822F07F455F
:100DE800B5EB132FA2F1013C2CEA020C0DD11CF03B
:100DF800803C08BF51F8043B0AD185EA0205B5EBEF
:100E0800036F0CD150F8042BE8E74FEA13235BE09B
:100E18003CF07F4C54D10B784FEA126554E04FEA0E
:100E2800126503F0FF034FE04FEA0245A2F1013CCF
:100E38004FEA15452CEA020CB5EB134F18D11CF0FC
:100E4800803C08BF51F8043B07D185EA0205B5EBA1
:100E5800034F09D150F8042BE6E75FEA0C4C2FD179
:100E68000B884FEA12452FE04FEA03434FEA124539
:100E78004FEA134328E000BF02F0FF05B5EB136FFC
:100E8800A2F1013C2CEA020C0DD11CF0803C08BFF9
:100E980051F8043B0AD185EA0205B5EB032F0AD1C4
:100EA80050F8042BE8E74FEA13630DE012F0FF0F48
:100EB80006D051F8043B4FEA122523F07F4303E0A4
:100EC8004FF0000020BC704705F0FF0203F0FF0060
:100ED800012828BF904204BF2D0A1B0AF4D0A2EBB8
:100EE800000020BC704700BF844641EA000313F0AD
:100EF800030349D1403A23D30B6803604B6843602E
:100F08008B688360CB68C3600B6903614B6943617D
:100F18008B698361CB69C3610B6A03624B6A436265
:100F28008B6A8362CB6AC3620B6B03634B6B43634D
:100F38008B6B8363CB6BC36340304031403ADBD269
:100F480030320BD30B6803604B6843608B68836057
:100F5800CB68C36010301031103AF3D20C3205D38D
:100F680051F8043B40F8043B043AF9D2043208D063
:100F7800D2071CBF11F8013B00F8013B01D30B88D5
:100F880003806046704700BF082A13D38B07B1D08F
:100F980010F00303AED0C3F10403D21ADB071CBF61
:100FA80011F8013B00F8013BA4D331F8023B20F8CB
:100FB800023B9FE7043AD9D3013A11F8013B00F804
:100FC800013BF9D20B7803704B7843708B788370B0
:100FD8006046704770B54FF0FF0C4CF4E06C1CEAAB
:100FE80011541DBF1CEA135594EA0C0F95EA0C0F17
:100FF80000F0DEF82C4481EA030621EA4C5123EA8A
:101008004C5350EA013518BF52EA033541F48011B8
:1010180043F4801338D0A0FB02CE4FF00005E1FB6B
:1010280002E506F00042E0FB03E54FF00006E1FBB5
:1010380003569CF0000F18BF4EF0010EA4F1FF04F8
:10104800B6F5007F64F5407404D25FEA4E0E6D4138
:1010580046EB060642EAC62141EA55514FEAC52049
:1010680040EA5E504FEACE2EB4F1FD0C88BFBCF5C5
:10107800E06F1ED8BEF1004F08BF5FEA500E50F176
:10108800000041EB045170BD06F0004646EA01013C
:1010980040EA020081EA0301B4EB5C04C2BFD4EB6E
:1010A8000C0541EA045170BD41F480114FF0000E67
:1010B800013C00F3AB8014F1360FDEBF002001F0D5
:1010C800004170BDC4F10004203C35DA0C341BDC4F
:1010D80004F11404C4F1200500FA05F320FA04F021
:1010E80001FA05F240EA020001F0004221F0004155
:1010F80010EBD37021FA04F642EB06015EEA430EC8
:1011080008BF20EAD37070BDC4F10C04C4F12005F7
:1011180000FA04F320FA05F001FA04F240EA0200AA
:1011280001F0004110EBD37041F100015EEA430E7B
:1011380008BF20EAD37070BDC4F1200500FA05F29B
:101148004EEA020E20FA04F301FA05F243EA02031A
:1011580021FA04F001F0004121FA04F220EA020029
:1011680000EBD3705EEA430E08BF20EAD37070BD6F
:1011780094F0000F0FD101F00046400041EB01014F
:1011880011F4801F08BF013CF7D041EA060195F031
:10119800000F18BF704703F00046520043EB0303EB
:1011A80013F4801F08BF013DF7D043EA06037047D8
:1011B80094EA0C0F0CEA135518BF95EA0C0F0CD0E3
:1011C80050EA410618BF52EA4306D1D181EA030129
:1011D80001F000414FF0000070BD50EA410606BF23
:1011E8001046194652EA430619D094EA0C0F02D168
:1011F80050EA013613D195EA0C0F05D152EA0336AD
:101208001CBF104619460AD181EA030101F00041CA
:1012180041F0FE4141F470014FF0000070BD41F013
:10122800FE4141F4780170BD70B54FF0FF0C4CF4ED
:10123800E06C1CEA11541DBF1CEA135594EA0C0F0C
:1012480095EA0C0F00F0A7F8A4EB050481EA030E59
:1012580052EA03354FEA013100F088804FEA033340
:101268004FF0805545EA131343EA12634FEA02220E
:1012780045EA111545EA10654FEA00260EF00041CF
:101288009D4208BF964244F1FD0404F5407402D221
:101298005B084FEA3202B61A65EB03055B084FEAB2
:1012A80032024FF480104FF4002CB6EB020E75EBAF
:1012B800030E22BFB61A754640EA0C005B084FEAD7
:1012C8003202B6EB020E75EB030E22BFB61A754654
:1012D80040EA5C005B084FEA3202B6EB020E75EB9F
:1012E800030E22BFB61A754640EA9C005B084FEA17
:1012F8003202B6EB020E75EB030E22BFB61A754624
:1013080040EADC0055EA060E18D04FEA051545EA12
:1013180016754FEA06164FEAC30343EA52734FEABB
:10132800C2025FEA1C1CC0D111F4801F0BD141EA34
:1013380000014FF000004FF0004CB6E711F4801F99
:1013480004BF01430020B4F1FD0C88BFBCF5E06F79
:101358003FF6AFAEB5EB030C04BFB6EB020C5FEA89
:10136800500C50F1000041EB045170BD0EF0004EDE
:101378004EEA113114EB5C04C2BFD4EB0C0541EA10
:10138800045170BD41F480114FF0000E013C90E60D
:1013980045EA060E8DE60CEA135594EA0C0F08BFD1
:1013A80095EA0C0F3FF43BAF94EA0C0F0AD150EAD0
:1013B80001347FF434AF95EA0C0F7FF425AF104663
:1013C80019462CE795EA0C0F06D152EA03353FF48B
:1013D800FDAE1046194622E750EA410618BF52EA08
:1013E80043067FF4C5AE50EA41047FF40DAF52EADC
:1013F80043057FF4EBAE12E74A0011D212F5001252
:1014080011D20DD56FF47873B3EB62520ED44FEA54
:10141800C12343F0004343EA505323FA02F07047D4
:101428004FF00000704750EA013002D14FF0FF3012
:1014380070474FF00000704753B94AB9002908BFF8
:1014480000281CBF4FF0FF314FF0FF3000F00CB800
:10145800ADF1080C6DE904CE18F08AFFDDF804E060
:10146800DDE9022304B07047704700BF0348044B0E
:10147800834202D0034B03B118477047F40700209A
:10148800F4070020000000000548064B1B1AD90F7E
:1014980001EBA301491002D0034B03B11847704771
:1014A800F4070020F40700200000000010B5064CE7
:1014B800237843B9FFF7DAFF044B13B10448AFF3BD
:1014C80000800123237010BDF407002000000000F5
:1014D8002CA6010808B5054B1BB105490548AFF313
:1014E8000080BDE80840FFF7CFBF00BF0000000044
:1014F800F80700202CA6010800B583B00A4B5A69EA
:1015080042F001025A615B6903F001030193019BF8
:10151800002211460F2003F0B9FA0F2003F0C6FA93
:1015280003B05DF804FB00BF0010024030B587B07F
:1015380000230293039304930593134B1B680BB189
:1015480007B030BD104B01221A60104B5A6942F4A3
:1015580080725A615B6903F480730193019B4FF6B3
:1015680080730293022503950324059402A9084871
:1015780003F0A8FD4CF6B37302930395059402A9F2
:10158800044803F09FFDDBE710080020001002402C
:10159800001801400014014010B588B000220192E3
:1015A80002920392049205920692079216484FF00F
:1015B8002043036003F5827343608260C260026166
:1015C800102141618261C261026242624FF480531C
:1015D8008362C2620263426382630F2301930293B0
:1015E800FF240394049305911123069301A906F09F
:1015F80078FB30B9054AD36943F48063D36108B0F6
:1016080010BD00F009F9F5E71408002000000140BA
:1016180008B5FFF78BFF08BD2DE9F0478AB0002415
:1016280006940794089409944B4B9A6942F0100267
:101638009A619A6902F010020192019A9A6942F03D
:1016480004029A619A6902F004020292029A9A6963
:1016580042F008029A619A6902F008020392039A1A
:101668009A6942F040029A619A6902F04002049233
:10167800049A9A6942F020029A619B6903F0200358
:101688000593059BDFF8D4A001222021504603F0E2
:101698003CFEDFF8CC9001220421484603F035FED9
:1016A800304E22464FF40041304603F02EFE4FF0F4
:1016B8000908CDF818802C4B07930225089506A930
:1016C800304603F0FFFC12230693284B07930127AB
:1016D800089706A9304603F0F5FC202306930797E0
:1016E8000894099506A9504603F0ECFC04230693D8
:1016F80007970894099506A9484603F0E3FC4FF4B8
:101708000043069307970894099506A9304603F005
:10171800D9FC22462946062003F0B8F9062003F032
:10172800C5F922462946072003F0B0F9072003F03F
:10173800BDF922462946404603F0A8F9404603F081
:10174800B5F9224629460A2003F0A0F90A2003F039
:10175800ADF90AB0BDE8F087001002400010014062
:10176800000C014000080140000011100000211089
:1017780038B502680C4B9A4200D038BD0B4C204655
:1017880002F0EEFA78252A46002120460EF0FAF8F3
:101798002A462146064807F0F3F9064B1A681368EB
:1017A80023F004031360E8E70038014064080020D0
:1017B800AC0A0020200A002010B50446002200F1DF
:1017C8000C0105F0B1FC134BDB78E27B934204D1AA
:1017D800104B5978637B994215D00221204605F0B9
:1017E8008BFD627B0321204605F086FDA27B042148
:1017F800204605F081FDE27B064BDA70627B5A7069
:10180800A27B9A7010BD034B9978A37B9942E4D1CF
:10181800F8E700BF5C08002072B6FEE700B597B095
:10182800282200210CA80EF0ADF800230793089396
:1018380009930A930B9301930293039304930593DB
:10184800069309230C934FF480330D9301221092D1
:1018580012920222139214934FF4E01315930CA8DA
:1018680004F0B6FDD8B90F2307930221089100238D
:1018780009934FF480620A920B9307A804F0DAFFE9
:1018880078B9112301934FF4007302930023069350
:1018980001A805F0ABF830B917B05DF804FBFFF705
:1018A800BBFFFFF7B9FFFFF7B7FF000010B503F064
:1018B8006FF8FFF7B3FF264C204600F053F8FFF708
:1018C800ABFEFFF719FEFFF767FE00F0BFFA00F066
:1018D80015FB00F04FF900F02BFB08F0E9FC0BF0CA
:1018E80071FE00F0AFF800F099F900F0B3FE78222D
:1018F8001849204607F044F9174B1A68136823F073
:101908000403136015480DF04DFE02F01BFB02F0B6
:1019180013FE00240EE002F061FC78B90134E4B251
:101928004FF6FF7000F018FC0D4B00221A7005E00E
:1019380002F0B8FB0A4B1B78022BECD0002CF7D036
:10194800012C01D00024F5E702F04EFCF2E700BFBD
:10195800AC0A002064080020200A002048A60108DC
:101968006008002008B5054B1860054B186800236F
:101978000222194680680DF01DFE08BDE00800200F
:10198800C8060020022801D80120704708B50EF0CB
:1019980017FB09230360002008BD000010B50138BB
:1019A80001280AD814464FF0FF3392B2074800685E
:1019B80006F07AFD40B9204610BD0EF001FB092360
:1019C80003604FF0FF30F7E70520F5E7E008002057
:1019D800022801D80020704708B50EF0F1FA092353
:1019E80003604FF0FF3008BD08B50EF0E9FA09238F
:1019F80003604FF0FF3008BD08B548B94FF0FF331A
:101A080001220848006806F0AEFD40B9012008BD73
:101A18000EF0D6FA092303604FF0FF30F7E70520F0
:101A2800F5E700BFE008002008B5022804D84FF405
:101A380000534B60002008BD0EF0C2FA0923036072
:101A4800F8E7000010B582B00023ADF804308DF837
:101A5800063000932D482E4B03604FF0FF33436050
:101A68004FF48073836005F0CBFB78BB274802688E
:101A7800136843F001031360012105F045FC41F2AE
:101A88003423984225D000228DF804208DF80520B3
:101A98008DF8062001A91D4805F0F5F978BB01234A
:101AA8008DF800308DF801308DF8023000228DF865
:101AB80003206946154805F0CDFA18BB41F23422D7
:101AC8000121124805F018FC02B010BDFFF7A4FE72
:101AD800CCE70E4C0221204605F016FCE0730321EA
:101AE800204605F011FC60730421204605F00CFC2B
:101AF800A073002201A9204605F026FAE4E7FFF7C3
:101B08008BFECCE7FFF788FED8E700BFE40800208B
:101B1800002800400268144B9A4200D0704700B574
:101B280083B004F039FC114BDA6942F00062DA61E3
:101B3800DB6903F000630193019B0D4B0122C3F89D
:101B48003C2400220321084602F0A0FF032002F0F3
:101B5800ADFF00220321292002F098FF292002F07E
:101B6800A5FF03B05DF804FB002800400010024008
:101B780000004242054B064A1A6000225A609A60E9
:101B8800DA601A615A6104229A617047F8080020E5
:101B98000080014030B589B0002304930593069373
:101BA800079302681A4B9A4201D009B030BD03F579
:101BB80010435A6942F480625A615A6902F4806299
:101BC8000192019A9A6942F010029A619A6902F0A8
:101BD80010020292029A9A6942F020029A619B6965
:101BE80003F020030393039B4FF4885304930225C7
:101BF80005950324079404A9064803F063FA04230F
:101C080004930595079404A9034803F05BFACCE70D
:101C180000800140001001400014014008B50E4842
:101C28000E4B03604FF48273436000238360C360EC
:101C3800036143614FF4007282610822C26103624A
:101C4800436283620A23C36205F0F0FF00B908BD4E
:101C5800FFF7E2FDFBE700BF7C09002000300140F0
:101C680010B586B00023029303930493059302688A
:101C7800164B9A4201D006B010BD03F560439A692D
:101C880042F480529A619A6902F480520092009A52
:101C98009A6942F004029A619B6903F00403019374
:101CA800019BA02302930223039303230593084C6B
:101CB80002A9204603F006FA402302930023039367
:101CC800049302A9204603F0FDF9D4E7003001404F
:101CD8000008014000B583B0124B9A6942F0010236
:101CE8009A619A6902F001020092009ADA6942F058
:101CF8008052DA61DB6903F080530193019B002273
:101D08001146052002F0C2FE052002F0CFFE064A69
:101D1800536823F0E06343F00073536003B05DF849
:101D280004FB00BF0010024000000140FEE7FEE790
:101D3800FEE7FEE7FEE770477047704708B502F018
:101D480039FE08BD08B5024805F0B3FA08BD00BF62
:101D5800E4080020704708B5012003F0DDFA08BD4B
:101D680008B5022003F0D8FA08BD08B5082003F02A
:101D7800D3FA08BD08B5102003F0CEFA08BD00005C
:101D880008B5024803F028F808BD00BF200A002063
:101D980008B5024804F0C2F808BD00BFFC1B0020CB
:101DA80008B5024806F055F808BD00BFD80900205C
:101DB80008B5024806F0F4FC08BD00BFAC0A0020D4
:101DC80008B5024806F0ECFC08BD00BF640A002014
:101DD80008B5024805F0DCF908BD00BFE40800209A
:101DE8000120704708B50EF0EBF8162303604FF09A
:101DF800FF3008BD08B54FF0FF31FFF7F3FFFEE7EE
:101E080010B503460C4A0D490D48006840B10C480E
:101E180000680344521A934206D8094A136010BD59
:101E28000748084C0460F2E70EF0CAF80C23036078
:101E38004FF0FF30F3E700BF00000120000400006E
:101E4800D4090020002200207047000000B587B0A8
:101E58000023029303930493059300930193154879
:101E6800154A026047224260836040F2E732C2604E
:101E78000361836106F0F6F890B94FF4805302933A
:101E880002A90C4806F026F968B9002300930193CB
:101E98006946084806F09EF940B907B05DF804FBAA
:101EA800FFF7BAFCE9E7FFF7B7FCEEE7FFF7B4FC8A
:101EB800F3E700BFD80900200008004002680E4B75
:101EC8009A4200D0704700B583B003F50233DA694F
:101ED80042F00402DA61DB6903F004030193019B19
:101EE800002201211E2002F0D1FD1E2002F0DEFD9D
:101EF80003B05DF804FB00BF0008004008B50A48BD
:101F08000A4B03604FF4E133436000238360C360EE
:101F180003610C2242618361C36106F095FA00B93E
:101F280008BDFFF779FCFBE7AC0A00200038014048
:101F380008B50A480A4B03604FF4E13343600023B5
:101F48008360C36003610C2242618361C36106F050
:101F58007BFA00B908BDFFF75FFCFBE7640A0020C5
:101F68000048004070B588B0002304930593069399
:101F780007930368404A934204D0404A934248D0AA
:101F880008B070BD04463E4B9A6942F480429A619B
:101F98009A6902F480420092009A9A6942F0040217
:101FA8009A619B6903F004030193019B4FF400734A
:101FB80004930223059303230793324E04A9304662
:101FC80003F080F84FF48063049300250595069587
:101FD80004A9304603F076F82B482C4B0360456083
:101FE80085608023C360056145618561C56102F034
:101FF80095FD58B9244BE3635C6200220221252039
:1020080002F044FD252002F051FDB9E7FFF704FC7A
:10201800F0E71B4BDA6942F48022DA61DA6902F4EC
:1020280080220292029A9A6942F008029A619B6998
:1020380003F008030393039B4FF480630493022384
:10204800059303250795124E04A9304603F03AF884
:102058004FF40063049300240594069404A93046C1
:1020680003F030F822462946272002F00FFD2720EA
:1020780002F01CFD84E700BF003801400048004022
:102088000010024000080140200A002058000240C9
:10209800000C0140034B044A1A60044B023A1A60D0
:1020A800704700BF081000200000026004100020E4
:1020B8000B4B2A225A812B229A812C221A81002228
:1020C8009A71F0221A804FF4A0725A80054B1B684F
:1020D80036221A80044B1B6808221A80704700BFFA
:1020E800F40F0020041000200810002070B5174ECF
:1020F8003468174DB5F80AC0A4F800C0154C4FEA6B
:10210800102CD4F800E0AEF800C0C0B2D4F800C07B
:10211800ACF8000020684FEA122CA0F800C0206834
:10212800D2B202803268A88910802268080A10801A
:102138002268C9B211802268190A11802268DBB2AC
:10214800138033682A891A8070BD00BF04100020EC
:10215800F40F00200810002010B504460A4B1A8816
:102168005B88013B013A9BB292B200210846FFF717
:10217800BDFF002303E0054A126814800133B3F55C
:10218800963FF8D310BD00BFF40F002008100020C0
:102198000020704700207047002070472DE9F84361
:1021A8008046894616461F46BDF82050BDF8244093
:1021B8001EE0194A12681580013B002B08DB41FA22
:1021C80003F212F0010FF4D0134A12681480F3E7F7
:1021D80002301F2806DC335C3218517841EA0321AB
:1021E8000F23EAE708F110082036B8F1E00F11DCF8
:1021F8003B46013FBFB26BB11FFA88F01FFA89F165
:1022080001F10F0300F10F029BB292B2FFF76EFFCC
:102218000020DEE7BDE8F883081000202DE9F84328
:102228008046894616461F46BDF82050BDF8244012
:102238001AE0174A12681580013B002B08DB41FAA7
:1022480003F212F0010FF4D0114A12681480F3E778
:102258000130472802DC315C0723EEE708F1180853
:102268004836B8F1D80F11DC3B46013FBFB26BB11D
:102278001FFA88F01FFA89F101F1170300F117021C
:102288009BB292B2FFF732FF0020E2E7BDE8F88385
:10229800081000202DE9F8438046894616461F4657
:1022A800BDF82050BDF824401AE0174A126815807E
:1022B800013B002B08DB41FA03F212F0010FF4D0C6
:1022C800114A12681480F3E701307F2802DC315C80
:1022D8000723EEE708F120088036B8F1D00F11DCAB
:1022E8003B46013FBFB26BB11FFA88F01FFA89F174
:1022F80001F11F0300F11F029BB292B2FFF7F6FE35
:102308000020E2E7BDE8F883081000202DE9F04737
:1023180007468A4690461D46BDF8206010460DF0D7
:1023280093FE5FFA80F900242DE0B8B21FFA8AF113
:10233800CB1D421D9BB292B2FFF7D8FE18F80400DD
:102348002038C000002111E0144B1B681D800CF1DF
:10235800FF3CBCF1010F08DD42FA0CF313F0010F4A
:10236800F2D00E4B1B681E80F1E70131072905DC0E
:1023780043180B4AD25C4FF0070CEAE70637E92FFF
:102388000ADC0134E4B24C4506D218F90430002BBB
:10239800CBDA0134E4B2F1E7BDE8F0870810002099
:1023A800F8DD01082DE9F04F83B007468A469046CC
:1023B8001C46BDF8305010460DF046FE5FFA80F915
:1023C800002633E0B8B21FFA8AF101F10F03C21DEB
:1023D8009BB292B2FFF78AFE18F806002038000177
:1023E800002116E0234B1B681C800CF1010C1FFA1E
:1023F8008CFCBCF1070F0AD8CCF1070342FA03F3AF
:1024080013F0010FEED01B4B1B681D80EDE7013167
:1024180089B20F2905D84318174AD25C4FF0000C2F
:10242800E7E708370136F6B2E82F20DC4E451ED222
:1024380008EB060118F90630002BC3DA14220F48FE
:10244800FFF7A6FE834610B90236F6B2ECE701950F
:102458000094C0F34F13094A51463846FFF79EFED1
:1024680007EB5B0706EB1B1B5FFA8BF6DCE703B099
:10247800BDE8F08F0810002008D80108F40A0020F1
:102488002DE9F04F85B08046039191461C46BDF872
:10249800385010460DF0D8FD5FFA80FB002637E073
:1024A8001FFA88F0BDF80C1001F1170300F10B02B8
:1024B8009BB292B2FFF71AFE19F80630203B03EBE5
:1024C8004303284F07EB0317002011E0264A126840
:1024D8001480013B9BB2032B08D941FA03F212F096
:1024E800010FF3D0204A12681580F2E7023080B25B
:1024F8002F2806D83B5C3A18517841EA03210F236C
:10250800E9E708F10C080136F6B2B8F1E40F26DC69
:102518005E4524D209EB060119F90630002BBFDA13
:1025280014221248FFF736FE074610B90236F6B2F3
:10253800EBE70F4BA3FB003A01950094CAF30F1386
:102548000A4A03994046FFF769FE0A4BA3FB07377F
:1025580008EB570806EBDA0A5FFA8AF6D5E705B002
:10256800BDE8F08F68C6010808100020F40A0020B2
:10257800398EE338ABAAAAAA2DE9F04F83B080467A
:102588008B4617461C46BDF8305010460DF05CFDD2
:102598005FFA80F9002634E01FFA88F01FFA8BF101
:1025A80001F11F0300F10F029BB292B2FFF79EFDEB
:1025B800BB5D203B244A02EB831C00200FE0234A2A
:1025C80012681480013B002B08DB41FA03F212F079
:1025D800010FF4D01D4A12681580F3E702303F2836
:1025E80008DC1CF800300CEB0002517841EA0321AA
:1025F8000F23E8E708F110080136F6B2B8F1E40F46
:102608001EDC4E451CD2B919BB57002BC4DA142264
:102618000F48FFF7C1FD824610B90236F6B2EDE762
:1026280001950094C0F3CF13094A59464046FFF775
:1026380031FE08EB9A0806EB9A1A5FFA8AF6DDE78C
:1026480003B0BDE8F08F00BFE8AE01080810002015
:10265800F40A00202DE9F04F83B0FFF71BFDA64DCB
:102668002B68CF221A80A54B1A68002414801A6898
:10267800C9211180196830220A802968ED20088054
:1026880019686420088019680320088019681220D6
:1026980008801968812008802968E820088019685E
:1026A80085200880196810270F8019687A2008800B
:1026B8002968CB20088019683920088019682C20DF
:1026C800088019680C80196834200880196802206D
:1026D80008802968F720088019684FF02009A1F8B8
:1026E80000902968EA20088019680C8019680C8015
:1026F8002968C020088019681B2008802968C12023
:10270800088019680C802968C520088019680A8023
:1027180019680A802A68C72111801A68B7211180B0
:102728002A684FF03608A2F800801A680826168032
:102738002A683A2111801A68552111802A68B12126
:1027480011801A6814801A681A2111802A68B62123
:1027580011801A680A2111801A68A22010802A683C
:10276800F22010801A6814802A68262010801A68BF
:102778004FF0010EA2F800E02A68E02010801868E7
:102788000F22028018684FF02A0AA0F800A01868E3
:102798004FF0280CA0F800C01868068018684FF0A1
:1027A8000E0CA0F800C01868068018684FF0540C8A
:1027B800A0F800C018684FF0A90CA0F800C018686D
:1027C8004FF0430CA0F800C01868018019680A800F
:1027D80019680C8019680C8019680C8019680C80BD
:1027E8002968E120088019680C801968152008807C
:1027F80019681720088019680720088019684FF0A1
:10280800110BA1F800B019680620088019684FF06C
:102818002B0CA1F800C019685620088019683C20C4
:10282800088019680520088019680F8019680A80CF
:1028380018683F21018018680180186802802A689A
:10284800A2F800C01A6814801A6814801A68A2F8DE
:1028580000E01A6811802A68A2F800A01A6814809B
:102868001A6814801A6814801B68EF221A802B6873
:10287800A3F800B0782002F0AFF82B6829221A805C
:10288800FFF716FC1E4AD36843F40043D3604FF4A5
:102898007840FFF761FCC82002F09EF84FF4FC6016
:1028A800FFF75AFCC82002F097F81F20FFF754FCE6
:1028B800C82002F091F84FF6FF70FFF74DFCC820D2
:1028C80002F08AF84FF4784500954FF6FF730D4AE9
:1028D80021462046FFF766FDDFF82CA000954FF64D
:1028E800FF7352462146A020FFF710FD4FF6FF75F3
:1028F80000952346524609E00410002008100020E5
:10290800000801405CA6010874A601083146A02011
:10291800FFF7FCFC4FF4FC6300932B460C4A394646
:102928002046FFF73FFD1F2300932B46094A4946DF
:102938002046FFF7A5FD4BF6404300932B46064A79
:1029480041462046FFF718FE03B0BDE8F08F00BFF0
:1029580084A601089CA60108B4A60108FFF774FA2A
:102968000B480C490C4A002302E0D458C4500433E5
:10297800C4188C42F9D3094A094C002301E01360BA
:102988000432A242FBD30DF021FBFEF78FFF704704
:1029980000000020F40700207C500208F407002003
:1029A80000220020FEE7000020B3844621B38842BD
:1029B80024D000B50DE086460B78124AD25C02F0AE
:1029C8000302012A10D09E4510D1C8B10CF1010CA8
:1029D80001319CF800000B4B1B5C03F00303012B37
:1029E800E9D100F1200EE7E72033ECE7AEEB030076
:1029F8005DF804FB012070470120704700207047F4
:102A08000020F5E739E201082E2070472DE9F84F3C
:102A180082468B4614461D4621F00049164623F08F
:102A280000473B464946FDF715FE08B156464F4656
:102A380022462B4650465946FDF7D6FB044621F060
:102A480000450022084B30463946FEF7C3FA0246D5
:102A58000B46012620462946FDF7E8FD00B9002669
:102A68003046BDE8F88F00BF0000B03C8446002225
:102A780010460BE0A1F14103DBB2052B12D80B186D
:102A8800A3F13700022A00D800010132032A12D824
:102A98001CF80210A1F13003DBB2092BEAD8084474
:102AA8003038EFE7A1F16103DBB2052B04D80B182E
:102AB800A3F15700E6E7704700207047F8B50B1AF6
:102AC800052B61DD06460F4615460230FFF7CEFF9F
:102AD8000446A0F55C43B3F5806F57D3A0F558437F
:102AE800B3F5806F1CD2B31DFF1A052F50DDB379E3
:102AF8005C2B4FD1F379752B4ED106F10800FFF707
:102B0800B5FFA0F55C43B3F5806F47D2254B03EAC8
:102B18008423C0F30900034303F580340C2002E04A
:102B28007F280CD90620B4F5006F0ED3B4F5803F8A
:102B38000ED3B4F5881F33D2F027042602E006200E
:102B480000270126731EDBB20EE0C0270226F9E734
:102B5800E0270326F6E704F03F012A6841F08001E8
:102B6800D154A409013BDBB2002BF4D1012E06D9C4
:102B78002B6827431F702B6833442B6005E02B68B4
:102B880004F07F041C70F6E70020F8BD0020FCE785
:102B98000020FAE70020F8E70020F6E70020F4E735
:102BA8000020F2E700FC0F002DE9F04182B08046DA
:102BB8000E460F688B685D1C3D4400220192F81890
:102BC800FB5C222B43D12C46944600E00134E11BE8
:102BD800726891420BD22378222B08D05C2BF5D156
:102BE8000134E31B934232D20CF1010CEEE791421F
:102BF8002DD22378222B2AD1201AA0EB0C0033697E
:102C080001309847074610B3019030E0631B002B52
:102C18001ADD6B78752B17D85C2B11D35C3B192BFD
:102C280012D8DFE803F04C11111111111D11111107
:102C38003011111111111111371111113E11455394
:102C4800222B3CD02F2B3AD0736938469847002D59
:102C580054D03368ED1AB560002002B0BDE8F081A9
:102C6800019B5A1C019208221A7002231D44A54296
:102C780035D22B785C2BC9D0019B5A1C019215F8D0
:102C8800012B1A70F3E7019B5A1C01920C221A704F
:102C98000223EBE7019B5A1C01920A221A700223B5
:102CA800E4E7019B5A1C01920D221A700223DDE70A
:102CB800019B5A1C019209221A700223D6E7019B34
:102CC8005A1C01926A781A700223CFE701AA21469A
:102CD8002846FFF7F3FE03460028C7D1B4E7019B57
:102CE80000221A701023C8F80C30C8F81070336826
:102CF800E41AB4600134B4600120AEE70020ACE708
:102D08000246D0B110B40468ACB18368406883420D
:102D180002D30AE0013393609368984202D9E15CD8
:102D28002029F7D99368984202D0104610BC704702
:102D3800013B9360F9E72246F7E770470160486076
:102D48007047A1B138B504460D4690B1814212D002
:102D580083683BB1586880B1FFF7F0FFA3685D60F6
:102D6800012038BD816049600B600120F9E700202F
:102D780070470020F5E70020F3E70120F1E77047EE
:102D880050B138B50546006828B1AC6820440DF04C
:102D98005BF90444AC6038BD704770B5064670B145
:102DA8000D460DF051F9441C2B68204698470546FE
:102DB80018B122463146FEF797F8284670BD0546F9
:102DC800FBE768B32DE9F0410D4614461E46074659
:102DD80041B34AB3904229D0069BBBB10846FFF7DE
:102DE800CEFF8046E56845F40075E36813F4007F7C
:102DF80003D1206A08B173689847C4F82080E56059
:102E080021463846FFF79DFFBDE8F0813146284648
:102E1800FFF7C3FF804658B1E56825F40075E4E77D
:102E2800002070470020EFE70020EDE70020EBE7E7
:102E38000698E9E770B50546002846D0066836B317
:102E4800436813B18268934241D9002941DBAA68DB
:102E5800114401318B420AD22B69002B3BD1B1F1CD
:102E6800804F08D3002904DB6FF0004404E01644C7
:102E78000DE000260BE04C002B6A8BB12146304652
:102E88009847064628B16C602E60AB681E443046F1
:102E980070BDEB692868984700236B602B60F6E7E4
:102EA800AB6920469847064640B1AA6801322968AE
:102EB800FEF71AF8EB6928689847E4E7EB69286891
:102EC800984700236B602B60E1E70646DFE70026A2
:102ED800DDE70026DBE70026D9E710B503682820E0
:102EE8009847044618B1282200210CF04BFD2046D3
:102EF80010BD000038B5044678B1006878B1A568FF
:102F08007DB92B1D6268934207D2032206492844E3
:102F18000CF088FD08B90335A560204638BD044685
:102F2800FBE70024F9E700BFCCA601080000000079
:102F38002DE9F04393B005460C4600231193FFF7A3
:102F480063FD002C65D02368002B64D0002330E09B
:102F5800652A28D048336B44002203F8442C0DF12D
:102F6800040911A948460CF0C1F906460F46DDF8D8
:102F78004480C84551D0C5E9066729A3D3E9002391
:102F8800FDF75EFB002833D06FF000436B61082328
:102F9800EB60A36801AAA8EB02084344A3600120E0
:102FA80013B0BDE8F08303F14801694401F8442CEB
:102FB80001333E2BCED8A2681A4461688A42C9D22E
:102FC80021688A5C452AC3D82B2AC3D3A2F12B06D1
:102FD800F6B20121B140144E0E40002EE3D111F09B
:102FE800080FB7D003F148026A4402F8440CDFE73F
:102FF80000220E4B30463946FDF718FB18B14FF04A
:1030080000436B61C3E730463946FDF743FB68610F
:10301800BDE70020C4E70020C2E70020C0E700BFEA
:103028000000C0FFFFFFDF41E57F00040000E0C1B2
:10303800002900F09480F8B50546084615B12A46DF
:10304800002614E00321FFF7F5FE002800F0898030
:10305800464A118892780180827001207EE05C2BBC
:1030680003D01F2B02D8053600E001360132137851
:1030780063B1222BF3D8082BF3D3A3F10804E4B2ED
:103088003B49E14011F0010FEFD1EAE7521B9419D7
:10309800E11CFFF7CFFE0746002864D026B106469C
:1030A800222306F8013B30E0222600F8016B224675
:1030B8002946FDF719FF631CFE54023400233B55D3
:1030C80001204BE030465C2300F8013B2A78222A95
:1030D80015D8082A36D3A2F108031A2B32D8DFE80C
:1030E80003F0222E2831252B313131313131313164
:1030F8003131313131313131313131311F005C2AD7
:1031080020D15C2373700135461C2B78FBB11F2B33
:10311800D8D9222BD6D05C2BD4D033703046F2E7E6
:1031280022237370EFE762237370ECE766237370F2
:10313800E9E76E237370E6E772237370E3E774239D
:103148007370E0E70B490CF007FB701DDBE7631CAD
:103158002222FA54023400233B550120F8BD0020F6
:1031680070470020FAE70020F8E700BFD0A6010862
:1031780037000004D4A6010808B50069FFF758FF16
:1031880008BD00002DE9F0478AB082460C46D0E918
:103198000667002303930493059306930793089304
:1031A800ADF82430FFF730FC00220023CDE90023DE
:1031B800002C76D0054632463B4630463946FDF768
:1031C80053FA88B927F000494FF0FF32374B3046A1
:1031D8004946FDF749FAB8B94FF0FF32334B30464C
:1031E8004946FDF723FA78B9314B93E80300039079
:1031F8008DF810104FF004084646B8F1190F32D96F
:1032080000200AB0BDE8F087DAF814804046FDF7E0
:1032180039F932463B46FDF7F5F930B142462549C2
:1032280003A80CF099FA8046E6E732463B46224965
:1032380003A80CF091FA80466A46204903A80CF0CE
:10324800ADFA012807D132463B46DDE90001FFF718
:10325800DDFB0028D0D132463B46194903A80CF0C3
:103268007BFA8046C8E708F101012046FFF7E2FD36
:103278000146C0B1002302E02E22CA5401339E4207
:1032880008D903F128026A4412F81C2CAA42F3D088
:10329800CA54F3E70022CA54A3681E44A66001205A
:1032A800AFE70020ADE70020ABE700BFFFFFEF7FEF
:1032B800DCA60108E4A60108E8A60108F0A60108B2
:1032C800F4A6010870B500286CD00D460646002902
:1032D8006AD0047B202C16DC002C67D0631E1F2BC1
:1032E80066D8DFE803F0364265286565654F656591
:1032F8006565656565536565656565656565656588
:10330800656565656557402C48D0802C11D10069EA
:10331800002856D00CF098FE441C21462846FFF79A
:1033280089FD00284FD022463169FDF7DDFD0124D3
:103338003FE000243DE005212846FFF77BFD0346DA
:10334800002838D0214A1068186012791A710124AF
:103358002FE006212846FFF76DFD034668B31C4A97
:103368001068186092889A8023E005212846FFF7A4
:1033780061FD034618B3174A1068186012791A716C
:10338800012416E0FFF7FEFE044612E0FFF7F4FE04
:1033980004460EE000F06EF804460AE000F0BEF8BD
:1033A800044606E0002404E0002402E0002400E0D3
:1033B8000024204670BD0024FBE70024F9E7002420
:1033C800F7E70024F5E70024F3E700BFDCA60108CF
:1033D800FCA6010804A7010870B58AB006460D4688
:1033E80014462422002101A80CF0CCFA23684FF4DB
:1033F80080709847034601904FF4807202920695B8
:1034080094E807000AAD05E9070023B101A9304691
:10341800FFF758FF40B9019D1DB1636828469847DA
:10342800002528460AB070BD01A8FFF7A9FCA368CB
:103438004BB1039901310198984705460028EAD015
:1034480000230193EDE72368039801309847054668
:103458000028E0D0039A0132029B9A4228BF1A46FC
:103468000199FDF741FD039B0022EA546368019826
:103478009847D6E770B58568002946D00C460121E3
:103488002046FFF7D7FC002842D05B220270A368D1
:103498000133A360E3680133E36007E0012616E027
:1034A80000221A70A3683344A3602D68FDB1214639
:1034B8002846FFF707FF034640B32046FFF760FCA6
:1034C8002B68002BF1D06369002BE7D00226711C12
:1034D8002046FFF7AFFCE8B103462C2103F8011B97
:1034E80061690029DCD0831C20214170D8E70221C2
:1034F8002046FFF79FFC78B15D22027000224270DF
:10350800E368013BE360012300E00023184670BD37
:103518000023FBE70023F9E70023F7E770B5856888
:10352800002900F0A3800C464B69A3B10226711C48
:103538002046FFF77FFC002800F09B807B23037068
:10354800E3680133E36063690BB10A234370A3683E
:103558003344A36022E00126E9E7E1682046FFF74B
:1035680069FC0346002800F08680002203E0092158
:1035780003F8011B0132E1689142F8D8A3681944A5
:10358800A16010E001261CE0002637E0002339E0A6
:1035980000221A70A3683344A3602D68002D44D01C
:1035A8006369002BD9D12146286AFFF741FD0346FC
:1035B80000285CD02046FFF7E3FB6369002BE1D0CD
:1035C800022631462046FFF735FC002855D03A221E
:1035D800027062690AB109224270A3683344A36089
:1035E80021462846FFF76EFE034600283FD02046B6
:1035F800FFF7C6FB6369002BC6D001262B68002B9A
:10360800C4D001231E44711C2046FFF713FC034657
:10361800A8B32A6812B12C2203F8012B6269002A88
:10362800B6D00A2203F8012BB2E763698BB1E168CF
:1036380001312046FFF7FEFB034610B362699AB9D1
:103648007D221A7000225A70E368013BE36001236F
:103658000DE00221EDE7092203F8012B0131E268B0
:10366800013A8A42F7D8EBE70021F8E70023184629
:1036780070BD0023FBE70023F9E70023F7E70023E9
:10368800F5E70023F3E738B50446C8B10D46C9B1DC
:1036980084680AB90AE024687CB1216A69B12846BD
:1036A800FDF744FB0028F6D107E024682CB1216A15
:1036B8002846FFF779F90028F7D12CB1236A2BB1F6
:1036C800204638BD0C46FBE70024F9E70024F7E75D
:1036D80038B5044616E0E36813F4807F04D1206906
:1036E80010B10F4B5B689847E36813F4007F04D16F
:1036F800206A10B10A4B5B689847094B5B68204603
:1037080098472C4654B12568E36813F4807FE2D1CA
:10371800A0680028DFD0FFF7DBFFDCE738BD00BF7B
:1037280004000020CB68B3F57A7F80F08B802DE908
:10373800F04106460C460133CB60002900F0848036
:103748008B684A68934280F081800A68D25C7B2A41
:1037580002D00020BDE8F08101338B600846FFF7F6
:10376800CFFAA3686268934203D22268D35C7D2BA8
:1037780059D0A3686268934204D2013BA360002534
:103788002F4634E0013BA3600020E3E70746A36827
:103798000133A3602046FFF7B3FA21462846FFF716
:1037A80003FA002839D02046FFF7AAFA2B692B62C2
:1037B80000232B61A368626893422ED22268D25CF0
:1037C8003A2A2AD10133A3602046FFF799FA214605
:1037D800284600F03FF800B32046FFF791FAA368A7
:1037E8006268934211D22268D35C2C2B0DD1A84673
:1037F80004F11000FFF771FB054670B1002FC5D02A
:10380800C8F80000C0F80480C1E7A3686268934262
:1038180003D22268D35C7D2B07D0CFB13846FFF79F
:1038280057FF002096E700252F46E368013BE36039
:1038380007B17D604023F360B760A3680133A360DC
:10384800012087E700207047002083E7002081E7F8
:1038580000207FE700296AD02DE9F84380460D460D
:103868000F68002F65D08C6804F104094E68B145D3
:1038780005D80422314938190CF0D4F850B3631D27
:103888009E4205D305222E4938190CF0CBF848B3CF
:10389800B14505D804222B4938190CF0C3F840B3B8
:1038A800B44202D23B5D222B2DD0B44206D23B5DFE
:1038B8002D2B2DD0303BDBB2092B29D9B44202D2B3
:1038C8003B5D5B2B29D0B44236D23B5D7B2B29D0A4
:1038D80000202FE00423C8F80C30AB680433AB6039
:1038E800012027E00120C8F80C00AA680532AA6068
:1038F80020E00223C8F80C300120C8F81400AA6898
:103908000432AA6016E029464046FFF74DF911E057
:1039180029464046FFF70CFB0CE02946404600F0DC
:1039280013F807E029464046FFF7FCFE02E00020B6
:1039380070470020BDE8F8830020FBE7DCA60108FB
:10394800FCA6010804A70108CB68B3F57A7F6DD2FD
:103958002DE9F04106460C460133CB600A688B68B6
:10396800D25C5B2A02D00020BDE8F08101338B6075
:103978000846FFF7C5F984B1A3686268934203D289
:103988002268D35C5D2B42D0A3686268934204D25C
:10399800013BA36000252F461CE0A368013BA36000
:1039A8000020E1E70746A3680133A3602046FFF73C
:1039B800A7F921462846FFF74DFF10B32046FFF729
:1039C8009FF9ACB1A3686268934211D22268D35CB4
:1039D8002C2B0DD1A84604F11000FFF77EFA0546FE
:1039E80078B1002FDED0C8F80000C0F80480DAE70C
:1039F8003CB1A3686268934203D22268D35C5D2B12
:103A080007D0AFB13846FFF763FE0020ACE70025CA
:103A18002F46E368013BE36007B17D602023F36034
:103A2800B760A3680133A36001209DE700207047B9
:103A3800002099E70000000070B5064614461D46B0
:103A480011A3D3E9002320462946FCF7F9FD38B134
:103A58006FF000437361C6E906452046294670BDEC
:103A680000220B4B20462946FCF7E0FD18B14FF029
:103A780000437361EFE720462946FCF70BFE7061AF
:103A8800E9E700BFAFF300800000C0FFFFFFDF41A0
:103A98000000E0C1F0B58BB015461E460024039423
:103AA800049405940694079408940994294B1C607F
:103AB8005C60044600B1B9B9002C49D001940023D8
:103AC8000293059A049B9A423DD2029215B1029B39
:103AD80023442B601F4B01AA92E8030083E80300EC
:103AE800002738460BB0F0BD039004911A4B93E8B9
:103AF80007000AAF07E907001846FFF7EEF907467F
:103B08000028D9D003A8FFF7F5F9FFF7F9F801461F
:103B18003846FFF79FFE90B136B9002DE1D0039BE0
:103B2800059A13442B60DCE703A8FFF7E9F8059B27
:103B3800049A934203D2039AD35C002BEDD0384603
:103B4800FFF7C6FDB8E7002BC0D0013B0293BDE7E5
:103B58002746C6E70C1000200400002070B5044674
:103B680048B10D4616460CF06FFA33462A46411CFA
:103B78002046FFF78FFF70BD08B500221146FFF7FA
:103B8800EDFF08BD08B5024A0121FFF725FC08BD75
:103B98000400002008B50122FFF775FD08BD0000EC
:103BA80070B504460D461648FFF797F9064670B1FA
:103BB8000823C360C0E906450FA3D3E900232046C4
:103BC8002946FCF73DFD20B16FF000437361304694
:103BD80070BD00220B4B20462946FCF727FD18B183
:103BE8004FF000437361F2E720462946FCF752FD87
:103BF8007061ECE7AFF300800000C0FFFFFFDF411A
:103C0800040000200000E0C170B582B005460E46F1
:103C180010461946FFF7C4FF044600230093074BDC
:103C2800024631462846FFF7CCF810B1204602B0CC
:103C380070BD2046FFF74CFD0024F7E70400002084
:103C480038B504460A48FFF748F9054640B110233D
:103C5800C36007492046FFF7A0F80446286108B169
:103C6800284638BD2846FFF733FD2546F8E700BF4C
:103C78000400002070B582B005460E461046FFF7D6
:103C8800DFFF044600230093074B024631462846CF
:103C9800FFF797F810B1204602B070BD2046FFF735
:103CA80017FD0024F7E700BF0400002008B503480B
:103CB800FFF713F908B14023C36008BD04000020D2
:103CC80028B1007B082814BF00200120704700207D
:103CD800704728B1007B102814BF002001207047CE
:103CE80000207047C8B130B583B014461D46B1B145
:103CF800BAB1C3B1009313460A460F490BF04EFD03
:103D0800032812D12368013B0B2B10D82B68013BE9
:103D18001E2B0ED8002003B030BDFF207047FF20B7
:103D2800F9E7FF20F7E7FF20F5E7FD20F3E7FC20A0
:103D3800F1E7FB20EFE700BF0CA7010800B583B04F
:103D4800009313460A4605490BF028FD032803D0C3
:103D5800002003B05DF804FB0120FAE718A701086A
:103D680010B588B004463D490CF008F810B13C4B3A
:103D780001221A703B4920460CF000F810B1384B6C
:103D880002221A70364B1B78012B09D0344B1B7852
:103D9800022B37D0214634480BF0A4FB08B010BDE5
:103DA80032480BF0FFFB32480BF0FCFB05AB06AAD0
:103DB80007A92046FFF796FF0146F8B9059B069A22
:103DC80007992C480BF08EFB079A2B4981FB02318F
:103DD800D317C3EB6113642101FB13238DF807305C
:103DE8009DF818308DF805309DF814308DF80630A0
:103DF800002201A9214803F02DF9C7E720480BF05C
:103E080071FBC3E71F480BF0CDFB1F480BF0CAFB43
:103E180002AB03AA04A92046FFF790FF0146012838
:103E280003D01A480BF05EFBB4E7029B039A04998F
:103E380017480BF057FB9DF810308DF800309DF8AF
:103E48000C308DF801309DF808308DF802300022D2
:103E580069460A4803F017F89CE700BF24A7010841
:103E6800141000202CA701087CAA010834A7010817
:103E780054A701086CA701081F85EB51E40800202E
:103E88008CA70108A4A70108C8A7010804A801086D
:103E9800DCA7010810B50446012806D0022C14D06E
:103EA800102C22D0082C30D010BD01211C4801F064
:103EB80025FA0128F2D10121194801F01FFA012839
:103EC800F9D0184B01221A70E8E70221144801F0D2
:103ED80015FA0028E4D10221114801F00FFA002850
:103EE800F9D0104B02221A70DAE710210C4801F0C1
:103EF80005FA0028D6D11021094801F0FFF9002859
:103F0800F9D0084B03221A70CCE70821044801F0C5
:103F1800F5F90128C8D1044A138801331380C3E78F
:103F2800000801406008002016100020014B188886
:103F3800704700BF16100020014B1880704700BF63
:103F48001610002070B5A0B04FF6FF70FEF704F908
:103F58002E4B1B78012B1AD04FF4784400944FF65F
:103F6800FF732B4A00210846FEF78AFA00944FF6A1
:103F7800FF73284A00210846FEF782FA142000F051
:103F88002BFD4FF6FF70FEF7E7F820B070BD4FF439
:103F9800FC6400944FF6FF731F4A00210846FEF7A1
:103FA8006FFA00944FF6FF731C4A19210020FEF7A0
:103FB80067FA1B4E706DFCF79BFC0546B06DFCF76D
:103FC80097FC01462846FCF7EBFC4FF06A51FCF7DA
:103FD800E7FC4FF06A51FCF7E3FCFCF765FA024690
:103FE8000B46104902A80BF0B7FB00944FF6FF737D
:103FF80002AA31210020FEF743FA00944FF6FF731E
:10400800094A49210020FEF73BFAB7E7DC080020FF
:1040180064A8010878A801081CA8010830A80108AC
:10402800F808002044A8010854A8010810B58CB06D
:10403800194C00220BA9204602F086FF00220AA98B
:10404800204603F071F89DF82A3000939DF8293036
:104058009DF82B20114902A80BF07EFB1F24009429
:104068004FF6FF7302AA00213C20FEF709FA9DF8DB
:104078002E3000939DF82D309DF82C20084902A879
:104088000BF06AFB00944FF6FF7302AA192148202F
:10409800FEF7F6F90CB010BDE40800208CA8010862
:1040A800A0A8010830B589B0FFF7C0FF002402942A
:1040B8000394049405940694ADF81C4000F034FB76
:1040C800FCF7F2F902460B463C4902A80BF044FB08
:1040D8001F2500954FF6FF7302AA78210A20FEF7E4
:1040E800CFF900F027FBFCF7DFF902460B4634490D
:1040F80002A80BF031FB00954FF6FF7302AA91213D
:104108000A20FEF7BDF900F01BFBFCF7CDF90246CB
:104118000B462C4902A80BF01FFB00954FF6FF73C6
:1041280002AAAA210A20FEF7ABF900F009FB05460E
:1041380000F0FAFA01462846FCF732FCFCF7B4F91D
:1041480002460B46204902A80BF006FB00944FF6E6
:10415800FF7302AADC212046FEF792F91B4B1B785D
:10416800032B09D01A4B1B78012B0CD0184B1B784A
:10417800032B17D009B030BD154A137801331370DB
:10418800124B1C70EEE7134803F00AFE002000F003
:10419800DDFA00220421104801F0B7F80C4B022286
:1041A8001A70E3E70B4803F037FE012204210A489E
:1041B80001F0ABF8064B00221A70DBE7B0A8010843
:1041C800C4A80108D8A80108ECA8010860080020C4
:1041D8001D100020D8090020000C0140014B187860
:1041E800704700BF1C10002010B588B01F23009333
:1041F8004FF6FF73724A00210A20FEF741F900F0DA
:1042080093FA704B1968FCF7C1FAFCF74DF90246AE
:104218000B466D4903A80BF09FFA6C4B1B7893B1C2
:104228006B4B1B78032B18D0684B1B78012B1CD0C9
:10423800664B1B78022B53D0644B1B78032B00F082
:104248008C8008B010BD1F2300934FF6FF7303AA9C
:1042580032210A20FEF714F9E2E75C4A13780133A9
:1042680013705B4B00221A70DEE74FF6FF74009460
:104278001F2303AA32210A20FEF702F90023009324
:104288002346544A4B210A20FEF7FAF8504B1B7874
:10429800012B16D04E4B1B78022BC9D1494C4E49E5
:1042A8002068FCF775FA206020F0004400F03CFA22
:1042B80001462046FCF726FD68B9454B00221A70D6
:1042C800B6E7404C44492068FCF760FA2060404B50
:1042D80000221A70DEE700F027FA3A4B1860ECE784
:1042E8004FF6FF7400941F2303AA32210A20FEF719
:1042F800C7F8002300932346384A4B210A20FEF7CB
:10430800BFF8334B1B78012B17D0314B1B78022B8E
:1043180092D12C4C4FF07E512068FCF739FA20607E
:1043280020F0004400F000FA01462046FCF7EAFCC1
:1043380070B9274B00221A707EE7224C4FF07E514D
:104348002068FCF723FA2060214B00221A70DCE772
:1043580000F0EAF91B4B1860EBE74FF6FF73009388
:104368001F2303AA32210A20FEF78AF800F0DCF99D
:10437800144B1968FCF70AFA00F0EEF901280FD07F
:104388001F2300934FF6FF73154A64210A20FEF796
:1043980077F80E4B00221A700A4B00221A6050E779
:1043A8001F2300934FF6FF730E4A64210A20FEF77D
:1043B80067F8064B00221A70024B00221A6040E789
:1043C80004A901081810002014A901081C100020D5
:1043D8006008002028A90108CDCCCC3D30A90108EF
:1043E80048A9010838A9010830B585B0002203A9F9
:1043F800324802F099FE102009F028FB05469DF886
:104408000E3000939DF80D309DF80F202C490BF0CD
:10441800A3F9FFF74BFC04462A462A49FFF72AFC72
:10442800294B1868FCF740F802460B4627492046F6
:10443800FFF7EAFB264B1868FCF736F802460B46EE
:1044480024492046FFF7E0FB234A24492046FFF78A
:1044580011FC234A23492046FFF70CFC2046FFF7AE
:1044680091FB044607222049204808F07BFBF8B955
:104478001F480BF097F820460BF0E6FD024602AB0A
:1044880021461A4808F055FD50B1184808F0CDFEED
:10449800284609F0E3FA204609F0E0FA05B030BDF5
:1044A80014480BF07FF8214613480BF01BF8ECE793
:1044B800014612480BF016F8EAE700BFE4080020AE
:1044C8008CA801085CA901081400002064A901084F
:1044D800100000206CA901087CA9010884A9010822
:1044E80090A901089CA90108A0A90108381000207A
:1044F800B4A90108CCA90108E4A90108ECA901089C
:1045080010B501220A490B4808F02CFB044638B1C3
:10451800042809D0074808F088FE0124204610BD69
:10452800044808F082FEF9E7FFF75EFFF2E700BFF4
:10453800A0A901083810002070B582B0FFF7E0FF8D
:1045480000285DD001225D495D4808F00BFB00287A
:104558005AD15B4BD3F80C4221465A480AF0C2FFA5
:10456800574D2146284608F074FED5F80862002108
:10457800284608F06EFE701C09F068FA044601AB84
:1045880032460146284608F0DEFB002846D04C4853
:1045980008F04BFE2046FFF7EFFA0546002845D005
:1045A80049492846FFF7F6FA064618B1FFF791FB86
:1045B800002842D145480AF0F5FF45492846FFF74B
:1045C800E9FA064600283FD0FFF77AFB00283BD0DF
:1045D80073693BB100220023D6E90601FCF712F803
:1045E800002831D1D6E90601FCF77CF8394B186070
:1045F800FBF75AFF02460B4637480AF073FF29E0DB
:1046080036480AF0CFFF9DE735480AF0CBFF2C4B20
:10461800D3F80C4233480AF0C5FF9DE7019B0022FE
:10462800E254214630480AF05DFFB0E72F480AF00F
:10463800B9FF204609F012FAB2E731692C4B19602C
:104648002C480AF04FFFB8E72B480AF0ABFF214B84
:104658002A4A1A602A492846FFF79CFA064610B1EA
:10466800FFF737FBE0B927480AF09CFF264B274A9B
:104678001A6027492846FFF78DFA064610B1FFF75A
:1046880028FBA0B923480AF08DFF234B234A1A6060
:104698002846FFF71DF8204609F0E0F902B070BD82
:1046A8003169194B19601E480AF01CFFE1E73169AE
:1046B800194B19601B480AF015FFE9E7A0A9010882
:1046C8003810002054AA01085CA90108A0AA010812
:1046D80064A9010814000020B0AA010808AA01086A
:1046E8001CAA01083CAA010870AA010880AA0108AE
:1046F8003010002094AA0108C0AA01080000404018
:1047080084A90108E0AA01082C1000207CA901084E
:104718009CA9010800AB01082810002090A90108F5
:10472800D0AA0108F4AA0108014B1868704700BF15
:1047380014000020014B1868704700BF20100020AB
:10474800014B1868704700BF24100020014B186007
:10475800704700BF241000202DE9F04383B0804645
:1047680001224A494A4808F0FDF9002857D106466F
:10477800474DD5F80C12284608F06BFDD5F808729D
:104788000021284608F065FD781C09F05FF9044609
:1047980001AB3A460146284608F0D5FA10B9019B04
:1047A8000022E2543A4808F040FD2046FFF7E4F9B9
:1047B800074600283BD03749FFF7ECF9054618B102
:1047C800FFF77EFA002839D13846FFF7DBF90546AE
:1047D80002222E492E4808F0C5F98146002836D114
:1047E80028460BF031FC02466B462946284808F05B
:1047F800A0FB002838D128480AF0D4FE274BC3F87C
:104808000080234808F011FD3846FEF761FF204676
:1048180009F024F9284609F021F9012603E0204887
:104828000AF0C0FE0026304603B0BDE8F0831D48FC
:104838000AF0B8FE204609F011F9F4E74046FBF704
:1048480033FE02460B462846FFF7F6F8BCE7164843
:104858000AF0A8FE3846FEF73BFF204609F0FEF8AE
:10486800284609F0FBF8DEE710480AF09BFE0848E6
:1048780008F0DBFC3846FEF72BFF204609F0EEF87F
:10488800284609F0EBF84E46CDE700BFA0A901087D
:104898003810002064A901085CAB0108140000204E
:1048A80010AB01082CAB010844AB010878AB010838
:1048B80038B502681A4B9A4200D038BD194A138895
:1048C80001339BB21380B3F57A7FF6D1FFF72EFB45
:1048D800FCF70EF81449FCF717F9144C2168FCF79B
:1048E8005FF81349FCF75CF8124D286000200D4B67
:1048F8001880FFF721FB28680146FBF749FF0E499E
:10490800FCF74EF82168FCF74BF80C49FCF748F81F
:1049180001460B4C2068FBF73BFF2060CDE700BF4A
:10492800000800401E1000200000A04110000020D8
:104938006666664020100020C3F54840B4A291394D
:104948002410002010B504460E4B1A784FF47A73E1
:10495800B3FBF2F30C4A1068B0FBF3F000F0B4F8C4
:1049680068B90F2C01D901200AE0002221464FF036
:10497800FF3000F08BF8054B1C60002000E00120A0
:1049880010BD00BF18000020000000201C000020FF
:1049980008B5074A136843F010031360032000F0BA
:1049A80063F80020FFF7CEFFFDF794F9002008BD5B
:1049B80000200240034A1168034B1B780B44136024
:1049C800704700BF3410002018000020014B186801
:1049D800704700BF3410002038B50446FFF7F6FFD3
:1049E8000546B4F1FF3F02D0044B1B781C44FFF787
:1049F800EDFF401BA042FAD338BD00BF18000020CD
:104A0800002808DB0901C9B200F1604000F56140E7
:104A180080F80013704700F00F000901C9B2014B7C
:104A28001954704714ED00E000B500F00700C0F11C
:104A3800070CBCF1040F28BF4FF0040C031D062B14
:104A48000FD9C31E4FF0FF3E0EFA0CF021EA000109
:104A580099400EFA03FE22EA0E0241EA02005DF8CE
:104A680004FB0023EEE70000074AD36823F4E06361
:104A78001B041B0C000200F4E060034343F0BF6317
:104A880043F40033D360704700ED00E010B50446EE
:104A9800054BD868C0F30220FFF7C6FF0146204641
:104AA800FFF7AEFF10BD00BF00ED00E0002807DBF8
:104AB80000F01F02400901239340024A42F82030C7
:104AC800704700BF00E100E00138B0F1807F0BD2F1
:104AD8004FF0E0235861054AF02182F823100020A6
:104AE800986107221A6170470120704700ED00E0C5
:104AF80030B40124056CAC40C56B6C60046863601D
:104B08004368102B05D0036899600368DA6030BCED
:104B1800704703689A600368D960F8E7002838D0BE
:104B280010B4024601681C4B994227D81B4B0B4412
:104B38001B48A0FB03031B099B001364194BD36399
:104B4800022382F8213008686FF30D1053689468C7
:104B58002343D46823431469234354692343946942
:104B68002343D469234303430B600020906301234C
:104B780082F8213082F8200010BC70470A4B0B44A1
:104B88000748A0FB03031B099B001364074BD3636F
:104B9800D6E70120704700BF07040240F8FFFDBFB9
:104BA800CDCCCCCC00000240F8FBFDBF0004024095
:104BB80038B5044690F82000012832D0012084F846
:104BC800200094F82100C0B2012804D0002384F802
:104BD8002030022038BD022084F821000020A06384
:104BE8002568286820F0010028602046FFF780FF2C
:104BF800E36A5BB12268136843F00E03136022680E
:104C0800136843F0010313600020E3E72268136888
:104C180023F0040313602268136843F00A03136047
:104C2800EDE70220D6E7034690F82120D2B2022A07
:104C380006D004228263002280F8202001207047D9
:104C480001680A6822F00E020A6001680A6822F008
:104C580001020A60026CC06B012101FA02F2426093
:104C680083F82110002083F82000704708B590F8D9
:104C78002130DBB2022B03D004238363012008BD5B
:104C88000268136823F00E0313600268136823F0A8
:104C98000103136003684C4A93424ED9783A934211
:104CA80024D01432934230D0143293422FD014328D
:104CB80093422FD0143293422FD0143293422FD0E4
:104CC800143293422FD002F5627293422ED01432DE
:104CD80093422DD0143293422CD01432934202D0F6
:104CE8004FF4803203E04FF4805200E00122374B4A
:104CF8005A60012380F82130002380F82030436B6C
:104D0800002B5ED098470020B9E71022EFE74FF458
:104D18008072ECE74FF48052E9E74FF48032E6E71F
:104D28004FF48012E3E74FF08072E0E70122DEE7FC
:104D38001022DCE74FF48072D9E7254A934224D049
:104D48001432934225D01432934224D01432934221
:104D580024D01432934224D01432934224D01432F3
:104D6800934224D002F56272934223D014329342C4
:104D780022D01432934221D01432934202D04FF4FD
:104D8800803203E04FF4805200E00122114B5A6058
:104D9800AFE71022FAE74FF48072F7E74FF480523A
:104DA800F4E74FF48032F1E74FF48012EEE74FF06A
:104DB8008072EBE70122E9E71022E7E74FF48072FF
:104DC800E4E700205BE700BF8000024000040240E7
:104DD800080002400000024038B5C36B1A68046836
:104DE8002568016C04238B40134200F09B8015F06A
:104DF800040F00F09780236813F0200F03D1236875
:104E080023F00403236003689A4A934246D9783A08
:104E1800934224D01432934228D01432934227D09C
:104E28001432934227D01432934227D0143293423B
:104E380027D01432934227D002F56272934226D0CB
:104E48001432934225D01432934224D01432934220
:104E580002D04FF4802203E04FF4804200E00422A5
:104E6800854B5A60C36A03B1984738BD4022F7E7BB
:104E78004FF48062F4E74FF48042F1E74FF4802268
:104E8800EEE74FF48002EBE74FF08062E8E7042298
:104E9800E6E74022E4E74FF48062E1E7774A93428D
:104EA80024D01432934225D01432934224D01432A1
:104EB800934224D01432934224D01432934224D003
:104EC8001432934224D002F56272934223D01432F2
:104ED800934222D01432934221D01432934202D00A
:104EE8004FF4802203E04FF4804200E00422644B38
:104EF8005A60B7E74022FAE74FF48062F7E74FF4C9
:104F08008042F4E74FF48022F1E74FF48002EEE7A5
:104F18004FF08062EBE70422E9E74022E7E74FF42D
:104F28008062E4E702238B40134200F0AB8015F067
:104F3800020F00F0A780236813F0200F06D1236822
:104F480023F00A032360012380F821300368494ACB
:104F580093424BD9783A934224D0143293422DD0BD
:104F6800143293422CD0143293422CD014329342F0
:104F78002CD0143293422CD0143293422CD002F508
:104F8800627293422BD0143293422AD01432934245
:104F980029D01432934202D04FF4003203E04FF488
:104FA800005200E00222344B5A60002380F820307F
:104FB800836A002B3FF459AF984756E72022F2E75F
:104FC8004FF40072EFE74FF40052ECE74FF4003271
:104FD800E9E74FF40012E6E74FF00072E3E7022238
:104FE800E1E72022DFE74FF40072DCE7234A93422F
:104FF80024D01432934225D01432934224D0143250
:10500800934224D01432934224D01432934224D0B1
:105018001432934224D002F56272934223D01432A0
:10502800934222D01432934221D01432934202D0B8
:105038004FF4003203E04FF4005200E00222104B1C
:105048005A60B2E72022FAE74FF40072F7E74FF40C
:105058000052F4E74FF40032F1E74FF40012EEE7A4
:105068004FF00072EBE70222E9E72022E7E74FF46E
:105078000072E4E780000240000402400800024099
:105088000000024008238B4013423FF4EEAE15F0B7
:10509800080F3FF4EAAE236823F00E032360026C86
:1050A800C16B012303FA02F24A60836380F821305E
:1050B800002380F82030036B002B3FF4D6AE9847CE
:1050C800D3E600BF70B582B00024A446ABE0854D9E
:1050D800AB4214D00CD8A5F58015AB420FD005F51E
:1050E8007025AB420BD0A5F58015AB4210D106E078
:1050F8007D4DAB4203D005F58035AB4208D18B68B6
:10510800002B5AD0012B53D04261082400E0CC6810
:10511800BEF1FF0F53D806464FEA8C0233680F25BD
:10512800954023EA050304FA02F2134333604B68FF
:1051380013F0805F75D06D4B9A6942F001029A6155
:105148009B6903F001030193019B4FEA9C02951CA4
:10515800674B53F825600CF00305AD000F23AB40F7
:1051680026EA0306634B984230D003F580639842E1
:1051780000F0968003F58063984200F0938003F571
:105188008063984200F0908003F58063984200F0B5
:105198008D8003F58063984216D0062317E0CC680B
:1051A8000434B5E7CC680834B2E7CC680C34AFE710
:1051B80002610824ACE70024AAE70424A8E7061D36
:1051C800ACF108029200A9E7052300E00023AB40F8
:1051D80033430232464D45F822304B6813F4801FA2
:1051E80066D0454A936843EA0E0393604B6813F40C
:1051F800001F63D0404AD36843EA0E03D3604B686C
:1052080013F4003F60D03C4A536843EA0E035360EE
:105218004B6813F4803F5DD0374A136843EA0E03A6
:1052280013600CF1010C0B6833FA0CF258D0012210
:1052380002FA0CF203EA020E32EA0303F1D14B68D8
:10524800122B3FF644AF122B3FF662AF01A555F87B
:1052580023F000BF0751000817510008AD5100089E
:10526800BF510008195100081951000819510008C8
:10527800195100081951000819510008195100085E
:10528800195100081951000819510008195100084E
:105298001951000819510008A7510008B351000816
:1052A800012394E7022392E7032390E704238EE780
:1052B800114A936823EA0E03936097E70E4AD3686E
:1052C80023EA0E03D3609AE70B4A536823EA0E03D6
:1052D80053609DE7084A136823EA0E031360A0E7AA
:1052E80002B070BD00002210000031100010024012
:1052F8000000014000080140000401408368194291
:1053080001D001207047002070470AB10161704741
:10531800090401617047000008B5054B5B69034249
:1053280000D108BD024B5861FEF7B4FDF9E700BF94
:105338000004014038B512F4804F44D00468B4F832
:1053480050309BB291F800C003EBCC03023304EB5E
:105358004304B4F80044C4F309048B69A34228D376
:105368001B1B8B618B697BB9056835F82C309BB2A8
:1053780023F4804323F0700383F4005343F4004381
:1053880043F0800325F82C3012F0400F0ED002684D
:105398000D7832F825309BB223F4E04323F07003F4
:1053A80043F4004343F0C00322F8253024B92046D3
:1053B80038BD00238B61D5E723460A89496900680F
:1053C80004F05EFFF3E70468B4F850309BB291F83C
:1053D80000C003EBCC03063304EB4304B4F80044E9
:1053E800C4F309048B69A3422FD31B1B8B618B6900
:1053F8007BB9056835F82C309BB223F4804323F041
:10540800700383F4005343F4004343F0800325F80A
:105418002C3012F0400F0FD1026891F800C032F81A
:105428002C309BB223F4E04323F0700343F4004391
:1054380043F0C00322F82C30002CB8D023464A8908
:105448004969006804F01CFFB1E700238B61CEE7CF
:1054580070B586B0002800F08180044690F8A93223
:10546800EBB1032384F8A932206803F098FF25469E
:1054780055F8106BEC460FCDACE80F002B68CCF854
:105488000030231D0ECB304603F079FF054658B196
:10549800022384F8A9320125284606B070BD80F899
:1054A800A83208F0BDF9DCE70021206803F081FF8D
:1054B8002B4616E05A1C02EB820104EBC1010120C5
:1054C800487002EB820104F8313004EBC10000217E
:1054D800C17003EB830004EBC0008163C163016406
:1054E800D3B261688B42E5D316E005EB850304EB84
:1054F800C303002283F8692183F8685183F86B217C
:10550800C3F87821C3F87C2105EB850304EBC303BA
:10551800C3F880210135EDB2A942E6D8254655F8F1
:10552800106BEC460FCDACE80F002B68CCF80030C0
:10553800231D0ECB304603F03EFF054620B1022363
:1055480084F8A9320125A7E7002384F82430012331
:1055580084F8A932206804F091FA9DE701259BE7B9
:1055680038B590F8A832012B11D00446012580F8EF
:10557800A852006803F00AFF2946204608F065FA99
:10558800206804F079FA002084F8A80238BD0220C7
:10559800FCE770B505460C46164612F0400F00F0C1
:1055A8000E810268B2F850309BB2097803EBC10350
:1055B800023302EB4302B2F80024C2F30902A369E2
:1055C80093424ED99B1AA361A369002B66D16378D5
:1055D800002B49D12B68B3F8502092B2134403EB47
:1055E8000113B3F80424C2F30902A3F80424B3F89E
:1055F80004246FEA42426FEA524292B2A3F80424AA
:105608002B686278002A3CD1B3F8502092B2134438
:10561800227803EB0213B3F80C24C2F30902A3F8AF
:105628000C24B3F80C246FEA42426FEA524292B259
:10563800A3F80C242178284608F026F916F4804FA0
:1056480041D02A68217832F821309BB223F4E04314
:1056580023F0700343F4404343F0800322F82130E1
:1056680031E00023A361AFE7012BC9D12B68B3F860
:10567800502092B2134403EB01130022A3F8042430
:10568800BEE7012AD6D1B3F8502092B2134422784B
:1056980003EB02130022A3F80C24CBE716F4804F87
:1056A8000DD0286830F821309BB223F4E04323F072
:1056B800700343F4404343F0800320F8213094F80A
:1056C8002430012B12D02A68217832F821309BB27D
:1056D80023F4E04323F0400383F0300343F4004312
:1056E80043F0800322F82130002070BD6369134421
:1056F8006361E3691344E361216A2369994224D30E
:10570800C91A21626278002A44D12A68B2F8501076
:1057180089B20A44217802EB0112B2F80414C1F3E9
:105728000901A2F804143E2B1BD9580913F01F0FC6
:1057380000D10138B2F8041489B2800280B2014362
:1057480041F40041A2F8041426E021B9002384F8AA
:1057580024301346D6E7002384F8243023620B460E
:10576800D0E74BB9B2F804146FEA41416FEA5141EE
:1057780089B2A2F804140FE0590813F0010F00D001
:105788000131B2F8040480B2890289B20143A2F857
:10579800041401E0012A06D09BB2228961692868B5
:1057A80004F074F98FE72A68B2F8501089B20A44F5
:1057B800217802EB011299B2A2F80414ECE702680E
:1057C800B2F850309BB2097803EBC103063302EB01
:1057D8004302B2F80024C2F30902A36993424FD3EB
:1057E8009B1AA361A369002B67D16378002B4AD168
:1057F8002B68B3F8502092B2134403EB0113B3F8AB
:105808000424C2F30902A3F80424B3F804246FEAB9
:1058180042426FEA524292B2A3F804242B6862789B
:10582800002A3DD1B3F8502092B21344227803EBFA
:105838000213B3F80C24C2F30902A3F80C24B3F83A
:105848000C246FEA42426FEA524292B2A3F80C2447
:105858002178284608F018F816F4804F7FF433AF03
:105868002A68217832F821309BB223F4E04323F0F0
:10587800700343F4404343F0800322F8213022E7C9
:105888000023A361AEE7012BC8D12B68B3F85020E1
:1058980092B2134403EB01130022A3F80424BDE7DA
:1058A800012AD5D1B3F8502092B21344227803EBE1
:1058B80002130022A3F80C24CAE716F4804F0DD176
:1058C800286830F821309BB223F4E04323F07003BA
:1058D80043F4404343F0800320F8213094F8243007
:1058E800012B7FF4F0AE636913446361E3691344E9
:1058F800E361216A2369994224D3C91A21622A687B
:105908006178002943D1B2F8501089B20A4421784D
:1059180002EB0112B2F80C14C1F30901A2F80C143D
:105928003E2B1BD9580913F01F0F00D10138B2F8CC
:105938000C1489B2800280B2014341F40041A2F8FC
:105948000C1426E021B9002384F824301346D6E746
:105958000023236284F824300B46D0E74BB9B2F811
:105968000C146FEA41416FEA514189B2A2F80C1454
:105978000FE0590813F0010F00D00131B2F80C0400
:1059880080B2890289B20143A2F80C1401E001290E
:1059980006D09BB262896169286804F077F892E6BC
:1059A800B2F8501089B20A44217802EB011299B278
:1059B800A2F80C14EDE72DE9F04105462868B0F887
:1059C800443013F4004F00F09282B0F84440A3B280
:1059D80014F00F0440F0E28013F0100F6BD003882E
:1059E8009AB213F4006F40F09D8012F4004FE5D096
:1059F800038823F070031B051B0D43F0800303800D
:105A08002868B0F850309BB295F8682103EBC203C0
:105A1800063300EB4303B3F80034C3F30903C5F8B6
:105A280084318BB1D5F87C1171B1B5F86E2104F0D1
:105A380027FCD5F87C31D5F884211344C5F87C318E
:105A48000021284607F014FF2A68138899B213F436
:105A5800006FB3D101F44051B1F5405FAED0B2F858
:105A680050309BB21A44B2F80C34C3F30903A2F8BD
:105A78000C34D5F878313E2B77D9590913F01F0F1C
:105A880000D10139B2F80C349BB2890289B20B43B8
:105A980043F40043A2F80C342A6813889BB223F419
:105AA800804323F0700383F4405343F4004343F0EE
:105AB8008003138082E703889BB223F4E14323F039
:105AC80070036FEA43436FEA53439BB203802A682B
:105AD800B2F850309BB295F8281003EBC10302339B
:105AE80002EB4302B2F80034C3F309036B64EA6BB8
:105AF8001A44EA630021284607F0C6FE95F82430C8
:105B0800002B3FF45BAF2B6C002B7FF457AF95F85D
:105B180024302A6843F08003A2F84C30002385F82B
:105B280024304BE7B0F850309BB295F8682103EB6E
:105B3800C203063300EB4303B3F80034C3F309038D
:105B4800C5F88431B5F86E2105F52C7104F098FB81
:105B58002A68138823F070031B051B0D43F080038C
:105B68001380284607F07CFE28E74BB9B2F80C34BE
:105B78006FEA43436FEA53439BB2A2F80C348BE7B6
:105B8800590813F0010F00D00131B2F80C3498B263
:105B98008B029BB20343A2F80C347DE730F8243023
:105BA8009EB213F4004F4CD116F0800F3FF406AFAD
:105BB800621C02EB820105EBC101286830F8243031
:105BC8009BB223F4E14323F070036FEA43436FEA87
:105BD80053439BB220F82430CB78012B00F0F2809D
:105BE80016F4807F40F07E812868B0F850309BB270
:105BF800621C02EB820215F8326003EBC603023323
:105C080000EB4303B3F80034C3F3090304EB840245
:105C180005EBC202126C9A4240F24C8104EB8407F5
:105C280005EBC707D21A3A6404EB840205EBC202FB
:105C3800126C002A40F045813146284607F024FEC0
:105C4800BCE630F8243023F070031B051B0D43F02D
:105C5800800320F8243004EB8401C90001F5B471F5
:105C680005EB010804EB840305EBC30393F87431D7
:105C7800002B42D12868B0F850309BB204EB840264
:105C880005EBC20292F8682103EBC203063300EB6E
:105C98004303B3F80074C7F3090717BB04EB840385
:105CA80005EBC303D3F884213A44C3F88421D3F81D
:105CB8007C213A44C3F87C21D3F880313BB104EB12
:105CC800840305EBC303D3F878319F4275D204EB04
:105CD800840305EBC30393F86811284607F0C8FD51
:105CE80062E704EB840105EBC1013B46B1F86E2184
:105CF800D1F87C1104F0C4FAD0E704EB840305EB77
:105D0800C30393F86B31022B35D0296804EB840266
:105D180005EBC20292F8680131F820309BB223F4F7
:105D2800E04323F0700343F4004343F0C00321F839
:105D38002030286892F8682130F8223013F4804F18
:105D480020D0B0F850309BB203EBC203023300EB13
:105D58004303B3F80074C7F30907002F9ED004EB80
:105D6800840105EBC1013B46B1F87021D1F87C11E3
:105D780004F086FA92E7324641462846FFF7DAFAF7
:105D880007468BE7B0F850309BB203EBC2030633EB
:105D980000EB4303B3F80074C7F30907002F3FF47F
:105DA8007DAF04EB840105EBC1013B46B1F87221DC
:105DB800D1F87C1104F064FA70E74146286803F0D2
:105DC80078FEF1E604EB840305EBC30300221A64B2
:105DD80093F83430FBB116F0400F37D04B781BBB2B
:105DE8002B68B3F8502092B21344621C02EB820273
:105DF80015F8322003EB0213B3F80424C2F30902A6
:105E0800A3F80424B3F804246FEA42426FEA52422A
:105E180092B2A3F80424013404EB840415F8341076
:105E2800284607F031FDC9E5012BF4D12B68B3F8FA
:105E3800502092B21344621C02EB820215F8322001
:105E480003EB02130022A3F80424E4E72A68631C86
:105E580003EB830305EBC3035B78D3B9B2F8503087
:105E68009BB21344621C02EB820215F8322003EB4A
:105E78000213B3F80C24C2F30902A3F80C24B3F8F4
:105E88000C246FEA42426FEA524292B2A3F80C2401
:105E9800C1E7012BBFD1B2F850309BB21344621C4A
:105EA80002EB820215F8322003EB02130022A3F85A
:105EB8000C24B0E704EB840205EBC2020027176448
:105EC800B2E604EB840205EBC202D66B1E44D6632D
:105ED800526C04EB840405EBC4041344636403F0BC
:105EE800E8FD6BE532462846FFF753FB66E50020E0
:105EF800BDE8F08190F8A832012B0DD010B504460A
:105F0800012380F8A83280F82410006803F0AEFD61
:105F1800002084F8A80210BD0220704710B584B094
:105F28000446006803F0ACFD10F4004F20D110F4D3
:105F3800806F21D110F4804F2FD110F4005F37D13A
:105F480010F4805F3ED110F4006F40F0878010F4A9
:105F5800007F40F0AE8010F4807F27D02268B2F82E
:105F680044309BB223F480739BB2A2F844301DE006
:105F78002046FFF720FD19E02268B2F844309BB2B2
:105F880023F480639BB2A2F84430204607F08DFCCE
:105F980000212046FFF7AEFF08E02268B2F844303F
:105FA8009BB223F480439BB2A2F8443004B010BDE6
:105FB8002268B2F844309BB223F400539BB2A2F893
:105FC8004430F3E72268B2F840309BB223F0040370
:105FD8009BB2A2F840302268B2F840309BB223F05E
:105FE80008039BB2A2F84030204607F081FC2268E3
:105FF800B2F844309BB223F480539BB2A2F84430E9
:10600800D4E7226832F8231004AA02EB430222F8EC
:10601800101C0133DBB2072BF3D92268B2F84030E9
:106028009BB243F00103A2F840302268B2F8403036
:106038009BB223F001039BB2A2F840302368B3F867
:10604800442012F4806FF9D0B3F8442092B222F4BD
:10605800806292B2A3F8442000230BE00023DAE721
:10606800226804A901EB430131F8101C22F823101F
:106078000133DBB2072BF3D92268B2F840309BB268
:1060880043F00803A2F840302268B2F844309BB2CB
:1060980023F400639BB2A2F844302268B2F840307F
:1060A8009BB243F00403A2F84030204607F010FCEE
:1060B8007CE72268B2F844309BB223F400739BB2A9
:1060C800A2F84430204607F0EAFB6FE710B5044613
:1060D800084611F0800F25D101F0070C0CEB8C015C
:1060E800C90001F5B47E04EB0E010CEB8C0C04EB3B
:1060F800CC0C4FF0000E8CF869E100F00700087036
:106108000A61CB70022B1AD094F8A832012B19D04F
:10611800012384F8A832206803F062F9002084F88B
:10612800A80210BD01F0070C0CF1010C0CEB8C015E
:1061380004EBC1014FF0010E81F801E0DDE7002317
:106148000B71E1E70220ECE710B504460B4611F0AD
:10615800800F1FD101F0070202EB8201C90001F58F
:10616800B471014402EB820200EBC202002082F803
:10617800690103F007030B7094F8A832012B13D0C0
:10618800012384F8A832206803F00FFB002084F86C
:10619800A80210BD01F00702013202EB820100EBF8
:1061A800C10101204870E4E70220F2E710B501F0D0
:1061B800070C0CEB8C01C90001F5B4710CEB8C0ECB
:1061C80000EBCE0ECEF87C21CEF880310024CEF83C
:1061D80084418EF869418EF868C10144006803F073
:1061E80068FC204610BD01F0070101EB810100EBBE
:1061F800C100D0F88401704738B501F0070404F1F4
:10620800010C0CEB8C0104EB840E00EBCE0ECEF8E7
:106218003C20CEF8403001228EF84C20CEF8483091
:106228000025CEF8445000EBC1035A7000F8314005
:106238001946006803F03DFC284638BD38B501F022
:1062480007054268954231D804460B4611F0800F85
:106258001ED101EB8101C90001F5B471014403EBC2
:10626800830300EBC303002283F8692101238B70A9
:106278000D7094F8A832012B1AD0012384F8A832A3
:10628800206803F07DFB5DB1002084F8A80238BDCA
:106298006B1C03EB830100EBC10101224A70E5E7A7
:1062A80004F52C71206803F0EFFBEDE70120EEE721
:1062B8000220ECE70B4601F00F014268914230D80A
:1062C80010B5044613F0800F21D103F0070202EB4A
:1062D8008201C90001F5B471014402EB820200EBAE
:1062E800C202002082F8690100228A7003F00703C5
:1062F8000B7094F8A832012B15D0012384F8A8322A
:10630800206803F062FB002084F8A80210BD03F0A7
:106318000702013202EB820100EBC1010120487043
:10632800E2E7012070470220F0E790F8A832012B3D
:1063380014D010B50446012380F8A83211F0800F5C
:1063480006D1006803F04AF8002084F8A80210BDBE
:1063580001F00701006803F03FF8F5E702207047F5
:1063680011F0800F0BD001F00701013101EB810121
:1063780000EBC10052B90273C3800020704701EBE3
:106388008101C90001F5B4710844F3E701220273E1
:1063980003811B0C4381F0E7014B01221A6270470D
:1063A80000000E4282B0084B1B68084AA2FB032378
:1063B8005B0A00FB03F3019300BF019B5A1E019285
:1063C800002BF9D102B0704700000020D34D6210B5
:1063D800002800F0F18170B582B00446036813F01C
:1063E800010F2CD0994B5B6803F00C03042B1DD0D4
:1063F800964B5B6803F00C03082B12D06368B3F567
:10640800803F41D0002B55D103F1804303F504337D
:106418001A6822F480321A601A6822F480221A60FC
:1064280037E08A4B5B6813F4803FE7D0874B1B68E3
:1064380013F4003F03D06368002B00F0BF8123688A
:1064480013F0020F75D0814B5B6813F00C0F5FD00F
:106458007E4B5B6803F00C03082B54D02369002B98
:1064680000F08A807A4B01221A60FEF7AFFA0546DF
:10647800764B1B6813F0020F75D1FEF7A7FA401B85
:106488000228F5D903209EE1704A136843F480334B
:106498001360636843B3FEF799FA05466B4B1B68B4
:1064A80013F4003FCBD1FEF791FA401B6428F5D9CD
:1064B800032088E1B3F5A02F09D0644B1A6822F4B1
:1064C80080321A601A6822F480221A60E1E703F128
:1064D8008043A3F53C331A6842F480221A601A6894
:1064E80042F480321A60D4E7FEF770FA0546574B3B
:1064F8001B6813F4003FA2D0FEF768FA401B64281B
:10650800F5D903205FE1514B5B6813F4803FA5D1B7
:106518004E4B1B6813F0020F03D02369012B40F088
:106528004F814A4A136823F0F803616943EAC103BB
:106538001360236813F0080F33D0A369002B5CD0D5
:10654800434B0122C3F88024FEF740FA05463F4B2F
:106558005B6A13F0020F21D1FEF738FA401B0228BC
:10656800F5D903202FE1394A136823F0F80361694C
:1065780043EAC1031360DCE7354B00221A60FEF7DB
:1065880025FA0546314B1B6813F0020FD1D0FEF7F0
:106598001DFA401B0228F5D9032014E10120FFF75A
:1065A80001FF236813F0040F00F09680274BDB6986
:1065B80013F0805F34D1254BDA6942F08052DA61FA
:1065C800DB6903F080530193019B0125214B1B6874
:1065D80013F4807F26D0E368012B3DD0002B53D1E4
:1065E80003F1804303F504331A6A22F001021A62A8
:1065F8001A6A22F004021A6233E0154B0022C3F82B
:106608008024FEF7E3F90546104B5B6A13F0020F8E
:10661800C7D0FEF7DBF9401B0228F5D90320D2E0EA
:106628000025D3E70B4A136843F480731360FEF721
:10663800CDF90646074B1B6813F4807FCBD1FEF7D4
:10664800C5F9801B6428F5D90320BCE0001002407E
:1066580000004242007000405F4A136A43F00103A1
:106668001362E36833B3FEF7B1F906465A4B1B6A67
:1066780013F0020F2FD1FEF7A9F9801B41F28833DE
:106688009842F3D903209EE0052B09D0524B1A6A91
:1066980022F001021A621A6A22F004021A62E0E782
:1066A8004D4B1A6A42F004021A621A6A42F0010259
:1066B8001A62D6E7FEF78AF90646474B1B6A13F0BB
:1066C800020F08D0FEF782F9801B41F28833984206
:1066D800F3D9032077E0E5B9E369002B72D03E4A8D
:1066E800526802F00C02082A56D0022B17D03B4BF6
:1066F80000221A66FEF76AF90446374B1B6813F046
:10670800007F47D0FEF762F9001B0228F5D9032065
:1067180059E0314AD36923F08053D361DCE72F4B2A
:1067280000221A66FEF752F905462B4B1B6813F038
:10673800007F06D0FEF74AF9401B0228F5D903204E
:1067480041E0236AB3F5803F1AD023494B6823F40C
:106758007413226A606A024313434B601F4B012281
:106768001A66FEF733F904461B4B1B6813F0007FCB
:106778000ED1FEF72BF9001B0228F5D9032022E0E1
:10678800154A536823F40033A1680B435360DCE7D0
:10679800002018E0002016E0012B16D00E4B5B6895
:1067A80003F48031226A914211D103F47013626AB2
:1067B80093420ED1002006E001207047012002E03C
:1067C800012000E0002002B070BD0120FBE701209D
:1067D800F9E70120F7E700BF00100240000042423D
:1067E8000F4B5B6803F00C02082A01D00D48704774
:1067F800C3F383420C49885C13F4803F0BD0084BE9
:106808005B68C3F34043094AD35C064A02FB00F0C5
:10681800B0FBF3F07047064B03FB00F0704700BF76
:106828000010024000127A00F4E00108F0E00108CC
:1068380000093D00002800F0A08070B50D46044610
:10684800524B1B6803F007038B420BD24F4A136865
:1068580023F007030B431360136803F007038B420D
:1068680040F08D80236813F0020F17D013F0040F47
:1068780004D0474A536843F4E0635360236813F035
:10688800080F04D0424A536843F460535360404AA7
:10689800536823F0F003A1680B435360236813F097
:1068A800010F31D06368012B20D0022B25D0384A44
:1068B800126812F0020F64D035494A6822F00302C8
:1068C80013434B60FEF782F80646314B5B6803F0D2
:1068D8000C036268B3EB820F16D0FEF777F8801BC3
:1068E80041F288339842F0D9032045E0284A1268DB
:1068F80012F4003FE0D101203EE0254A126812F070
:10690800007FD9D1012037E0204B1B6803F0070333
:10691800AB420AD91D4A136823F007032B431360BF
:10692800136803F00703AB422DD1236813F0040F5B
:1069380006D0174A536823F4E063E1680B435360B9
:10694800236813F0080F07D0114A536823F46053E3
:10695800216943EAC1035360FFF742FF0C4B5B68B0
:10696800C3F303130B4AD35CD8400B4B18600B4B93
:106978001868FDF7E7FF002070BD0120704701206F
:10698800FAE70120F8E70120F6E700BF00200240FF
:1069980000100240D8AE0108000000201C000020B2
:1069A800014B1868704700BF0000002008B5FFF7CA
:1069B800F7FF044B5B68C3F30223034AD35CD84058
:1069C80008BD00BF00100240D0AE010808B5FFF7AF
:1069D800E7FF044B5B68C3F3C223034AD35CD84088
:1069E80008BD00BF00100240D0AE010870B582B0EB
:1069F8000446036813F0010F36D03F4BDB6913F0F0
:106A0800805F49D13C4BDA6942F08052DA61DB6938
:106A180003F080530193019B0125384B1B6813F445
:106A2800807F3BD0344B1B6A13F4407313D06268E9
:106A380002F440729A420ED02F4A136A23F440702F
:106A48002F490126C1F840640026C1F8406410624D
:106A580013F0010F36D1284A136A23F44073616892
:106A68000B431362002D3ED1236813F0020F06D0AA
:106A7800214A536823F44043A1680B4353602368B9
:106A880013F0100F34D01C4A536823F48003616953
:106A98000B43536000202CE00025BEE7174A13681B
:106AA80043F480731360FDF791FF0646134B1B6890
:106AB80013F4807FB6D1FDF789FF801B6428F5D9D0
:106AC800032016E0FDF782FF06460B4B1B6A13F006
:106AD800020FC0D1FDF77AFF801B41F2883398423C
:106AE800F3D9032005E0D36923F08053D361BBE7D2
:106AF800002002B070BD00BF0010024000700040CE
:106B08000000424208B501380F2863D8DFE800F0DA
:106B18003557622F62626232626262626262620842
:106B28002F4B5A68186810F0807054D0C2F3834312
:106B38002C49C85C12F4803F15D0294B5B68C3F31D
:106B48004043294AD25C294BB3FBF2F303FB00F024
:106B5800234B5B6813F4800F3DD14000244BA3FB0B
:106B68000030400837E0234B03FB00F0F0E7FFF765
:106B780037FE30E0FFF734FE2DE0194B1B6A40F278
:106B880002321A40B2F5817F26D003F44073B3F580
:106B9800007F04D0B3F5407F09D000201BE0104AE5
:106BA800526A12F0020FF5D049F6404013E00C4B40
:106BB800186810F400300ED04FF224400BE0FFF7B5
:106BC80005FF074B5B68C3F3813301335B00B0FB00
:106BD800F3F000E0002008BD4FF40040FBE700BFE1
:106BE8000010024008E1010804E1010800127A00DF
:106BF800ABAAAAAA00093D0000B5036899691FFA63
:106C080081FED8699A691FFA82FCE64505D0D869E1
:106C180080B240EA02405DF804FB80B240EA0140DD
:106C2800F9E70368186A5B6A9BB243EA0040704759
:106C3800002302E001330A38C0B20928FAD81B0140
:106C4800DBB218437047030903EB830300F00F001E
:106C580000EB4300C0B2704710F0030F14D10D4B86
:106C6800A3FB00235B09642202FB13039BB26BB9ED
:106C7800084BA3FB0023DB094FF4C87202FB130087
:106C880080B228B901207047002070470120704762
:106C9800002070471F85EB5100F5FA6C022921D8B6
:106CA80001EB4103C1EBC3011E4BA3FB013102EB16
:106CB8005103634400F2CF7003EB90031A4AA2FB1E
:106CC8000020A3EB501303EBD01304331748A0FBA9
:106CD80003201A1A00EB52008008C0EBC000181AF3
:106CE800C0B2704701EB4103C1EBC3010D4BA3FBDD
:106CF800013102EB5103634403EB9C030A4AA2FBF4
:106D08000C12A3EB521303EBD21302330748A0FB78
:106D180003201A1A00EB52008008C0EBC000181AB2
:106D2800DEE700BF398EE3381F85EB5125499224F1
:106D38002DE9F8430746894690F80F80457B867B06
:106D4800002403E01E2E15D8013601344C4533D2F9
:106D58000C2DFAD80123AB4041F2AA521342F1D1CB
:106D680013F4256F10D113F0040FEED01B2E12D898
:106D78000136EAE70C2D02D001350126E5E708F1D6
:106D8800010801263546E0E71D2E01D80136DCE76B
:106D980001350126D9E71C2E04D01D2ED5D1013589
:106DA8000126D2E71FFA88F0FFF756FF08B101362F
:106DB800CBE701350126C8E787F80F80E9B2797378
:106DC800F2B2BA734046FFF767FF3873BDE8F8833D
:106DD80038B50446FDF7FAFD054623685A6812F0EF
:106DE800200F07D1FDF7F2FD401BB0F57A7FF4D9EB
:106DF800032004E05A6842F010025A60002038BDAF
:106E080038B504460268536823F010035360FDF751
:106E1800DDFD054623685B6813F0200F07D1FDF7F9
:106E2800D5FD401BB0F57A7FF4D9032000E000209F
:106E380038BD38B505460C46FFF7CAFF08B1012032
:106E480038BD2B68220C9A612B68A4B2DC612846F5
:106E5800FFF7D6FF0028F3D00120F1E738B5054643
:106E68000C46FFF7B5FF08B1012038BD2B68220C8E
:106E78001A622B68A4B25C622846FFF7C1FF00289B
:106E8800F3D00120F1E770B5002857D00D4606462B
:106E9800002955D0037C012B54D00123037402230D
:106EA8004374BAB90B784C78C4EB0414A4004FF4BB
:106EB800616202FB03448B781C4421463046FFF78D
:106EC800B8FF0546C8B10423737400233374012541
:106ED800284670BD0878FFF7B6FE4FF4616303FBE0
:106EE80000F46878FFF7AFFEC0EB001004EB8004F5
:106EF800A878FFF7A8FE0444DFE73268536823F058
:106F0800050353603046FFF78CFEB0F1FF3F01D018
:106F1800844204D80123737400233374D8E700F53E
:106F2800A83101F5C0713046FFF798FF0028F1D06D
:106F380004237374002333740125C9E70125C7E7C7
:106F48000125C5E70225C3E700286FD02DE9F843DE
:106F58000C461546074600296AD003685B6813F09B
:106F6800040F02D00120BDE8F883FFF745FE06466E
:106F7800334BA3FB0023DB0A4FF4616202FB1302CD
:106F88003049A1FB02014809C1F347116170C0EB08
:106F98000010A2EB8002A2702B4A964210D82370F0
:106FA800002D4BD02078FFF743FE20706078FFF764
:106FB8003FFE6070A078FFF73BFEA0700020D2E78C
:106FC800224AA2FB03284FEA181808EB4802A3EB51
:106FD800C20323703846FFF724FE8146B0F1FF3F15
:106FE80006D0864202D2A0EB060901E04FF0FF3935
:106FF800174B03FB186631463846FFF71AFFC8B926
:10700800B9F1FF3F0AD009EB06013846FFF726FF22
:1070180090B941463846FFF78BFEC1E749463846E6
:10702800FFF71CFF0028F4D001209CE701207047DF
:10703800012098E7012096E7012094E7002092E7D5
:10704800C5B3A291898888887F510100ABAAAAAAF2
:107058008051010000285AD038B50D460446002951
:1070680057D0037C012B56D00123037402234374A9
:10707800BAB9CB78C3734B7843738B788373A27B8D
:10708800617BE07BFFF708FE207328702046FFF73E
:10709800B3FD224B984211D8012363740020207459
:1070A80038BDC878FFF7CFFDE0736878FFF7CBFDF0
:1070B8006073A878FFF7C7FDA073E0E7184DA5FB3C
:1070C80000352D0C174B03FB150529462046FFF705
:1070D800B0FE28B104236374002323740120DFE782
:1070E8002046FFF79EFDB0F1FF3FD5D08542D3D9AA
:1070F80000F5A83101F5C0712046FFF7AFFE002862
:10710800CAD004236374002323740120C8E7012034
:1071180070470120C4E70220C2E700BF8F5F01006B
:1071280007452EC2805101002DE9F04182B00023AD
:10713800ADF804308DF8063000B30C461746054606
:10714800F1B11A4601A9FFF7FFFE0646E8B92B7B05
:107158002370E87BE07095F80D8084F80180AD7BA2
:10716800A57077B1FFF764FDE0704046FFF760FD5A
:1071780060702846FFF75CFDA07002E0012600E081
:107188000126304602B0BDE8F0810126F9E77047D4
:1071980010B5044603681A6812F0020F03D05B6842
:1071A80013F0020F06D1074B4FF400325A61012346
:1071B800637410BDFFF7EBFF2268536823F00203E6
:1071C8005360F0E700040140C0B138B505460268D5
:1071D800536823F008035360FDF7F8FB04462B6857
:1071E8005B6813F0080F07D1FDF7F0FB001BB0F543
:1071F8007A7FF4D9032000E0002038BD01207047D1
:10720800002850D010B50446437C4BB10223637468
:107218002046FFF7D9FF38B104236374012010BD5D
:107228000374FAF777FCF1E72046FFF7D1FD28BB96
:107238002268536823F007035360A36823B11B4AED
:10724800136B23F001031363184AD36A23F46073A2
:10725800A1680B43D3626368B3F1FF3F12D0226881
:10726800C3F30341916022689BB2D3602046FFF7C5
:10727800C7FD88B1042363740120D0E70423637435
:107288000120CCE70120FFF73DFC08B1431EE6E7EB
:10729800042363740120C2E70023E37301236373AB
:1072A800A3736374BBE70120704700BF006C004004
:1072B800704703681A6812F0010F1CD010B5044615
:1072C8005A6812F0010F10D05B6813F0040F0DD04C
:1072D800FFF7EEFF23686FF004025A60042363741B
:1072E8002268536823F00103536010BDFAF764FA6B
:1072F80001236374F4E77047890001F1804101F5C7
:10730800D84192B20A607047890001F1804101F5C5
:10731800D841086880B2704770B582B0044600232F
:107328000193006801F04BFD054610B1284602B0F4
:1073380070BD206802F00CF838B90123A364A36C6F
:10734800012B0BD02E46284614E00023A3642068A6
:1073580001F035FD0028F2D00546E7E70021206856
:1073680001F094FE0028EDD04FF08055DEE7019B38
:1073780001330193019A4FF6FE739A4213D896B9D6
:107388000021206801F082FEE0B91249206801F06E
:107398002BFF0646C0B90021206801F0FBFCC30F93
:1073A800E5D01E46E3E7019A4FF6FE739A420ED8DF
:1073B80010F0804302D001236364B7E700226264BF
:1073C8001D46B3E70546B1E74FF08055AEE74FF0ED
:1073D8008075ABE7000010C170B581B104460E4658
:1073E800016D0904006801F069FE054608B12846E8
:1073F80070BD0021206801F0CDFC3060F7E74FF048
:107408000065F4E72DE9F04F87B005460C461646AF
:107418009B46DDF840A0FDF7D9FA002C36D081460E
:1074280095F83470FFB2012F40F005810023AB635B
:1074380006EB0B03EA6D93422ED8032385F834300C
:107448002B680022DA626B6C012B00D076024FF0B9
:10745800FF3300934FEA4B230193902302930223B7
:10746800039300230493012305936946286801F0D8
:1074780094FCBBF1010F14D902232B633146286811
:1074880001F08AFDA0B9DDF8048038E0AB6B43F069
:107498000063AB630127D3E0AB6B43F00073AB63CE
:1074A800CEE001232B633146286801F05DFDE9E752
:1074B8002B68654A9A63AB6B0343AB63012385F87A
:1074C800343000232B63BBE0286801F040FC2070B7
:1074D800C0F307236370C0F30743A370000EE07086
:1074E8000434A8F104080136072EEDD9FDF76EFA29
:1074F800A0EB0900504510D2BAF1000F0DD0286852
:10750800466B40F22A331E4015D1436B13F4004FEB
:10751800ECD0B8F1000FE9D0E6E72B684A4A9A6345
:10752800AB6B43F00043AB63012385F83430002391
:107538002B63032784E0436B13F4807F05D0BBF1F2
:10754800010F02D96B6C032B38D12B685A6B12F0E0
:10755800080F44D15A6B12F0020F4CD15A6B12F03B
:10756800200F54D12868436B13F4001F5BD0B8F187
:10757800000F58D001F0EBFB2070C0F307236370B5
:10758800C0F30743A370000EE0700434A8F10408A8
:10759800FDF71CFAA0EB0900504502D2BAF1000F22
:1075A800E0D12B68284A9A63AB6B43F00043AB6386
:1075B800012385F8343000232B6341E001F034FDCA
:1075C80003460028C1D02A681F499163AA6B134358
:1075D800AB63012385F8343000232B6330E01A4A6B
:1075E8009A63AB6B43F00803AB63012385F834302F
:1075F80000232B6324E0144A9A63AB6B43F0020325
:10760800AB63012385F8343000232B6318E00E4A5E
:107618009A63AB6B43F02003AB63012385F83430E6
:1076280000232B630CE040F23A538363012385F86F
:107638003430002704E0AB6B43F00053AB63012701
:10764800384607B0BDE8F08FFF0540002DE9F04F40
:107658008BB005460C4616469B46DDF850A0FDF754
:10766800B5F9002C37D0804695F83470FFB2012F59
:1076780040F0E2800023AB6306EB0B03EA6D934214
:107688002FD8032385F834302B680022DA626B6C1C
:10769800012B00D076024FF0FF3304934FEA4B23BF
:1076A80005939023069300230793089301230993D6
:1076B80004A9286801F071FBBBF1010F16D920233A
:1076C8002B633146286801F097FC0190019BABB908
:1076D800DDF8149040E0AB6B43F00063AB63012727
:1076E800AFE0AB6B43F00073AB63AAE010232B63EE
:1076F8003146286801F068FC0190E7E72B68534A97
:107708009A63AB6B019A1343AB63012385F834305A
:1077180000232B6395E023780393627843EA0223DE
:107728000393A27843EA02430393E27843EA0263AD
:1077380003930434A9F1040903A9286801F00AFB9A
:107748000136072EE7D9FDF741F9A0EB08005045AF
:1077580010D2BAF1000F0DD02868466B40F21A33E8
:107768001E4015D1436B13F4804FECD0B9F1000FD4
:10777800E9D0E6E72B68354A9A63AB6B019A134365
:10778800AB63012385F8343000232B63032758E0CB
:10779800436B13F4807F05D0BBF1010F02D96B6CEA
:1077A800032B18D12B685A6B12F0080F24D15A6B8F
:1077B80012F0020F2CD15A6B12F0100F34D0234A5A
:1077C8009A63AB6B43F01003AB63012385F8343045
:1077D80000232B6335E001F027FC03460028E1D0A5
:1077E8002A681A499163AA6B1343AB63012385F88E
:1077F800343000232B6324E0144A9A63AB6B43F0C4
:107808000803AB63012385F8343000232B6318E0A9
:107818000E4A9A63AB6B43F00203AB63012385F80E
:10782800343000232B630CE040F23A529A63012370
:1078380085F83430002704E0AB6B43F00053AB63AA
:10784800012738460BB0BDE8F08F00BFFF054000A8
:107858000346426E920F0A70426EC2F383624A7008
:1078680090F8672002F003028A7090F86620CA70C8
:1078780090F865200A7190F864204A71826E120DA2
:10788800CA80B0F86A2002F00F020A72826EC2F350
:10789800C0324A72826EC2F380328A72826EC2F33A
:1078A8004032CA72826EC2F300320A7300224A73EF
:1078B800426C002A40F08680806E40F6FC7202EA34
:1078C8008002D86E42EA90720A61DA6EC2F3C2622E
:1078D8000A7593F86F2002F007024A75DA6EC2F350
:1078E80042528A75DA6EC2F38242CA75DA6EC2F300
:1078F800C2320A760A6901325A65087E00F007002A
:10790800023082405A6591F808C00CF00F0C012033
:1079180000FA0CF09865400A00FB02F2DA654FF4B1
:1079280000721A66DA6EC2F380324A76DA6EC2F3F1
:10793800C6128A76DA6E02F07F02CA761A6FD20F02
:107948000A771A6FC2F341724A771A6FC2F38262DA
:107958008A771A6FC2F38352CA771A6FC2F34052FA
:1079680081F82020002081F82100B3F8722002F06D
:10797800010281F822201A6FC2F3C03281F8232055
:107988001A6FC2F3803281F824201A6FC2F3403292
:1079980081F825201A6FC2F3003281F826201A6F69
:1079A800C2F3812281F827201A6FC2F3012281F8DD
:1079B80028201B6FC3F3460381F82930012381F87F
:1079C8002A307047012A11D1826E120402F47C1207
:1079D800B0F86E0002430A610A69013292025A65E0
:1079E800DA654FF400729A651A669BE702680549E2
:1079F8009163826B42F080528263012083F83400E5
:107A0800704700BFFF05400070B590B004460123E1
:107A1800ADF81230006801F0A6F900286CD0636C4C
:107A2800032B45D1636C032B5DD1636C032B1DD0F5
:107A3800BDF8121021650904206801F09AFB05467B
:107A480000285BD10021206801F0A4F960660421B8
:107A5800206801F09FF9A0660821206801F09AF9D2
:107A6800E0660C21206801F095F920670421206860
:107A780001F090F9000DE06405A92046FFF7E8FE43
:107A880000283ED1226D12040023206801F0E6FA96
:107A9800054698BB234653F8106B93E807008DE81A
:107AA8000700043494E80E00304601F037F925E069
:107AB800206801F049FB054600BB0021206801F061
:107AC80069F960670421206801F064F9A06708215A
:107AD800206801F05FF9E0670C21206801F05AF98D
:107AE800C4F880009EE70DF11201206801F0E6FB62
:107AF8000546002899D001E04FF08065284610B06F
:107B080070BD4FF08055F9E770B58AB00446002380
:107B180004930593069307930893762309930AAB76
:107B280013E907008DE8070004AB0ECB206801F0CD
:107B3800F5F818B1012528460AB070BD05461A4E59
:107B48000023C6F8A030206801F009F90123C6F81F
:107B5800A0300220FCF740FF2046FFF7DDFB30B1E4
:107B6800012584F83450A36B0343A363E3E720465D
:107B7800FFF74AFF30B1012584F83450A36B034363
:107B8800A363D8E74FF40071206801F0D5F9002805
:107B9800D1D0236805499963A36B0343A3630125E7
:107BA80084F83450C7E700BF00003042FF054000AA
:107BB800A8B110B5044690F8343063B1032384F8B3
:107BC80034302046FFF7A0FF58B9A0632063012393
:107BD80084F8343010BD0377F9F7DCFFEEE70120B5
:107BE80070470120F6E7436C0B60836C4B60C36CF5
:107BF8008B60036DCB60436D0B61836D4B61C36D0F
:107C08008B61036ECB610020704710B582B00446CB
:107C18000023019301A9FFF7DFFB10B1A36B034316
:107C2800A3630198C0F3432002B010BD002856D0CA
:107C380010B50446436A33B94368B3F5827F05D06B
:107C48000023C36102E00023036143610023A362B0
:107C580094F85130002B3CD0022384F8513022682C
:107C6800136823F040031360636803F48273A26807
:107C780002F404421343E26802F4006213432269E7
:107C880002F002021343626902F001021343A2697F
:107C980002F400721343E26902F038021343226AC5
:107CA80002F080021343A26A02F4005221681343CF
:107CB8000B60638B226803F0040353602268D36966
:107CC80023F40063D36100206065012384F85130F8
:107CD80010BD84F850302046F9F7C2FFBCE70120F8
:107CE800704760B370B50E46154604468369B3F510
:107CF800807F26D090F84130E3B1214651F8080B37
:107D080000F072FFA2683146206800F0A1FF236BE3
:107D1800A2682946606800F0C3FF2268A16852F88B
:107D2800213043F0010342F82130012384F8413027
:107D3800002070BD80F84030F9F76AFCDDE70120CB
:107D480070470120F5E710B4036A046A24F00104BF
:107D58000462846924F0F00C4CEA021223F00A034E
:107D68000B438261036210BC704710B4036A046A53
:107D780024F010040462846924F4704C4CEA023242
:107D880023F0A00343EA01138261036210BC704729
:107D9800836823F070030B4343F007038360704745
:107DA80090F83D30DBB2012B2FD1022380F83D3013
:107DB8000268D36843F00103D3600368154A93420D
:107DC80018D002F50062934214D0B3F1804F11D05D
:107DD800A2F5983293420DD002F58062934209D001
:107DE80002F58062934205D01A6842F001021A60D7
:107DF800002070479A6802F00702062A07D01A681E
:107E080042F001021A6000207047012070470020EC
:107E1800704700BF002C01400268D36823F00103BB
:107E2800D3600368196A41F21112114208D1196A24
:107E380040F24442114203D11A6822F001021A604A
:107E4800012380F83D300020704770477047704725
:107E5800704710B5044603681A6912F0020F11D072
:107E6800DA6812F0020F0DD06FF002021A610123D6
:107E7800037703689B6913F0030F70D0FFF7E6FFE1
:107E88000023237723681A6912F0040F12D0DA68E6
:107E980012F0040F0ED06FF004021A610223237748
:107EA80023689B6913F4407F5FD02046FFF7CEFF1D
:107EB8000023237723681A6912F0080F12D0DA68B2
:107EC80012F0080F0ED06FF008021A61042323770E
:107ED8002368DB6913F0030F4ED02046FFF7B6FF87
:107EE8000023237723681A6912F0100F12D0DA687A
:107EF80012F0100F0ED06FF010021A6108232377CA
:107F08002368DB6913F4407F3DD02046FFF79EFFCE
:107F18000023237723681A6912F0010F03D0DA6867
:107F280012F0010F36D123681A6912F0800F03D0BE
:107F3800DA6812F0800F34D123681A6912F0400F02
:107F480003D0DA6812F0400F32D123681A6912F0B0
:107F5800200F03D0DA6812F0200F30D110BDFFF7E0
:107F680074FF2046FFF773FF8AE72046FFF76DFF8F
:107F78002046FFF76CFF9BE72046FFF766FF204689
:107F8800FFF765FFACE72046FFF75FFF2046FFF7E6
:107F98005EFFBDE76FF001021A612046FCF788FC1E
:107FA800C1E76FF080021A61204600F052F9C3E77A
:107FB8006FF040021A612046FFF74AFFC5E76FF0ED
:107FC80020021A61204600F043F9C7E70368244AF3
:107FD800904212D002F5006290420ED0B0F1804F6C
:107FE8000BD0A2F59832904207D002F580629042F9
:107FF80003D002F58062904203D123F070034A68EF
:108008001343174A904212D002F5006290420ED0F4
:10801800B0F1804F0BD0A2F59832904207D002F50C
:108028008062904203D002F58062904203D123F42B
:108038004073CA68134323F080034A6913430360FB
:108048008B68C3620B688362054B984203D003F5C3
:108058000063984201D10B690363012343617047B0
:10806800002C014040B310B5044690F83D30F3B100
:10807800022384F83D30214651F8040BFFF7A6FF90
:10808800012384F8463084F83E3084F83F3084F881
:10809800403084F8413084F8423084F8433084F822
:1080A800443084F8453084F83D30002010BD80F815
:1080B8003C30F9F703FFDBE70120704710B4846810
:1080C80024F47F4C42EA03220A4342EA0C0282600B
:1080D80010BC704790F83C30012B78D010B504469E
:1080E800012380F83C30022380F83D300268936811
:1080F80023F47F4323F0770393600B68602B4CD005
:1081080023D8402B54D011D8202B03D00AD80BB138
:10811800102B05D119462068FFF73AFE002028E009
:10812800012026E0302BF5D0012022E0502B0AD187
:10813800CA6849680068FFF706FE50212068FFF703
:1081480027FE002015E0012013E0B3F5805F3AD048
:10815800B3F5005F14D0702B37D1CB684A688968B3
:108168000068FFF7ABFF2268936843F077039360DA
:108178000020012384F83D30002384F83C3010BDF2
:10818800CB684A6889680068FFF798FF2268936897
:1081980043F4804393600020EBE7CA6849680068AD
:1081A800FFF7E3FD60212068FFF7F2FD0020E0E71C
:1081B800CA6849680068FFF7C6FD40212068FFF7D4
:1081C800E7FD0020D5E70020D3E70120D1E7022012
:1081D8007047000090F83C20012A34D010B40346C0
:1081E800012280F83C20022280F83D200268506875
:1081F800946820F0700C086840EA0C0050601A6817
:108208001248824212D000F5006082420ED0B2F1CC
:10821800804F0BD0A0F59830824207D000F58060DF
:10822800824203D000F58060824204D124F08004A9
:10823800496821439160012283F83D20002083F89A
:108248003C0010BC70470220704700BF002C014062
:1082580070477047026802F10C0353E8003F23F0AF
:10826800C0030C3242E800310029F3D1202380F802
:1082780041307047026802F10C0353E8003F23F4D1
:1082880090730C3242E800310029F3D1026802F100
:10829800140353E8003F23F00103143242E800318D
:1082A8000029F3D1036B012B05D0202380F842303D
:1082B800002303637047026802F10C0353E8003F90
:1082C80023F010030C3242E800310029F3D1ECE727
:1082D80090F84130DBB2212B01D00220704783682F
:1082E800B3F5805F17D0036A5A1C02621A780368D4
:1082F8005A60C38C9BB2013B9BB2C3844BB90268E2
:10830800D36823F08003D3600268D36843F0400346
:10831800D360002070470369002BE4D1036A1B88EF
:108328000268C3F308035360036A02330362E0E799
:1083380010B504460268136923F44053C1680B431F
:10834800136183680269134342691A430168CB6861
:1083580023F4B05323F00C031343CB600268536932
:1083680023F4407381690B4353610268134B9A42AB
:1083780020D0FEF71BFB024602EB820202EB8202D0
:1083880063689B00B2FBF3F20D48A0FB0231490978
:10839800642303FB11231B013233A0FB03035B0996
:1083A80003F0F00202EB011203F00F0321681344FB
:1083B8008B6010BDFEF70AFB0246DDE7003801407E
:1083C8001F85EB512DE9F84305460F461646994699
:1083D800DDF820802B681C6837EA04040CBF0124F0
:1083E8000024B4422DD1B8F1FF3FF3D0B8F1000F0B
:1083F80005D0FCF7EBFAA0EB09004045EAD92A685A
:1084080002F10C0353E8003F23F4D0730C3242E826
:1084180000310029F3D12A6802F1140353E8003F20
:1084280023F00103143242E800310029F3D120235C
:1084380085F8413085F84230002385F84030032024
:1084480000E00020BDE8F88360B310B5044690F85A
:10845800413013B3242384F841302268D36823F4CD
:108468000053D3602046FFF763FF2268136923F4A3
:10847800904313612268536923F02A0353612268E9
:10848800D36843F40053D36000206064202384F849
:10849800413084F84230606310BD80F84030F9F70D
:1084A80061FDD7E7012070472DE9F04182B01E46F3
:1084B80090F84130DBB2202B4BD104460D46904654
:1084C80000294AD00AB9012044E00023436421234B
:1084D80080F84130FCF77AFA0746A4F82480A4F81B
:1084E8002680A368B3F5805F02D04FF000080FE044
:1084F8002369FBB14FF000080AE038F8023B226814
:10850800C3F308035360E28C92B2013A92B2E28458
:10851800E38C9BB28BB100963B460022802120461B
:10852800FFF750FFD8B9002DE7D015F8012B2368C5
:108538005A60E8E7A8460025EAE700963B4600228D
:1085480040212046FFF73EFF58B9202384F84130E8
:1085580000E0022002B0BDE8F0810120FAE7032024
:10856800F8E70320F6E72DE9F04182B01E4690F8BF
:108578004230DBB2202B53D104460D4690460029E9
:1085880052D00AB901204CE000234364222280F82B
:1085980042200363FCF71AFA0746A4F82C80A4F8D3
:1085A8002E80A368B3F5805F02D04FF0000817E073
:1085B800236913B14FF0000812E0A84600250FE028
:1085C80023685B68C3F3080328F8023B03E02368C9
:1085D8005B682B700135E28D92B2013A92B2E28566
:1085E800E38D9BB2BBB100963B460022202120467A
:1085F800FFF7E8FED0B9002DE2D0A368B3F5805F9D
:10860800E5D013B92369002BE1D023685B6803F038
:108618007F032B70DEE7202384F84230002000E03F
:10862800022002B0BDE8F0810120FAE70320F8E754
:10863800704708B50168CA6822F04002CA60202263
:1086480080F84120FFF7F4FF002008BD704770470D
:10865800704710B5446A23685A6994F84130DBB210
:10866800212B10D023685A6902F0400294F8423056
:10867800DBB2222B11D0636C43F0100363642046F5
:10868800FFF7E6FF10BD02F08002002AEAD00023BF
:10869800E3842046FFF7DEFDE4E7002AEBD0002361
:1086A800E3852046FFF7E6FDE5E708B5406A0023C5
:1086B800C385C384FFF7CCFF08BD90F84230DBB216
:1086C800222B69D18368B3F5805F4FD0826AB3F5F6
:1086D800805F04D0002B56D10369002B53D1036867
:1086E8005B681370836A01338362C38D9BB2013B5D
:1086F8009BB2C385002B51D100B583B00268D36803
:1087080023F02003D3600268D36823F48073D36016
:108718000268536923F001035361202380F8423033
:1087280000234363036B012B33D1002303630268E7
:1087380002F10C0353E8003F23F010030C3242E827
:1087480000310029F3D103681A6812F0100F06D01F
:10875800002201921A6801925B680193019B818D46
:10876800F9F706F8002003B05DF804FB0269002A57
:10877800ACD1826A03685B68C3F308031380836A19
:1087880002338362B1E703685B6803F07F03137009
:10879800A8E7FFF75BFFE5E7022070470020704776
:1087A80010B582B0044602681368D068516913F0A6
:1087B8000F0F09D113F0200F0CD010F0200F09D0A3
:1087C8002046FFF77AFF16E011F0010115D110F4E9
:1087D800907F12D1216B012979D013F0800F03D03B
:1087E80010F0800F40F0138113F0400F03D010F009
:1087F800400F40F0108102B010BD13F0010F06D0F9
:1088080010F4807F03D0626C42F00102626413F0BE
:10881800040F04D019B1626C42F00202626413F0D2
:10882800020F04D019B1626C42F00402626413F0C2
:10883800080F07D010F0200F00D119B1626C42F078
:1088480008026264626C002AD5D013F0200F02D0AF
:1088580010F0200F29D123685B6903F04003626C94
:1088680012F0080F00D163B32046FFF703FD236819
:108878005B6913F0400F20D0226802F1140353E81B
:10888800003F23F04003143242E800310029F3D1BD
:10889800E36B73B1624A5A63E06BFCF7E7F90028AF
:1088A800A9D0E06B436B9847A5E72046FFF705FF83
:1088B800D1E72046FFF7CCFE9DE72046FFF7C8FE2C
:1088C80099E72046FFF7C4FE0023636493E713F09B
:1088D800100F82D010F0100F3FF47FAF00230193E8
:1088E8001368019353680193019B536913F0400F78
:1088F80051D0E26B13685B689BB2002B3FF47BAFEF
:10890800A18D99427FF677AFE3859369202B37D005
:10891800226802F10C0353E8003F23F480730C3201
:1089280042E800310029F3D1226802F1140353E828
:10893800003F23F00103143242E800310029F3D14B
:10894800226802F1140353E8003F23F04003143275
:1089580042E800310029F3D1202384F84230002373
:108968002363226802F10C0353E8003F23F010034D
:108978000C3242E800310029F3D1E06BFCF753F9DF
:1089880002236363A18DE38D9BB2C91A89B2204685
:10899800F8F7EEFE2FE7A18DE38D9BB2C91A89B2D5
:1089A800E38D9BB2002B3FF426AF00293FF423AFA1
:1089B800226802F10C0353E8003F23F490730C3251
:1089C80042E800300028F3D1226802F1140353E88A
:1089D800003F23F00103143242E800300028F3D1AD
:1089E800202384F8423000232363226802F10C0319
:1089F80053E8003F23F010030C3242E8003000280F
:108A0800F3D1022363632046F8F7B2FEF3E620466B
:108A1800FFF75EFCEFE62046FFF70BFEEBE600BF34
:108A2800B386000808B5406A01234363036B012B32
:108A380002D0FFF70CFE08BD818D4908F8F798FEB3
:108A4800F9E708B50346406A1B681B6813F0200F56
:108A58002BD10023C385026802F10C0353E8003FC1
:108A680023F480730C3242E800310029F3D1026804
:108A780002F1140353E8003F23F00103143242E8E3
:108A880000310029F3D1026802F1140353E8003FD2
:108A980023F04003143242E800310029F3D12023A7
:108AA80080F84230036B012B07D000234363036B2C
:108AB800012B0FD0FFF7CAFD08BD026802F10C03B5
:108AC80053E8003F23F010030C3242E8003100293C
:108AD800F3D1EAE7818DF8F74BFEEDE730B583B0C7
:108AE800044613468162828500254564222280F867
:108AF8004220C26B1F489062E26B1F48D062E26B53
:108B08001E481063E26B556320680A46011DE06B3E
:108B1800FCF74EF8019523681A6801925B68019387
:108B2800019B23695BB1226802F10C0353E8003F03
:108B380043F480730C3242E800310029F3D12268F3
:108B480002F1140353E8003F43F00103143242E8F2
:108B580000310029F3D1226802F1140353E8003FE1
:108B680043F04003143242E800310029F3D10020D9
:108B780003B030BD4B8A00082D8A00085B860008C8
:108B880090F84230DBB2202B29D110B582B00446D0
:108B980039B312B9012002B010BD012303630023C9
:108BA8004363FFF79BFF0028F5D1236B012B01D00E
:108BB8000120F0E70023019323681A6801925B689B
:108BC8000193019B226802F10C0353E8003F43F034
:108BD80010030C3242E800310029F3D1DBE7022010
:108BE80070470120D7E7000010B40A6850F8223017
:108BF80023F0010340F822308B68082B24D000248E
:108C08004A6822431343CA6813430A6913434A69EB
:108C18001343CA6913430A6A13434A6A13438A6AA5
:108C28001343CA6A13430A6B13438A691A434B6B8B
:108C38001A43096850F82140044B2340134340F875
:108C48002130002010BC70474024D9E78000F0FF95
:108C580000B5013250F8223003F0404C0B68D1F8CF
:108C680004E043EA0E13D1F808E043EA0E23D1F8F2
:108C78000CE043EA0E43D1F810E00EF1FF3E43EA60
:108C88000E53D1F814E0AEF1020E43EA0E6389697F
:108C98000B434CEA030340F8223000205DF804FB44
:108CA800B3F5804F05D06FF0704340F822300020B4
:108CB800704730B450F82230094C1C400B684D689E
:108CC80043EA05138D6843EA05238D692B43C96878
:108CD80043EA01431C4340F82240002030BC70475F
:108CE8000000F0CF0B4B1B680B4AA2FB03235B0A67
:108CF80041F2883202FB03F31A46013B3AB1426B58
:108D080012F0800FF8D0C5238363002070474FF01E
:108D18000040704700000020D34D621084B00DF170
:108D2800040C8CE80E000B461343039A1343049A71
:108D38001343059A1343069A1343426822F4FD42EB
:108D480022F07F0213434360002004B07047D0F83C
:108D5800800070470B68C0F88030002070470323FC
:108D6800036000207047006800F0030070470B683C
:108D780083604B688A681343CA6813430A691343BC
:108D8800C2686FF30B021343C36000207047006989
:108D9800C0B270471430405870470B6843624B6844
:108DA80083628B68CA6813430A6913434A69134389
:108DB800C26A22F0F7021343C3620020704710B55D
:108DC80086B00446002301930293039304934FF45F
:108DD8008063059301A9FFF7CAFF2046FFF782FFCA
:108DE80006B010BD38B504460D46504B1B685049B7
:108DF800A1FB03135B0A03FB02F21346013A002BA3
:108E08005DD0636B13F0450FF7D013F4006FF4D106
:108E1800636B13F0040F06D1636B13F0010F05D0D9
:108E28000120A0634DE00420A0634AE0C523A363AA
:108E38002046FFF7ACFFA84201D0012041E0002105
:108E48002046FFF7A7FF03463A481840C8B3002B4F
:108E580038DB13F0804F38D113F0005F37D113F0AF
:108E6800805F36D113F0006F36D113F0806F36D1A2
:108E780013F0807F36D113F4000F36D113F4800F2E
:108E880036D113F4001F36D113F4801F36D113F4F2
:108E9800802F36D113F4003F36D113F4803F36D1FA
:108EA80013F4004F36D113F4804F36D113F4005F1A
:108EB80036D113F0080F36D04FF4000001E04FF020
:108EC800004038BD4FF00070FBE74020F9E78020F4
:108ED800F7E74FF48070F4E74FF40070F1E74FF4D0
:108EE8008060EEE74FF40060EBE74FF48050E8E76E
:108EF8004FF40050E5E74FF48040E2E74FF40040BC
:108F0800DFE74FF40030DCE74FF48020D9E74FF477
:108F18000020D6E74FF48010D3E74FF40010D0E7D5
:108F28004FF48000CDE74FF48030CAE700000020FE
:108F3800D34D621008E0FFFD30B587B004460191BB
:108F48001025029540230393002304934FF4806374
:108F5800059301A9FFF70BFF41F288322946204605
:108F6800FFF740FF07B030BD30B587B00446019128
:108F78001125029540230393002304934FF4806343
:108F8800059301A9FFF7F3FE41F2883229462046EE
:108F9800FFF728FF07B030BD30B587B00446019110
:108FA8001225029540230393002304934FF4806312
:108FB800059301A9FFF7DBFE41F2883229462046D6
:108FC800FFF710FF07B030BD30B587B004460191F8
:108FD8001825029540230393002304934FF48063DC
:108FE800059301A9FFF7C3FE41F2883229462046BE
:108FF800FFF7F8FE07B030BD30B587B004460191E1
:109008001925029540230393002304934FF48063AA
:10901800059301A9FFF7ABFE41F2883229462046A5
:10902800FFF7E0FE07B030BD30B587B00446002337
:1090380001930C2502954022039204934FF4806318
:10904800059301A9FFF793FE034A29462046FFF737
:10905800C9FE07B030BD00BF00E1F50530B587B0E7
:1090680004460192072502954023039300230493A5
:109078004FF48063059301A9FFF779FE41F2883226
:1090880029462046FFF7AEFE07B030BD30B587B0A1
:109098000446019137250295402303930023049346
:1090A8004FF48063059301A9FFF761FE41F288320E
:1090B80029462046FFF796FE07B030BD30B587B089
:1090C800044601910D250295402303930023049340
:1090D8004FF48063059301A9FFF749FE41F28832F6
:1090E80029462046FFF77EFE07B030BD0146144BE7
:1090F8001B68144AA2FB03235B0A41F2883202FB75
:1091080003F31A46013BBAB14A6B12F0450FF8D087
:1091180012F4006FF5D14B6B13F0040F06D1486BB6
:1091280010F0010005D1C5238B63704704208863C4
:1091380070470120886370474FF00040704700BFB8
:1091480000000020D34D621010B586B004460023FD
:10915800019302220292C022039204934FF4806387
:10916800059301A9FFF703FE2046FFF7BFFF06B0EE
:1091780010BD10B586B00446019109230293C0239F
:109188000393002304934FF48063059301A9FFF729
:10919800EEFD2046FFF7AAFF06B010BD0146104BB2
:1091A8001B68104AA2FB03235B0A41F2883202FBC8
:1091B80003F31A46013B82B14A6B12F0450FF8D00F
:1091C80012F4006FF5D1486B10F0040002D1C523EA
:1091D8008B6370470420886370474FF000407047E6
:1091E80000000020D34D621010B586B0044641F04F
:1091F800004141F4801101912923029340230393F4
:10920800002304934FF48063059301A9FFF7AFFD92
:109218002046FFF7C3FF06B010BD0000F8B50546AD
:109228000E461746234B1B68234AA2FB03235B0AFF
:1092380041F2883202FB03F31A46013B8AB36C6B96
:1092480014F0450FF8D014F4006FF5D16B6B13F0E0
:10925800040F06D16B6B13F0010F05D00120A86332
:1092680021E00420A8631EE02846FFF790FDB042E5
:1092780001D0012017E0C523AB6300212846FFF782
:1092880089FD034610F4604008D013F4804F0BD1D9
:1092980013F4004F0BD04FF4805004E01B0C3B80BC
:1092A80001E04FF00040F8BD4FF40050FBE74FF4E9
:1092B8008030F8E700000020D34D621070B586B00A
:1092C80004460D460023019303260296402203928A
:1092D80004934FF48063059301A9FFF748FD2A46DC
:1092E80031462046FFF79AFF06B070BD0146164B7F
:1092F8001B68164AA2FB03235B0A41F2883202FB71
:1093080003F31A46013BE2B14A6B12F0450FF8D05D
:1093180012F4006FF5D14B6B13F0040F0BD14B6BAC
:1093280013F001030AD1486B10F040000BD0402223
:109338008A63184670470420886370470120886351
:1093480070474FF00040704700000020D34D621076
:1093580010B586B004464FF4D573019308230293E1
:1093680040230393002304934FF48063059301A9DA
:10937800FFF7FDFC2046FFF7B9FF06B010BD84B02B
:1093880001A880E80E00002004B0704703460020C2
:10939800A3F844004FF43F42A3F840207047B0F8C8
:1093A800403023F47C535B045B0CA0F84030002071
:1093B80070470020704784B0844601A880E80E00FA
:1093C8000123ACF840300020ACF84000ACF8440071
:1093D800ACF8500004B07047002070470020704778
:1093E80010B5034691F800C030F82C2092B222F450
:1093F800EC4222F0700292B2C878032861D8DFE804
:1094080000F0555C0258002048F2800E42EA0E0235
:1094180023F82C2091F800C033F82C2092B222F4C3
:10942800E04222F0700242EA0C0242EA0E0223F8FD
:109438002C200A7B002A40F0DC804A78002A51D090
:10944800B3F8502092B21A440C7802EB0412B1F827
:1094580006C04FEA5C0C4FEA4C0CA2F800C40C782A
:1094680033F8242012F0400F0CD033F8242092B2A5
:1094780022F4E04222F0700242F4004242F0C002BC
:1094880023F82420CA78012A1DD0097833F821202E
:1094980092B222F4E04222F0400282F0200242F42A
:1094A800004242F0800223F8212017E142F40072C2
:1094B800AAE742F4C0620020A6E742F480620020D6
:1094C800A2E70120A0E7097833F8212092B222F41C
:1094D800E04222F0400242F4004242F0800223F8C7
:1094E8002120FBE0B3F8502092B21A440C7802EB2A
:1094F8000412B1F806C04FEA5C0C4FEA4C0CA2F813
:1095080008C4B3F8502092B21A440C7802EB041243
:10951800B2F80CC4CCF3090CA2F80CC40C693E2CAC
:1095280039D94FEA541E14F01F0F01D10EF1FF3E36
:10953800B2F80CC41FFA8CFC4FEA8E2E1FFA8EFE6E
:109548004CEA0E0C4CF4004CA2F80CC40C7833F81E
:10955800242012F4804F0CD033F8242092B222F445
:10956800E04222F0700242F4404242F0800223F8C6
:109578002420097869BB33F8212092B222F4804272
:1095880022F0700282F4405242F4004242F080021B
:1095980023F82120A2E04CB9B2F80C446FEA444405
:1095A8006FEA5444A4B2A2F80C44CFE74FEA540C33
:1095B80014F0010F01D00CF1010CB2F80C44A4B264
:1095C8004FEA8C2C1FFA8CFC44EA0C04A2F80C44D9
:1095D800BCE733F8212092B222F4804222F07002D4
:1095E80082F4005242F4004242F0800223F8212023
:1095F80074E0CA78022A72D00C7833F8242092B228
:1096080022F4E24222F0700242F4004242F0800268
:1096180023F82420B3F8502092B21A4491F800C0DD
:1096280002EB0C12B1F808C04FEA5C0C4FEA4C0C84
:10963800A2F800C4B3F8502092B21A4491F800C0BE
:1096480002EB0C12B1F80AC04FEA5C0C4FEA4C0C62
:10965800A2F808C44A78002A50D10C7833F824209C
:1096680012F4804F0CD033F8242092B222F4E04256
:1096780022F0700242F4404242F0800223F8242093
:109688000C7833F8242012F0400F0CD033F8242043
:1096980092B222F4E04222F0700242F4004242F018
:1096A800C00223F8242091F800C033F82C2092B28D
:1096B80022F4804222F0700282F4405248F2800480
:1096C800224323F82C20097833F8212092B222F47F
:1096D800E04222F04002224323F8212010BD0C78FA
:1096E80033F8242092B222F4E04222F0700242F4CD
:1096F800014242F0800223F824208BE70C7833F8EB
:10970800242012F4804F0CD033F8242092B222F493
:10971800E04222F0700242F4404242F0800223F814
:1097280024200C7833F8242012F0400F0CD033F8A2
:10973800242092B222F4E04222F0700242F4004265
:1097480042F0C00223F82420CA78012A1ED00C78DF
:1097580033F8242092B222F4E04222F0400282F050
:10976800200242F4004242F0800223F824200978C3
:1097780033F8212092B222F4804222F0700242F49F
:10978800004242F0800223F82120A7E70C7833F842
:10979800242092B222F4E04222F0400242F4004235
:1097A80042F0800223F82420E1E70B7B002B46D10E
:1097B8004B7813B30A7830F8223013F0400F0CD0EE
:1097C80030F822309BB223F4E04323F0700343F4D3
:1097D800004343F0C00320F822300A7830F82230E2
:1097E8009BB223F4E04323F0400343F4004343F0E7
:1097F800800320F82230002070470A7830F82230A1
:1098080013F4804F0CD030F822309BB223F4E0439D
:1098180023F0700343F4404343F0800320F82230E0
:109828000A7830F822309BB223F4804323F0700387
:1098380043F4004343F0800320F82230DBE74B7801
:10984800002B4ED10A7830F8223013F4804F0CD018
:1098580030F822309BB223F4E04323F0700343F442
:10986800404343F0800320F822300A7830F8223051
:1098780013F0400F0CD030F822309BB223F4E043B1
:1098880023F0700343F4004343F0C00320F8223070
:109898000A7830F822309BB223F4E04323F07003B7
:1098A80043F4004343F0C00320F822300A7830F82C
:1098B80022309BB223F4804323F0700348F2800CDB
:1098C80043EA0C0320F822300A7830F822309BB2A1
:1098D80023F4E04323F0400343EA0C0320F822304A
:1098E80089E70A7830F8223013F4804F0CD030F82A
:1098F80022309BB223F4E04323F0700343F4404347
:1099080043F0800320F822300A7830F8223013F030
:10991800400F0CD030F822309BB223F4E04323F000
:10992800700343F4004343F0C00320F822300A7860
:1099380030F822309BB223F4E04323F0700343F461
:10994800404343F0800320F822300A7830F8223070
:109958009BB223F4E04323F0400348F2800C43EA2F
:109968000C0320F822300A7830F822309BB223F416
:10997800804323F0700343EA0C0320F822303AE7CF
:109988004B788BB10A7830F822309BB223F4E0434D
:1099980023F0400383F0100343F4004343F08003B3
:1099A80020F82230002070470A7830F822309BB225
:1099B80023F4804323F0700383F4805343F400437B
:1099C80043F0800320F82230ECE70B7B002B4BD1CF
:1099D8004B7833B30A7830F8223013F0400F0CD0AC
:1099E80030F822309BB223F4E04323F0700343F4B1
:1099F800004343F0C00320F82230CB78012B33D04A
:109A08000A7830F822309BB223F4E04323F0400375
:109A180083F0200343F4004343F0800320F822300E
:109A280022E00A7830F8223013F4804F0CD030F856
:109A380022309BB223F4E04323F0700343F4404305
:109A480043F0800320F822300A7830F822309BB2A5
:109A580023F4804323F0700383F4405343F400431A
:109A680043F0800320F822300020704711B980238A
:109A7800A0F84C3000207047002070470020704745
:109A8800B0F8440080B270470020704701335B088B
:109A980000EB420000F5806008E00A7891F801C008
:109AA80042EA0C2220F8042B0231013B002BF4D1AE
:109AB800704770B505460C464A78012A3BD00B7BA7
:109AC800002B40F0A6828B690A69934240F2848297
:109AD8009B1A8B61B5F850309BB22B44217803EB6D
:109AE8000113B3F80C14C1F30901A3F80C143E2AAE
:109AF80040F27682510912F01F0F00D10139B3F8F4
:109B08000C2492B2890289B20A4342F40042A3F8B3
:109B18000C24227835F822309BB223F4804323F0BA
:109B2800700383F4405343F4004343F0800325F863
:109B38002230002070BD8E6909698E4200D90E4618
:109B4800237B73B3E378022B4DD0236A9B1B2362DC
:109B5800217835F8213013F0400F00F0F581002A04
:109B680040F0E281B5F850309BB22B4403EB01136F
:109B7800B3F80C24C2F30902A3F80C243E2E40F2D9
:109B8800BA81710916F01F0F00D10139B3F80C24FE
:109B980092B2890289B20A4342F40042A3F80C2423
:109BA800CBE1B6B23346E28861692846FFF76EFF1B
:109BB800B5F850309BB22B44227803EB0213A3F87C
:109BC8000464227835F822309BB223F4E04323F072
:109BD800400383F0300343F4004343F0800325F847
:109BE80022300020A6E7236A994280F06681227815
:109BF80035F822309BB223F4E04323F0700343F49A
:109C0800014343F0800325F82230236A9B1B23621B
:109C1800227835F8223013F0400F00F0A7806378DF
:109C2800B3BBB5F850309BB22B4403EB0213B3F827
:109C38000C24C2F30902A3F80C243E2E0FD9710993
:109C480016F01F0F00D10139B3F80C2492B2890223
:109C580089B20A4342F40042A3F80C241AE04EB930
:109C6800B3F80C246FEA42426FEA524292B2A3F868
:109C78000C240FE0720816F0010F00D00132B3F87F
:109C88000C1489B2920292B20A43A3F80C2401E0A0
:109C9800012B30D0B3B2628961692846FFF7F6FE1E
:109CA800636933446361236A226993422DD99B1BFC
:109CB80023626378002B45D1B5F850309BB22B4412
:109CC800227803EB0213B3F80424C2F30902A3F8C1
:109CD80004243E2E1DD9710916F01F0F00D1013939
:109CE800B3F8042492B2890289B20A4342F40042CA
:109CF800A3F8042428E0B5F850309BB22B4403EBBA
:109D08000213B2B2A3F80C24C4E7002222621E4652
:109D1800CFE74EB9B3F804246FEA42426FEA5242E1
:109D280092B2A3F804240FE0720816F0010F00D0D5
:109D38000132B3F8041489B2920292B20A43A3F82A
:109D4800042401E0012B06D0B3B2228961692846B8
:109D5800FFF79CFE35E7B5F850309BB22B442278CC
:109D680003EB0213B2B2A3F80424EDE76378B3BBA4
:109D7800B5F850309BB22B4403EB0213B3F804241C
:109D8800C2F30902A3F804243E2E0FD9710916F074
:109D98001F0F00D10139B3F8042492B2890289B2A5
:109DA8000A4342F40042A3F804241AE04EB9B3F877
:109DB80004246FEA42426FEA524292B2A3F80424A2
:109DC8000FE0720816F0010F00D00132B3F8041446
:109DD80089B2920292B20A43A3F8042401E0012B4B
:109DE80030D0B3B2228961692846FFF74FFE636914
:109DF80033446361236A226993422DD99B1B2362F2
:109E08006378002B45D1B5F850309BB22B442278AB
:109E180003EB0213B3F80C24C2F30902A3F80C24D1
:109E28003E2E1DD9710916F01F0F00D10139B3F864
:109E38000C2492B2890289B20A4342F40042A3F880
:109E48000C2428E0B5F850309BB22B4403EB0213E6
:109E5800B2B2A3F80424C4E7002222621E46CFE768
:109E68004EB9B3F80C246FEA42426FEA524292B2FA
:109E7800A3F80C240FE0720816F0010F00D001328D
:109E8800B3F80C1489B2920292B20A43A3F80C24D4
:109E980001E0012B06D0B3B2628961692846FFF759
:109EA800F5FD8EE6B5F850309BB22B44227803EBD3
:109EB8000213B2B2A3F80C24EDE7217835F821207B
:109EC80092B222F4E24222F0700242F4004242F0DE
:109ED800800225F82120B5F8502092B22A44217832
:109EE80002EB01129BB2A2F8043422896169284668
:109EF800FFF7CCFD65E64EB9B3F80C246FEA424291
:109F08006FEA524292B2A3F80C2416E0720816F0D7
:109F1800010F00D00132B3F80C1489B2920292B248
:109F28000A43A3F80C2408E0B5F850309BB22B4440
:109F380003EB0113B2B2A3F80C24B3B262896169CE
:109F48002846FFF7A3FD3CE6B2BBB5F850309BB2FC
:109F58002B4403EB0113B3F80424C2F30902A3F85A
:109F680004243E2E0FD9710916F01F0F00D10139B4
:109F7800B3F8042492B2890289B20A4342F4004237
:109F8800A3F8042421E04EB9B3F804246FEA42424E
:109F98006FEA524292B2A3F8042416E0720816F04F
:109FA800010F00D00132B3F8041489B2920292B2C0
:109FB8000A43A3F8042408E0B5F850309BB22B44B8
:109FC80003EB0113B2B2A3F80424B3B22289616986
:109FD8002846FFF75BFDF4E500228A611A4679E519
:109FE8004AB9B3F80C246FEA42426FEA524292B27D
:109FF800A3F80C248DE5510812F0010F00D00131AF
:10A00800B3F80C2492B2890289B20A43A3F80C244B
:10A018007FE5CB78022B4DD0012B40F02F81896949
:10A028002369994240F2E680C91AA161F2B9B5F8EC
:10A03800502092B22A44217802EB0112B2F804149B
:10A04800C1F30901A2F804143E2B40F2D780580945
:10A0580013F01F0F00D10138B2F8041489B280023E
:10A0680080B2014341F40041A2F804146278002A46
:10A0780040F0F680B5F8502092B22A44217802EBDD
:10A088000112B2F80C14C1F30901A2F80C143E2B0A
:10A0980040F2CD80590913F01F0F00D10139B2F8F1
:10A0A8000C349BB2890289B20B4343F40043A2F8F3
:10A0B8000C342EE5F2B9B0F850309BB203440A785C
:10A0C80003EB0213B3F80424C2F30902A3F804242F
:10A0D8000A693E2A31D9510912F01F0F00D10139FE
:10A0E800B3F8042492B2890289B20A4342F40042C6
:10A0F800A3F804246378002B51D1B5F850309BB2F3
:10A108002B44227803EB0213B3F80C24C2F30902A0
:10A11800A3F80C2422693E2A28D9510912F01F0FEE
:10A1280000D10139B3F80C2492B2890289B20A43EA
:10A1380042F40042A3F80C2433E04AB9B3F80424EB
:10A148006FEA42426FEA524292B2A3F80424D1E77E
:10A15800510812F0010F00D00131B3F8042490B275
:10A168008A0292B20243A3F80424C3E74AB9B3F8B7
:10A178000C246FEA42426FEA524292B2A3F80C24CE
:10A188000FE0510812F0010F00D00131B3F80C2490
:10A1980090B28A0292B20243A3F80C2401E0012B88
:10A1A8001DD0E369002B3FF4B4AC227835F82210B7
:10A1B80044F2400303EA01008B4302D000287FF4F5
:10A1C800A8AC35F822309BB223F4E04323F07003A7
:10A1D80043F4004343F0C00325F8223099E4B5F86E
:10A1E80050309BB22B44227803EB0213228AA3F847
:10A1F8000C24D6E70023A3610B4617E74BB9B2F846
:10A2080004146FEA41416FEA514189B2A2F804147B
:10A218002CE7590813F0010F00D00131B2F80404FB
:10A2280080B2890289B20143A2F804141EE74BB92F
:10A23800B2F80C346FEA43436FEA53439BB2A2F877
:10A248000C3466E4590813F0010F00D00131B2F85C
:10A258000C3498B28B029BB20343A2F80C3458E436
:10A26800012A7FF456ACB5F8502092B22A442178DE
:10A2780002EB01129BB2A2F80C344AE4012059E423
:10A2880010B45C0800EB420000F5806007E030F88D
:10A29800042B0A70C2F307224A700231013C002CD9
:10A2A800F5D113F0010F01D003880B7010BC704773
:10A2B80038B51D4C21461D4803F07EF91C4B18701B
:10A2C800012221461B4802F01DFC1B4B187018BBCD
:10A2D8001A4805F067F91A4805F064F9194D686DD0
:10A2E800F6F706FB0446A86DF6F702FB2146F6F7DB
:10A2F80057FB4FF06A51F6F753FB4FF06A51F6F7E8
:10A308004FFBF6F7D1F802460B460F4805F0EAF87E
:10A318000E4B01221A7038BD0D4805F043F90B4B5E
:10A3280000221A70F7E700BF9414002030E10108FA
:10A33800981400206412002020000020E0A90108E1
:10A3480090AB0108F8080020A4AB0108DC08002045
:10A35800C4AB01080020704700B583B000931346D2
:10A368000A4601460348FDF74DF800B1012003B045
:10A378005DF804FBF808002000B583B0009313468D
:10A388000A4601460348FDF761F900B1012003B010
:10A398005DF804FBF808002008B50348FDF735FC14
:10A3A800043818BF012008BDF808002008B5014688
:10A3B8000148FDF718FC08BDF808002082B0012309
:10A3C8008DF807309DF8070002B0704708B5FFF711
:10A3D800F5FF012801D0012008BD0248FDF7E8FB80
:10A3E800FAE700BFF80800202023038000487047E0
:10A3F8007000002020230380004870475000002090
:10A408002023038000487047300000200A2303807F
:10A41800004870472400002038B50446037CE3B99F
:10A428004FF400730222012103F0AAFA0125C4F8AF
:10A438006C514FF4007302228121204603F0A0FAE8
:10A44800E5624FF41B7003F0FBFAC4F8B802A0B140
:10A45800204600F042F9002038BD402302220121A5
:10A4680003F08EFA0125C4F86C51402302228121A1
:10A47800204603F085FAE562E3E70220ECE738B509
:10A488000446012103F087FA0025C4F86C518121A4
:10A49800204603F080FAE562204600F04AF9D4F835
:10A4A800B80218B103F0D0FAC4F8B852002038BD89
:10A4B8002DE9F04182B006460C46D0F8B872002368
:10A4C800ADF806300B7813F0600536D0202D40F03B
:10A4D800B4804A78FE2A05D0FF2A1DD000F0B1FECC
:10A4E8000225ADE04A8812B9CA88012A05D021465A
:10A4F800304600F0A6FE0225A2E013F0800FF6D049
:10A50800D0F8BC329B6998473860012239463046FA
:10A5180001F0A4F9002593E04A8842B9CA8832B903
:10A5280013F0800F03D100F0F7F8002588E02146EA
:10A53800304600F086FE022582E091F80180B8F1ED
:10A548000B0F76D8DFE808F0062D757575757575EB
:10A558007575152290F89C32032B03D000F071FE1C
:10A5680002256DE002220DF1060101F077F945465A
:10A5780066E090F89C32032B03D000F062FE0225BF
:10A588005EE00122391D01F069F959E090F89C322A
:10A59800032B02D18B787B6052E000F052FE02253B
:10A5A8004EE0097903F0FFF92179304603F0F3F919
:10A5B800A38894F90420002A19DB03F00F0303EBA6
:10A5C800830306EB83030022C3F85821337C4BBB7B
:10A5D8004FF4007302220121304603F0D1F9012320
:10A5E800C6F86C312179304600F04EF928E003F0C6
:10A5F8000F0303EB830306EB830300229A61337C8A
:10A608004BB94FF4007302228121304603F0B8F9A8
:10A618000123F362E6E7402302228121304603F05A
:10A62800AFF9F5E7402302220121304603F0A8F9EB
:10A63800D5E700F006FE022502E000F002FE022542
:10A64800284602B0BDE8F08108B500F093F8002074
:10A6580008BD08B500F000F9002008BD09B1C0F830
:10A66800BC120020704710B51346D0F8B842D4F891
:10A6780014229C469A4200D293B2D4F83422A2EB18
:10A688000C02C4F83422002284F8382204222272F0
:10A698000A46812103F0BEF910BD38B50446D0F84A
:10A6A800B85295F8183223B9D5F814320BB16B7A31
:10A6B8003BB18121204603F07EF96B7A022B04D04E
:10A6C80038BD012103F077F9F3E71F2305F503727D
:10A6D8000121204603F0A6F9F2E738B50446D0F880
:10A6E800B85200202872687285F85D0285F85C020D
:10A6F800D4F8BC321B6898470121204603F053F96F
:10A708008121204603F04FF91F2305F5037201212B
:10A71800204603F087F938BD08B5D0F8B8220023E1
:10A728001372012151721F2302F5037203F07AF9A3
:10A7380008BDD0F8B83200221A72704738B50546FD
:10A74800D0F8B8420A4BC4F82C3284F838120023E7
:10A7580023720D2304F50B72812103F05BF91F238B
:10A7680004F503720121284603F05CF938BD00BFE7
:10A778005553425310B50446D0F8B8120B7A022B41
:10A7880008D006D3033BDBB2012B02D80021FFF728
:10A79800D5FF10BD01F21B2291F8191200F060FBE1
:10A7A8000028F6DA01212046FFF7C8FFF1E700008C
:10A7B80038B50546D0F8B842D4F81032C4F830326B
:10A7C800D4F81432C4F83432012103F033F91F28C5
:10A7D80004D1D4F80C221F4B9A420CD02023052216
:10A7E80094F81912284600F0EFF8022363722846FD
:10A7F800FFF753FF38BD94F819120129EED894F8E1
:10A808001A32002BEAD0102BE8D804F21B22284673
:10A8180000F026FB00280CDB237A013BDBB2022B7D
:10A82800E8D962898AB104F10C012846FFF71BFFB9
:10A83800E0E7237A052B03D02846FFF72EFFD9E758
:10A8480001212846FFF77AFFD4E700212846FFF7C1
:10A8580075FFCFE75553424310B50446D0F8B832D8
:10A868001A7A72B1012A0ED103F21B2293F8191237
:10A8780000F0F6FA002806DA01212046FFF75EFF0D
:10A8880001E0FFF795FF10BD10B5D0F8B842637A24
:10A89800022B08D011F0800F04D0012B02D0012127
:10A8A800FFF74CFF10BD812103F085F80023637288
:10A8B800F8E7000010B4D0F8B842537813F0010F4D
:10A8C8000DD00723638105E0013B9BB20F4AD15CA1
:10A8D800E2181173002BF7D1002010BC7047D0F894
:10A8E800BC32D86901EBC10100EB81000179053167
:10A8F80013798B4200D90B46638104E0013B9BB27C
:10A90800C15CE2181173002BF8D1E5E728E10108D2
:10A91800D0F8B8020823438105E0013B9BB2044A02
:10A92800D15CC2181173002BF7D10020704700BF0B
:10A9380020E10108D0F8B8020823438105E0013B73
:10A948009BB2044AD15CC2181173002BF7D10020C6
:10A95800704700BF18E1010810B4D0F8B8420023CE
:10A9680004E0E118002008730133DBB2112BF8D999
:10A97800702323730C23E37494F85C3294F85D120B
:10A988008B420FD003F1470104EBC1010879A07392
:10A99800487A2076097A61760133DBB284F85C3232
:10A9A800042B08D0122363811379122B00D86381FA
:10A9B800002010BC7047002384F85C32F2E7D0F81E
:10A9C800B832002058817047D0F8B80290F85D324C
:10A9D80003F1470100EBC1010A7100220A72013339
:10A9E800DBB280F85D32042B00D0704780F85D221E
:10A9F800FBE770B50446D0F8B862D6F814324BB904
:10AA08000D46D0F8BC329B680846984758B90023D1
:10AA1800738170BD2023052296F81912FFF7D4FF21
:10AA28004FF0FF30F5E73A23022229462046FFF788
:10AA3800CBFF052333724FF0FF30EAE770B582B0E1
:10AA480005460E46D0F8B842002306E0E2184FF05B
:10AA5800000C82F80CC001339BB20B2BF6D9D5F849
:10AA6800BC325B680DF10602694630469847D0B99A
:10AA78000823E373009A531E190E2174C3F3074188
:10AA88006174C3F30723A374013AE27402232375A4
:10AA9800BDF80630002262751A0AA275E3750C2308
:10AAA800638102B070BD3A23022231462846FFF77F
:10AAB8008BFF4FF0FF30F4E770B505460E46D0F82F
:10AAC800B842D0F8BC325B6804F25E2204F5187113
:10AAD80030469847B8B9D4F86022531E190E21732E
:10AAE800C3F307416173C3F30723A373013AE27306
:10AAF800B4F85E320022227462741A0AA274E374F3
:10AB08000823638170BD3A23022231462846FFF7A5
:10AB18005BFF4FF0FF30F5E708B51A44D0F8B832BC
:10AB2800D3F860329A4201D8002008BD21230522BB
:10AB3800FFF74AFF4FF0FF30F7E72DE9F8430646E5
:10AB48000F46D0F8B842D4F86852B4F85E3203FB26
:10AB580005F5B5F5007F28BF4FF40075D0F8BC2285
:10AB6800D2F8109004F10C08B5FBF3F39BB2D4F8BB
:10AB7800642241463846C84700281DDBABB242462E
:10AB88008121304602F046FFD4F86432B4F85E22E0
:10AB9800B5FBF2F21344C4F86432D4F868329B1A55
:10ABA800C4F86832D4F83422521BC4F8342263B98A
:10ABB80003232372002009E011230422394630467A
:10ABC800FFF702FF4FF0FF3000E00020BDE8F883F8
:10ABD800F8B506460F46D0F8B842237A73BB154637
:10ABE80094F91832002B31DAD0F8BC329B68084649
:10ABF8009847A0BBAA78EB781B0443EA02632A793A
:10AC080043EA02236A791A43C4F86422E9792B7A61
:10AC180043EA0123C4F8683239463046FFF77CFF1F
:10AC280000282FDB02232372D4F81422D4F86832C8
:10AC3800B4F85E1201FB03F39A4219D14FF4007382
:10AC4800638139463046FFF778FFF8BD2023052297
:10AC580094F81912FFF7B8FE4FF0FF30F5E73A23E2
:10AC6800022239463046FFF7AFFE4FF0FF30ECE7DF
:10AC78002023052294F819123046FFF7A5FE4FF05D
:10AC8800FF30E2E74FF0FF30DFE72DE9F8430646F3
:10AC98008846D0F8B842D4F86852B4F85E3203FB5C
:10ACA80005F5B5F5007F28BF4FF40075D0F8BC2234
:10ACB800D2F8149004F10C07B5FBF3F39BB2D4F867
:10ACC800642239464046C84700281ADBD4F8642273
:10ACD800B4F85E32B5FBF3F10A44C4F86422D4F840
:10ACE8006822521AC4F86822D4F83412491BC4F8EE
:10ACF80034127AB900213046FFF720FD0020BDE864
:10AD0800F8830323042241463046FFF75DFE4FF0E7
:10AD1800FF30F4E702FB03F3B3F5007F28BF4FF4DD
:10AD280000739BB23A460121304602F07BFE0020B8
:10AD3800E5E72DE9F04106460F46D0F8B842237AF8
:10AD4800002B6AD1154694F91832002B40DBD0F855
:10AD5800BC329B6808469847002842D1D6F8BC32D6
:10AD6800DB68384698478046002843D1AA78EB78B4
:10AD78001B0443EA02632A7943EA02236A791A43E5
:10AD8800C4F86422E9792B7A43EA0123C4F86832CB
:10AD980039463046FFF7C0FE002842DBD4F8683257
:10ADA800B4F85E2202FB03F3D4F814229A422AD1A3
:10ADB800B3F5007F28BF4FF40073012121729BB2C5
:10ADC80004F10C02304602F02DFE4046BDE8F08149
:10ADD8002023052294F81912FFF7F6FD4FF0FF38EB
:10ADE800F3E73A23022239463046FFF7EDFD4FF0EC
:10ADF800FF38EAE72723022239463046FFF7E4FD09
:10AE08004FF0FF38E1E72023052294F81912304665
:10AE1800FFF7DAFD4FF0FF38D7E7FFF736FF804638
:10AE2800D3E74FF0FF38D0E710B5D0F8B8425378E1
:10AE380013F0020F0AD1D4F86832D4F86422FFF76D
:10AE48006BFE002809DB0020608110BD2423052249
:10AE5800FFF7BAFD4FF0FF30F7E74FF0FF30F4E7A8
:10AE680008B513785A2B5FD8DFE803F02E5E5E3200
:10AE78005E5E5E5E5E5E5E5E5E5E5E5E5E5E365E12
:10AE88005E5E5E5E5E5E423A5E5E3E5E5E5E5E4A4E
:10AE98005E4E5E5E525E565E5E5E5E5A5E5E5E5EF2
:10AEA8005E5E5E5E5E5E5E5E5E5E5E5E5E5E5E5EBA
:10AEB8005E5E5E5E5E5E5E5E5E5E5E5E5E5E5E5EAA
:10AEC8005E5E5E5E5E5E4600FFF793FD002008BD95
:10AED800FFF742FD0020FAE7FFF7ECFC0020F6E759
:10AEE800FFF76DFD0020F2E7FFF769FD0020EEE7B0
:10AEF800FFF70EFD0020EAE7FFF71CFD0020E6E75C
:10AF0800FFF79CFD0020E2E7FFF7D6FD0020DEE713
:10AF1800FFF75EFE0020DAE7FFF70BFF0020D6E719
:10AF2800FFF782FF0020D2E720230522FFF74CFD20
:10AF38004FF0FF30CBE798B108B50346D0F8B4021C
:10AF480010B10020C3F8B40209B1C3F8B01201214E
:10AF580083F89C121A70184602F0D0FC002008BD35
:10AF68000220704719B1C0F8B412002070470220BF
:10AF7800704708B502F0FCFC002008BD08B5D0F801
:10AF8800B4322BB11B68984700B908BD0220FCE712
:10AF98000220FAE708B5D0F8B4325B689847002079
:10AFA80008BD38B5044600F52A75284600F035F97D
:10AFB8000123C4F89432B4F8AE32C4F8983294F845
:10AFC800A81201F01F03012B08D0022B0BD07BB96C
:10AFD8002946204600F0D0FA002038BD29462046F0
:10AFE80000F0FEFAF8E72946204600F029FBF3E7CF
:10AFF80001F08001204602F0DEFCEDE738B504469A
:10B008000D4691BB1346D0F89422032A03D0052A93
:10B0180024D0084633E0D0F86011D0F8642191427A
:10B028000DD9891AC0F860118A4206D98AB2194620
:10B03800204600F028FC284621E092B2F7E7D0F835
:10B04800B4321B691BB190F89C22032A04D0204615
:10B0580000F021FC284612E09847F8E70021C0F8E4
:10B06800941202F0A8FC284609E0D0F8B4329B6993
:10B0780033B190F89C22032A04D19847002038BDA8
:10B088000220FCE70220FAE738B504460D460029FD
:10B0980053D11346D0F89422022A0CD0042A00D0A7
:10B0A8001AB98021204602F086FC94F8A032012BC0
:10B0B8003ED0284638BD026A416A8A421BD8C26916
:10B0C800B2FBF1F301FB13232BB9914203D8D0F85B
:10B0D80098329A421CD3D4F8B432DB681BB194F886
:10B0E8009C22032A21D08021204602F064FC2046BD
:10B0F80000F0DCFBD9E7521A026292B2194600F05E
:10B10800BAFB00231A461946204602F08BFCCCE70E
:10B118000022114600F0AFFB0021C4F898120B463C
:10B128000A46204602F07EFCBFE720469847DAE749
:10B13800002384F8A0322846BCE7D0F8B4325B6913
:10B1480033B190F89C22032A04D198470020B1E734
:10B158000220AFE70220ADE770B504464023002285
:10B16800114602F00DFC0125C4F858514026C4F8D8
:10B178006461334600228021204602F001FCA5616B
:10B18800666284F89C520023C4F894326360C4F861
:10B19800A432D4F8B8322BB1D4F8B4325B680021A9
:10B1A80020469847002070BD01740020704790F831
:10B1B8009C3280F89D32042380F89C32002070472E
:10B1C80090F89C32042B01D00020704790F89D32F3
:10B1D80080F89C32F8E708B590F89C32032B01D030
:10B1E800002008BDD0F8B432DB69002BF8D09847AE
:10B1F800F6E70346002002E00130C0B201331A78B6
:10B20800002AF9D1704708B54B88012B00D008BD3A
:10B21800C0F8A43200F03FFBF9E70B7803704B78D5
:10B2280043708B78CA7803EB022343800B794A7901
:10B2380003EB022383808B79CA7903EB0223C38053
:10B24800704710B50446802102F0B5FB0021204666
:10B2580002F0B1FB10BD30B583B005460C460023A3
:10B26800ADF806304A88130A013B062B00F2A48089
:10B27800DFE803F004182CA2A2869300D0F8B032BD
:10B288001B680DF10601007C9847BDF806201AB12D
:10B29800E388002B40F09480E388002B00F09A802C
:10B2A80003B030BD037C43B9D0F8B4329B6A0DF1CA
:10B2B8000600984702234370E7E7D0F8B432DB6A08
:10B2C8000DF10600984702234370DEE7D2B2052A43
:10B2D80052D8DFE802F003101D2A3744D0F8B03204
:10B2E8005B6823B10DF10601007C9847CDE7214644
:10B2F800FFF7A7FFD4E7D0F8B0329B6823B10DF170
:10B308000601007C9847C0E72146FFF79AFFC7E788
:10B31800D0F8B032DB6823B10DF10601007C984704
:10B32800B3E72146FFF78DFFBAE7D0F8B0321B69C3
:10B3380023B10DF10601007C9847A6E72146FFF7E7
:10B3480080FFADE7D0F8B0325B6923B10DF106019B
:10B35800007C984799E72146FFF773FFA0E7D0F8EC
:10B36800B0329B6923B10DF10601007C98478CE748
:10B378002146FFF766FF93E72146FFF762FF8FE755
:10B38800037C33B9D0F8B4325B6B0DF106009847F3
:10B398007BE72146FFF755FF82E7037C43B9D0F8E6
:10B3A800B4321B6B0DF106009847072343706CE716
:10B3B8002146FFF746FF73E72146FFF742FF6FE795
:10B3C8009A4228BF1A46ADF806200146284600F0E2
:10B3D80045FA61E7284600F05EFA61E738B50446A9
:10B3E8008B88F3B9CB88E3B94B887F2B19D803F046
:10B3F8007F0590F89C32032B0CD080F89E5229468A
:10B4080002F000FB204600F046FA35B1022384F82A
:10B418009C3209E0FFF715FF06E0012384F89C320F
:10B4280002E02046FFF70DFF38BD000038B504469E
:10B438000D468978284B197001290ED890F89C324E
:10B44800022B0ED0032B21D02946FFF7FAFE224B00
:10B4580019782046FFF79EFD02E02946FFF7F1FE26
:10B4680038BD81B14160032380F89C32FFF786FD27
:10B47800022803D0204600F00EFAF1E729462046BC
:10B48800FFF7DFFEECE700F006FAE9E789B1436869
:10B4980099421DD0D9B2FFF77DFD0F4B1978616035
:10B4A8002046FFF76BFD02280DD0204600F0F3F987
:10B4B800D6E7022380F89C324160FFF76BFD2046F7
:10B4C80000F0E9F9CCE729462046FFF7BAFEC7E7BE
:10B4D80000F0E1F9C4E700BF9914002008B5CB8853
:10B4E800012B0AD190F89C32022B09D9032B11D1D8
:10B4F8000122011D00F0B2F901E0FFF7A2FE08BD2C
:10B508005BB23BB10146002341F8083F012200F03D
:10B51800A5F9F4E7FFF795FEF1E708B590F89C3236
:10B52800013B022B12D8CB88022B0CD10123C3601C
:10B53800D0F8A4320BB10323C360022200F10C013E
:10B5480000F08CF908BDFFF77CFEFBE7FFF779FEFA
:10B55800F8E708B590F89C32013B022B09D84B88D4
:10B56800012B00D008BD0023C0F8A43200F093F9E5
:10B57800F8E7FFF766FEF5E708B50B7803F0600318
:10B58800202B05D0402B03D043B1FFF75AFE03E030
:10B59800D0F8B4329B689847002008BD4B78092B37
:10B5A8001BD8DFE803F011171A141A08051A0E0B36
:10B5B800FFF751FEF0E7FFF711FFEDE7FFF736FF62
:10B5C800EAE7FFF78BFFE7E7FFF7A7FFE4E7FFF7F7
:10B5D8001AFEE1E7FFF7BDFFDEE7FFF732FEDBE724
:10B5E80038B505460C460B7803F06003202B06D0CF
:10B5F800402B04D01BB1FFF724FE002038BD95F87E
:10B608009C32013B022B16D82379012B0ED8D5F892
:10B61800B4329B68214628469847E388002BECD132
:10B628000028EAD1284600F036F9E6E72146284600
:10B63800FFF707FEE1E721462846FFF702FEDCE7B1
:10B6480070B505468B880C7804F06004202C07D070
:10B65800DAB2402C04D05CB1FFF7F3FD002405E01A
:10B66800D5F8B4329B68284698470024204670BD18
:10B67800202C09D04E78012E33D0032E0AD0002E6C
:10B6880055D0FFF7DEFDF1E7D0F8B4329B68984754
:10B698000446EBE790F89C32022B04D0032B11D020
:10B6A800FFF7CFFDE2E70AB1802A03D12846FFF76A
:10B6B800C8FDDBE7114602F07EF98021284602F03A
:10B6C8007AF9D3E74B8823B91AB1802A01D0CB88FD
:10B6D8001BB1284600F0DFF8C8E7114602F06BF905
:10B6E800F7E790F89C32022B04D0032B11D0FFF718
:10B6F800A8FDBBE70AB1802A03D12846FFF7A1FDC0
:10B70800B4E7114602F057F98021284602F053F9B0
:10B71800ACE74B88002BA9D112F07F0F03D1284644
:10B7280000F0B9F8A2E7114602F04DF9F7E790F8F2
:10B738009C02022806D0032829D02846FFF781FD5D
:10B74800344693E70AB1802A13D113F0800F15D13C
:10B7580002F07F0202EB8202910001F5A8712944F0
:10B76800043100230B600222284600F077F83446A3
:10B778007CE72846FFF765FD344677E702F07F024D
:10B7880002EB82029100103129440431E9E75BB2EF
:10B79800002B1FDB02F00F0000EB800005EB8000A0
:10B7A800D0F8580120B3002B27DB02F07F0303EB0E
:10B7B80083039C0004F5A8742C4404340AB1802A3D
:10B7C80024D10023236002222146284600F046F8AF
:10B7D80034464BE702F00F0000EB800005EB8000D9
:10B7E80080690028DFD12846FFF72BFD34463DE766
:10B7F8002846FFF726FD344638E702F07F0303EBBF
:10B8080083039C0010342C440434D7E7114628469F
:10B8180002F0E1F810B101232360D4E7002323608C
:10B82800D1E7D0B170B50D4616460446FFF7E1FCE6
:10B83800431C5B009BB233802B7003236B70022385
:10B8480007E001345A1CD2B2E8540233DBB20021BB
:10B85800A95420780028F4D170BD704708B5134664
:10B868000222C0F89422C36103620A46002102F052
:10B87800D1F8002008BD08B513460A46002102F099
:10B88800C9F8002008BD08B513460A46002102F091
:10B89800C9F8002008BD08B50423C0F89432002375
:10B8A8001A46194602F0B6F8002008BD08B5052367
:10B8B800C0F8943200231A46194602F0B3F8002063
:10B8C80008BD000008B5044B03EB800252685268BB
:10B8D8000344187A904708BDBC14002008B5084BEB
:10B8E8001B5C53B9064B01221A5403EB80025268C1
:10B8F80012680344187A904708BD0020FCE700BF8F
:10B90800BC14002038B5044C04EB80056D68AD68A4
:10B918000444207AA84738BDBC14002038B5044C2C
:10B9280004EB80056D68ED680444207AA84738BDAB
:10B93800BC14002010B5044B03EB80046468246930
:10B948000344187AA04710BDBC14002008B5074B63
:10B9580001221A70FEF73AFD20B9044A137803F061
:10B96800FE031370014B187808BD00BFC800002003
:10B9780008B5074B01221A70FEF70EFD20B9044ADC
:10B98800137803F0FE031370014B187808BD00BF4D
:10B99800C800002010B5084611461A46094BFEF7A4
:10B9A800DBFC10B10123184610BD074CFEF7F4FC70
:10B9B80003460028F7D0631E0CB11C46F6E70123A6
:10B9C800F1E700BF00E1F505A086010010B50846C3
:10B9D80011461A46094BFEF7CFFC10B10123184651
:10B9E80010BD074CFEF7D8FC03460028F7D0631EAD
:10B9F8000CB11C46F6E70123F1E700BF00E1F505AD
:10BA0800A086010030B589B0124B187810F00104F7
:10BA18001AD1154603291BD8DFE801F002040A10E1
:10BA28000C4612E06846FEF7C1FC069B2B600CE052
:10BA38006846FEF7BBFC079B2B8006E06846FEF7CE
:10BA4800B5FC079B2B6000E00324204609B030BDFD
:10BA58000424FAE7C800002004E011F8012B00F8DC
:10BA6800012B1A46531E002AF7D1704702E000F84E
:10BA7800011B1A46531E002AF9D1704710B4034619
:10BA880000201446013A34B113F8010B11F801CB28
:10BA9800B0EB0C00F5D010BC7047034600E0013352
:10BAA800187808B18842FAD17047000030B40025F0
:10BAB8002B4601E001250133012B1ED803EB43027D
:10BAC8001C4C54F82220002AF4D0D0F80042A2429C
:10BAD800F1D103EB4304174A02EB84025468D0F80F
:10BAE80008229442E7D103EB4304124A02EB840292
:10BAF8001489B0F806229442DDD1022B0CD0B1B9DA
:10BB080003EB43030B4A02EB83035B89B3F5807FA6
:10BB18000BD0002030BC70472DB9022901D012206B
:10BB2800F8E70020F6E70020F4E71020F2E71020FD
:10BB3800F0E700BF9C140020002000E0013001283D
:10BB480006D800EB40029300034AD358002BF5D1E6
:10BB5800023818BF012070479C14002010B500233C
:10BB680000E00133012B1CD803EB43022D4C54F8A1
:10BB78002240D0F800229442F3D103EB4304294A2F
:10BB880002EB84025468D0F808229442E9D103EB0E
:10BB98004304244A02EB84021489B0F80622944232
:10BBA800DFD1022B0AD041B303EB43011D4A02EB5C
:10BBB800810252899ABB4FF4807226E00023012B40
:10BBC80007D803EB4302174C54F822200AB101337B
:10BBD800F5E7022B21D0134C03EB430C04EB8C024A
:10BBE800D0F800E244F82CE0D0F808425460B0F8ED
:10BBF8000602108100205081D5E703EB4301094A72
:10BC080002EB81025289013292B203EB43000549EB
:10BC180001EB80014A81581C10BD0020FCE7002080
:10BC2800FAE700BF9C140020013801281BD800EB5C
:10BC380040020F4B03EB82035B89B3F5807F03D08F
:10BC480053B1013B9BB200E0002300EB4001084ADE
:10BC580002EB8102538143B900EB400083000020CE
:10BC6800034AD0507047022070470020704700BF39
:10BC78009C140020002302E010BC70470133012B04
:10BC880017D803EB43020B4951F822208242F5D121
:10BC980010B403EB4302920000248C500133012BB3
:10BCA800EAD803EB4302034951F822208242F5D136
:10BCB800EFE770479C140020D0F824320433490A77
:10BCC800D0F8002292F80222B1FBF2F101E0091A41
:10BCD8000833186818B18142F9D258680844704787
:10BCE8000246C87E8B7E43EA002092F80032032B7E
:10BCF80000D070474A7D0B7D43EA022340EA0340A7
:10BD0800F7E78176C1F30723C376C1F307430375C9
:10BD1800090E4175704700002DE9F84F89460C68F7
:10BD280000E0013423782F2BFBD05C2BF9D0D0F81E
:10BD380018A20B2220215046FFF798FE0026334612
:10BD48004FF00808374619E0BF00FFB246464FF0EB
:10BD58000B0812E015F0800F25D129463148FFF76E
:10BD68009CFE00285AD1A5F14103DBB2192B20D83B
:10BD780047F002070AF8065001365B4603F1010B4B
:10BD8800E55C202D1FD92F2D1DD05C2D1BD02E2D0D
:10BD980001D0B045DED8B8F1080F3DD12E2DD3D053
:10BDA8000620BDE8F88F47F00307803D1E4B5D5D18
:10BDB800D3E7A5F16103DBB2192BDBD847F0010704
:10BDC800203DEDB2D6E75C44C9F80040202D14D8D8
:10BDD80004232EB39AF80020E52A10D0B8F1080FF2
:10BDE80011D007F00302012A10D007F00C07042F26
:10BDF8000FD08AF80B300020D3E70023E9E70522AB
:10BE08008AF80020EAE7BF00FFB2EAE743F0100330
:10BE1800EBE743F00803ECE70620C2E70620C0E79B
:10BE28000620BEE7DCAB010844E1010801460068D2
:10BE380038B102461378202B06D93A2B04D00132A8
:10BE4800F8E74FF0FF3070473A2B01D000207047D9
:10BE580010B4034613F8010B3038092808D89A4261
:10BE680002D04FF0FF3005E030B901320A6001E03E
:10BE78004FF0FF3010BC70474FF0FF30FAE7F8B5CD
:10BE880090F804520DB92846F8BD0446D0F82C7233
:10BE980001233A46014690F80102FFF73FFD0546A7
:10BEA800D0B9002384F80432D4F82032FB1AD4F82D
:10BEB80018229342E7D294F803620AE0D4F81832C1
:10BEC8001F4401233A46214694F80102FFF726FD54
:10BED800013E012EF2D8D6E70125D4E770B5D0F897
:10BEE8002C328B4202D10026304670BD04460D46E6
:10BEF800FFF7C5FF06460028F6D101232A4621464A
:10BF080094F80102FFF7FEFC10B101264FF0FF354F
:10BF1800C4F82C52E8E7000010B50446002380F866
:10BF280004324FF0FF33C0F82C32FFF7D7FF98BB2D
:10BF3800024694F8FF1194F8FE3143EA01231BB23C
:10BF480017498B422AD194F8391094F838301B04D9
:10BF580043EA016394F8371043EA012394F8361052
:10BF68000B4323F07F430F498B4213D094F85510AD
:10BF780094F854301B0443EA016394F8531043EADD
:10BF8800012394F852100B4323F07F4305498B4259
:10BF980000D00122104610BD0322FBE70222F9E778
:10BFA80055AAFFFF46415400B0B108B5D0F8003299
:10BFB80043B193F8001229B1B3F80612B0F804227D
:10BFC800914201D0092008BD93F80102FFF77AFCDD
:10BFD80010F00100F7D0F5E7092070472DE9F0438C
:10BFE80085B005461746002303600846FFF71EFF85
:10BFF800061EC0F29E819F4B53F82640002C00F08D
:10C008009D812C6094F800327BB194F80102FFF70F
:10C0180059FC10F0010508D1002F00F08B8110F0B9
:10C02800040F00F087810A2584E1002384F8003298
:10C03800F0B284F80102FFF751FC10F0010F40F054
:10C048007F811FB110F0040F40F07C810021204651
:10C05800FFF762FF0546012800F095800027032DB1
:10C0680000F07281002D40F07181227BE37A43EA6F
:10C0780002231BB2B3F5007F40F06A81E27DA37D05
:10C0880053EA02230DD194F8272094F826301B0494
:10C0980043EA026394F8252043EA022394F8242013
:10C0A8001343C4F81832217C84F803124A1ED2B212
:10C0B800012A00F24F8103FB01F1607B84F8020240
:10C0C800002800F04981421E104240F04781A67CBA
:10C0D800627C42EA06221646A4F8082212F00F0FE4
:10C0E80040F03E8194F814C0E27C52EA0C220ED152
:10C0F80094F823C094F82220120442EA0C6294F8BF
:10C1080021C042EA0C2294F820C042EA0C0294F8BA
:10C118000FE094F80EC05CEA0E2C00F023810CEBC3
:10C12800010909EB16194A45C0F01E81A2EB090264
:10C13800B2FBF0FE8242C0F0198140F6F5729645D6
:10C148003AD94FF6F572964577D84FF0020835E0A0
:10C15800002304AA02EB810242F8103C01310329B2
:10C1680013D80B0103F5DF7323441A79002AEFD0A3
:10C17800D87A9A7A120442EA0062587A42EA00228D
:10C188001B7A1343E5E70021E9E700260BE039466F
:10C198002046FFF7C1FE054600283FF460AF013690
:10C1A800032E3FF65CAF04AB03EB860353F8107C19
:10C1B800002FECD10225F2E74FF001080EF1020E34
:10C1C800C4F814E2C4F81C720CEB0702C4F820226D
:10C1D80007EB0900C4F82802B8F1030F30D0002E8D
:10C1E80000F0C8800A44C4F82422B8F1020F3DD0F8
:10C1F8000EEB4E010EF0010202EB510202F2FF12A9
:10C20800B3EB522FC0F0B8804FF0FF33C4F81032B0
:10C21800C4F80C32802384F80532B8F1030F2DD00E
:10C2280084F80082144A138801339BB21380A4F85F
:10C2380006322046FFF71EFD7CE04FF00308BDE7FD
:10C24800002E40F0958094F82F1094F82E201204B8
:10C2580042EA016294F82D1042EA012294F82C1067
:10C268000A43C4F824224FEA8E02C7E74FEA4E0277
:10C27800C4E700BFB8140020B414002094F831209B
:10C2880094F8303043EA02231BB2012BC8D1791C41
:10C298002046FFF723FE0028C2D1002384F8053288
:10C2A80094F8FF2194F8FE3143EA02231BB2334A83
:10C2B8009342B5D1E278A3781B0443EA026362781B
:10C2C80043EA0223227813432D4A9342A8D194F8D3
:10C2D800E72194F8E6311B0443EA026394F8E52168
:10C2E80043EA022394F8E4211343264A934297D160
:10C2F80094F8EB2194F8EA311B0443EA026394F8BA
:10C30800E92143EA022394F8E8211343C4F81032E0
:10C3180094F8EF2194F8EE311B0443EA026394F891
:10C32800ED2143EA022394F8EC211343C4F80C32BC
:10C3380076E70B25284605B0BDE8F0830C25F9E71C
:10C348000325F7E70A25F5E70125F3E70D25F1E7CA
:10C358000D25EFE70D25EDE70D25EBE70D25E9E7C1
:10C368000D25E7E70D25E5E70D25E3E70D25E1E7D1
:10C378000D25DFE70D25DDE70D25DBE755AAFFFFD6
:10C38800525261417272416138B50446FFF777FD38
:10C39800054658B994F80032032B09D000221146FB
:10C3A80094F80102FFF7C6FA00B10125284638BD06
:10C3B80094F80532012BF1D14FF400720021204688
:10C3C800FFF754FB552384F8FE31AA2384F8FF3184
:10C3D8005223237063706123A3704122E27072219B
:10C3E80084F8E41184F8E51184F8E62184F8E7314B
:10C3F800D4F8103284F8E831C3F3072284F8E9212D
:10C40800C3F3074284F8EA211B0E84F8EB31D4F811
:10C418000C3284F8EC31C3F3072284F8ED21C3F31E
:10C42800074284F8EE211B0E84F8EF31D4F81C2261
:10C438000132C4F82C220123214694F80102FFF7A7
:10C448006DFA002384F80532A8E70239D0F81432CF
:10C45800023B8B4206D990F80232D0F8280201FB41
:10C46800030070470020704701295CD9F8B50546DC
:10C478000C46D0F814328B4257D990F80032022B70
:10C4880029D0032B37D0012B51D101EB5106D0F81D
:10C49800201201EB5621FFF721FD10B14FF0FF30BC
:10C4A80044E0771CC6F30806AE5DD5F8201201EB10
:10C4B80057212846FFF712FD00283AD1C7F308078D
:10C4C800EB5D46EA032014F0010F01D000092DE0CE
:10C4D800C0F30B002AE0D0F8201201EB1421FFF77B
:10C4E800FDFC48BB640004F4FF742B195B78285DDD
:10C4F80040EA03201AE0D0F8201201EBD411FFF72C
:10C50800EDFCE0B9A40004F4FE742B19DA789878ED
:10C51800000440EA02605B7840EA03202B5D184380
:10C5280020F0704002E0012070470120F8BD012092
:10C53800FCE74FF0FF30F9E74FF0FF30F6E74FF038
:10C54800FF30F3E7F8B50746A0F80612D0F808421E
:10C55800012C44D00E46D0F80032D3F81422A2425F
:10C568003FD9F4B993F80022032A17D0CCB9B3F80D
:10C578000822B24237D9D3F82402C7F80C42D0B304
:10C5880000EB1610C7F81002D7F8003206F00F01BA
:10C5980003EB4113C7F814320020F8BDD3F8244246
:10C5A800E4E793F802522D01AE4212D32146D7F8A0
:10C5B8000002FFF759FF0446B0F1FF3F15D00128EC
:10C5C80015D9D7F80032D3F81432834211D9761B23
:10C5D800EAE72146D7F80002FFF737FFCDE7022048
:10C5E800DBE70220D9E70220D7E70120D5E70220C0
:10C5F800D3E70220D1E70220CFE701297CD92DE932
:10C60800F04105460C461646D0F814328B4275D9CF
:10C6180090F80032022B3CD0032B4DD0012B70D167
:10C6280001EB5107D0F8201201EB5721FFF756FC18
:10C63800002864D107F10108C7F3080714F00104C2
:10C648001DD0EB5D03F00F0343EA0613DBB2EB5595
:10C65800012385F80432D5F8201201EB5821284629
:10C66800FFF73CFC00284AD1C8F308084CB1C6F3D0
:10C67800071305F80830012385F804323FE0F3B2C8
:10C68800E5E715F80830C6F3032223F00F03134338
:10C69800EFE7D0F8201201EB1421FFF71FFC70BB65
:10C6A800640004F4FF742B192E55C6F307225A7040
:10C6B800012385F8043222E0D0F8201201EBD411CE
:10C6C800FFF70CFCD8B9A40004F4FE742919CA7841
:10C6D8008B781B0443EA026303F0704333432E55FF
:10C6E800C6F307224A70C6F307428A701B0ECB7046
:10C6F800012385F8043202E0022070470220BDE8D9
:10C70800F0810220FBE7F8B505460F4641B9D0F89D
:10C718000C629EB1D0F81432B34210D801260EE054
:10C72800FFF7A2FE034601284BD9B0F1FF3F4DD0D9
:10C73800D5F81422824249D83E4600E00126344604
:10C748000CE021462846FFF78FFE034678B1B0F18A
:10C75800FF3F3BD0012839D0B44236D00134D5F858
:10C768001432A342EDD8012E2DD90224E9E76FF047
:10C77800704221462846FFF740FF0346D0B997B9D3
:10C78800C3B9C5F80C42D5F81032B3F1FF3F1FD03A
:10C79800013BC5F8103295F8053243F0010385F8DE
:10C7A8000532234612E0224639462846FFF725FF80
:10C7B8000346E5E7012B01D0012307E04FF0FF33E3
:10C7C80004E0012302E0002300E000231846F8BD3E
:10C7D8002346FBE72DE9F843B0F806526B1C9AB2E2
:10C7E800002A00F0838004460F46D0F81022002A61
:10C7F8007ED013F00F060BD10132C0F81022D0F80A
:10C808000C1289B9D0F80022B2F808229A4271D9DC
:10C818000135A4F80652D4F8003203EB4613C4F8E5
:10C8280014320020BDE8F883D0F8000290F8022204
:10C83800013A12EA1318EBD1FFF716FE81460128D8
:10C848005AD9B0F1FF3F59D0D4F80002D0F81432C9
:10C858004B4541D8002F53D0D4F80C12FFF753FFA3
:10C86800814600284ED001284ED0B0F1FF3F4DD070
:10C87800D4F80002FFF703FB08B10120D2E74FF418
:10C8880000720021D4F80002FFF7F0F8D4F8007223
:10C8980049463846FFF7D9FDC7F82C02D4F80032CC
:10C8A80093F80222424511D9012283F80422D4F8D0
:10C8B8000002FFF7E4FA58BBD4F80022D2F82C3271
:10C8C8000133C2F82C3208F10108E7E7D3F82C222B
:10C8D800A2EB0802C3F82C22C4F80C924946D4F8FB
:10C8E8000002FFF7B2FDC4F8100291E7042099E7AF
:10C8F800042097E7042095E7022093E7012091E7B9
:10C9080004208FE707208DE702208BE7012089E7C5
:10C91800012087E738B504460021FFF713FE0546D6
:10C9280040B1284638BD00212046FFF753FF054691
:10C938000028F6D1D4F81012D4F80002FFF7CEFA86
:10C9480005460028EDD1D4F8140203785BB1C37A08
:10C9580013F0080FE7D10B22D4F81812FFF78EF85E
:10C968000028E0D1DDE70425DBE710B582B00446F6
:10C9780001910B782F2B01D05C2B01D10131019152
:10C988000023C4F80832019B1B781F2B1DD901A96D
:10C998002046FFF7C1F90346F8B92046FFF7BAFF6A
:10C9A800D4F81832DA7A0346D0B912F0040F14D149
:10C9B800D4F81412CB7A13F0100F18D0D4F8000260
:10C9C800FFF78EF9C4F80802E1E700212046FFF7D7
:10C9D800B9FD03460022C4F81422184602B010BD5F
:10C9E8000428FAD112F0040FF7D10523F5E705233F
:10C9F800F3E770B504460E460021FFF7A3FD024693
:10CA0800D8B9002508E00135B54216D001212046E5
:10CA1800FFF7E0FE024680B9D4F81012D4F80002FD
:10CA2800FFF75CFA024640B9D4F814321B78E52BBC
:10CA3800E9D0002BE7D00025E8E7042A01D010460A
:10CA480070BD0722FBE738B504460121FFF7D1FF87
:10CA5800054608B1284638BDD4F81012D4F80002AB
:10CA6800FFF73CFA05460028F4D120220021D4F82B
:10CA78001402FEF7FBFF0B22D4F81812D4F81402A4
:10CA8800FEF7EAFFD4F80032012283F80422E1E736
:10CA9800F8B501292DD904460D46D0F814328B4239
:10CAA8002AD9002700E03546D4F81432AB4221D900
:10CAB80029462046FFF7D8FC0646D8B101281DD0E4
:10CAC800B0F1FF3F1CD0002229462046FFF795FD14
:10CAD800074678B9D4F81032B3F1FF3FE3D00133F9
:10CAE800C4F8103294F8053243F0010384F8053293
:10CAF800D9E702273846F8BD0227FBE70227F9E7FE
:10CB08000127F7E770B584B00190009116460391AC
:10CB180003A8FFF78BF9041E1DDB114B53F82450B3
:10CB28002DB12846FFF7A6F8002385F80032019BAF
:10CB380013B1002283F80022094A42F8243063B175
:10CB4800012E02D0002004B070BD0022694601A861
:10CB5800FFF744FAF7E70B20F5E70020F3E700BFFB
:10CB6800B81400202DE9F043ADF50F7D01910028A0
:10CB780000F0E580144606460023C0F8003202F0B3
:10CB88001F0802F01E073A4601A986A8FFF726FAF1
:10CB9800054620B128460DF50F7DBDE8F08303ABAF
:10CBA8008C93019906A8FFF7E0FEDDF82C92054664
:10CBB80048B9B9F1000F5AD0391E18BF012106A88B
:10CBC800FEF774FF054614F01C0F00F0A480002D3A
:10CBD80059D0042D4DD048F00808DDF82C9215B92D
:10CBE80018F0080F5BD1002DD4D118F0080F01D030
:10CBF80048F02008869BD3F82C32C6F81C32C6F8B9
:10CC08002092B8F1010F94BF0021012106A8FEF778
:10CC1800A5FFC6F82802002800F0938086F806824F
:10CC2800002486F80742869F49463846FFF758F899
:10CC3800C6F8100299F81F2099F81E301B0443EA21
:10CC4800026399F81D2043EA022399F81C20134334
:10CC5800C6F80C32C6F80842C6F81842C6F824428C
:10CC6800C6F80072B7F80632A6F8043292E706252D
:10CC7800A9E7FEF761FF08B91225ACE706A8FFF798
:10CC8800E2FE0546A7E799F80B3013F0110F04D11F
:10CC980014F0040FA3D00825A1E707259FE7FDF7A7
:10CCA80059FB89F80E00C0F3072389F80F30C0F349
:10CCB800074389F81030000E89F81100002489F81C
:10CCC8000B4089F81C4089F81D4089F81E4089F8F6
:10CCD8001F4049468698FFF703F80746214648460D
:10CCE800FFF70FF88698012380F80432002F3FF4ED
:10CCF8007AAFD0F82C423946FFF7CAFE054600281D
:10CD08007FF471AF8698013FC0F80C722146FFF797
:10CD1800E5F8054667E7002D7FF465AF99F80B3015
:10CD280013F0100F09D114F0020F3FF45CAF13F0A9
:10CD3800010F3FF458AF072555E7042553E70925A8
:10CD480028E7022526E72DE9F04F83B004460F4671
:10CD5800164698460023C8F80030FFF725F90190D9
:10CD6800002840F0D18094F807320193002B40F05E
:10CD7800CB8094F8063213F0010F00F0D780D4F876
:10CD88000C52D4F80832ED1AB54276D3354674E021
:10CD9800D4F824321BB12046FEF78EFF83E0D4F886
:10CDA8001412FFF761FB7EE04FF0020A84F807A235
:10CDB800CDF804A0A8E04FF0010A84F807A2CDF846
:10CDC80004A0A1E04FF0020A84F807A2CDF804A05D
:10CDD8009AE094F8063213F0400F05D0D4F8180200
:10CDE800A0EB0900504502D34FEA4A2639E04FF438
:10CDF8000072214607EB4020FEF72EFEF4E7D4F838
:10CE080018224A451DD094F8063213F0400F0DD071
:10CE1800012321469BF80102FEF780FD002877D107
:10CE280094F8063223F0400384F80632D4F800025E
:10CE380001234A46214690F80102FEF763FD0028C7
:10CE48006DD1C4F81892D4F80812C1F30801C1F5DD
:10CE58000076B54200D22E46324621443846FEF7C7
:10CE6800FBFD3744D4F808323344C4F80832D8F804
:10CE780000303344C8F80030AD1B002D44D0D4F83E
:10CE88000812C1F30803002BDDD1D4F8000290F892
:10CE98000262013EF6B216EA51260CD100297FF44F
:10CEA80077AFD4F8100201287FF67EAFB0F1FF3FCC
:10CEB80081D0C4F81402D4F800B2D4F81412584639
:10CEC800FFF7C3FA814600283FF47CAFB1444FEA2C
:10CED800552AB5F5007F92D306EB0A039BF8022288
:10CEE800934201D9A2EB060A53464A4639469BF8B3
:10CEF8000102FEF707FD00283FF46BAF4FF0010A6F
:10CF080084F807A2CDF804A0019803B0BDE8F08F1B
:10CF18004FF0010A84F807A2CDF804A0F4E74FF017
:10CF2800010A84F807A2CDF804A0EDE707230193CE
:10CF3800EAE72DE9F04F83B004460F4615469846B8
:10CF48000023C8F80030FFF72FF80190002853D1CC
:10CF580094F807320193002B4ED194F8063213F05F
:10CF6800020F00F00081D4F80832EB42C0F0BF8015
:10CF78000025BCE0D4F82432002B41D02046FEF72F
:10CF88009BFE0346002B00F0DF80012B3ED0B3F15F
:10CF9800FF3F42D0C4F81432D4F810220AB9C4F8BA
:10CFA800103294F8063213F0400F3DD1D4F800B295
:10CFB800D4F814125846FFF748FA814600284CD096
:10CFC800B1444FEA552AB5F5007F64D306EB0A034E
:10CFD8009BF80222934201D9A2EB060A53464A461D
:10CFE80039469BF80102FEF799FCE8B34FF0010AB5
:10CFF80084F807A2CDF804A0019803B0BDE8F08F2B
:10D00800D4F81412FFF77FFB0346BBE74FF0020A80
:10D0180084F807A2CDF804A0EEE74FF0010A84F8DF
:10D0280007A2CDF804A0E7E7D4F800020123D4F85A
:10D038001822214690F80102FEF770FC30B994F8E6
:10D04800063223F0400384F80632AFE74FF0010AB6
:10D0580084F807A2CDF804A0CEE74FF0020A84F8BE
:10D0680007A2CDF804A0C7E7D4F81812A1EB09016C
:10D07800514502D34FEA4A262DE04FF4007207EBE0
:10D0880041212046FEF7E8FC94F8063223F04003DD
:10D0980084F80632EEE7D4F818324B4505D0D4F8B8
:10D0A8000822D4F80C329A423ED3C4F81892D4F825
:10D0B8000802C0F30800C0F50076B54200D22E463B
:10D0C800324639462044FEF7C7FC94F8063243F04E
:10D0D800400384F806323744D4F808323344C4F89D
:10D0E8000832D8F800303344C8F80030AD1B5DB3BF
:10D0F800D4F80812C1F30803002BD8D1D4F80002E1
:10D1080090F80262013EF6B216EA51267FF449AF62
:10D1180000297FF42FAFD4F81032002B7FF435AFFD
:10D12800FFF7F1FA03462DE701234A4621469BF80B
:10D138000102FEF7E7FB0028B7D04FF0010A84F898
:10D1480007A2CDF804A057E7D4F80832D4F80C2287
:10D15800934201D9C4F80C3294F8063243F0200304
:10D1680084F8063248E70723019345E738B50446B3
:10D17800FEF71AFF00BB94F8063213F0200F1BD0FD
:10D1880013F0400F11D0D4F800020123D4F818226C
:10D19800214690F80102FEF7C1FB002843D194F81C
:10D1A800063223F0400384F80632D4F81C12D4F86F
:10D1B8000002FEF793FE00B138BDD4F82052EB7A96
:10D1C80043F02003EB7294F80C322B77B4F80C324E
:10D1D8001B0A6B7794F80E32AB7794F80F32EB7723
:10D1E800D4F810122846FEF78CFDFDF7B3F8A875A1
:10D1F800C0F30723EB75C0F307432B76000E687660
:10D208000023AB74EB7494F8063223F0200384F8FF
:10D218000632D4F80032012283F80422D4F800023E
:10D22800FFF7B2F8C8E70120C6E710B50446FFF7D4
:10D238009DFF00B110BD2046FEF7B6FE0028F9D1CB
:10D24800D4F82802FEF7F0FC0028F3D1C4F8000255
:10D25800F0E72DE9F84F04460D46FEF7A5FE064611
:10D26800002840F0798194F80732002B40F0738150
:10D27800D4F82432002B00F09D80B5F1FF3F4BD04D
:10D28800D4F80C72AF4200D32F46C4F80872002FAE
:10D2980000F0628107F1FF3841462046FEF70CFD99
:10D2A8000146C4F81402D4F800522846FFF7CDF816
:10D2B800002873D095F80212013901EA582101EBD0
:10D2C8000008C7F30807002F00F04681D4F8182299
:10D2D800424500F0418194F8063213F0400F0DD01A
:10D2E8000123214695F80102FEF718FB002859D1C1
:10D2F80094F8063223F0400384F80632D4F800028A
:10D3080001234246214690F80102FEF7FBFA002865
:10D318004CD1C4F818821FE1984658F804BBD4F8D9
:10D3280010A2BAF1000F2CD04FF0020909F102093E
:10D338005146002701370D46D4F80002FFF794F84C
:10D348000146012815D9B0F1FF3F16D001358542B5
:10D35800F0D0CB4505D3434643F8087BC8F804A072
:10D368009846D4F80032D3F814328B420BD98A4647
:10D37800DCE7022684F80762EEE0012684F80762FB
:10D38800EAE04FF00209D4F82432C3F80090D945F6
:10D3980000F2E5800023C8F80030DDE0022684F8BA
:10D3A8000762D9E0012684F80762D5E0012684F8EF
:10D3B8000762D1E0D4F80C32AB4205D294F80622C9
:10D3C80012F0020F00D11D46D4F808320022C4F82A
:10D3D80008220DB3D4F8000290F802824FEA4828D8
:10D3E80083B16A1EB2FBF8F2013BB3FBF8F18A4243
:10D3F80008D3C8F100021340C4F80832EF1AD4F871
:10D40800145207E0D4F81032002B3FD0C4F814327D
:10D418002F461D46002D67D1D4F80832C3F3080300
:10D428002BB3D4F81822AA4221D094F8063213F06C
:10D43800400F0FD0D4F800020123214690F80102D2
:10D44800FEF76CFA00287ED194F8063223F04003E8
:10D4580084F80632D4F8000201232A46214690F8BF
:10D468000102FEF74FFA002871D1C4F81852D4F817
:10D478000832D4F80C2293426ED9C4F80C3294F8CE
:10D48800063243F0200384F8063265E00021FFF7F6
:10D498003AF90346012805D0B0F1FF3F06D0C4F899
:10D4A8001002B3E7022684F8076255E0012684F8E3
:10D4B800076251E02946D4F80002FEF7D5FF054679
:10D4C800B5F1FF3F31D0012D33D9D4F80032D3F86C
:10D4D8001432AB422DD9C4F81452D4F8083243445C
:10D4E800C4F80832A7EB080747450DD994F8063267
:10D4F80013F0020FDED02946D4F80002FFF703F933
:10D5080005460028DCD14746D4F808323B44C4F825
:10D518000832C7F30803A3B12946D4F80002FEF77E
:10D5280094FF50B100EB572576E7012684F807628F
:10D5380012E0022684F807620EE0022684F80762E9
:10D548000AE01D4668E7012684F8076204E0012620
:10D5580084F8076200E01E463046BDE8F88F1126C1
:10D56800FAE70000134B5B7ADBB2012B01D90120EB
:10D57800704710B404460F4B93F809C05FFA8CFC4F
:10D58800002003F80C0093F809C003EB8C0CCCF8CE
:10D5980004405C7A1C4422725A7A541CE4B25C72CD
:10D5A80030320A703A234B702F238B70C87010BC2E
:10D5B800704700BFBC14002008B50022FFF7D2FF57
:10D5C80008BD000008B500220F491048FDF7B3FC5C
:10D5D80070B90F490D48FDF7C5FC60B90D490B48F6
:10D5E800FDF73CF850B90948FDF7C3FC48B908BD38
:10D5F800F4F712F9EDE7F4F70FF9EFE7F4F70CF9A0
:10D60800F1E7F4F709F9F2E700010020C814002057
:10D61800900000201C01002012230B800048704756
:10D62800EC00002004230B8000487047E80000202D
:10D63800002393421ED200B510E00CF1370C01F81C
:10D6480013C000014FEA430C0CF1010C4FF0000E1F
:10D6580001F80CE00133DBB2934209D24FEA107CA7
:10D66800B0F1204FE9D20CF1300C01F813C0E8E713
:10D678005DF804FB7047000038B50B4BD3F8E8079A
:10D68800D3F8EC47D3F8F037C01800D138BD074DB0
:10D6980008222946FFF7CCFF042205F11001204695
:10D6A800FFF7C6FFF2E700BF00F0FF1FCE00002023
:10D6B80008B51A230B80FFF7DFFF014808BD00BF3C
:10D6C800CC00002008B50A4628B905490548FEF7E8
:10D6D800A8F8034808BD02490248FEF7A2F8F8E78F
:10D6E8008C170020ECAB010810B50A46034C214604
:10D6F8000348FEF796F8204610BD00BF8C1700209F
:10D7080000AC010808B50A4628B905490548FEF7DE
:10D7180088F8034808BD02490248FEF782F8F8E78E
:10D728008C17002014AC010808B50A4628B9054929
:10D738000548FEF776F8034808BD02490248FEF797
:10D7480070F8F8E78C17002020AC0108034B586DDF
:10D7580008609B6D13800020704700BFF808002008
:10D7680000207047002070470020704770B50846B9
:10D7780015461E460B4B32462946FCF7FDFD38B9C7
:10D78800094CFCF709FE18B1601E44B10446F8E7DD
:10D7980032462946054801F0A5FE002070BD02204A
:10D7A800FCE700BF00E1F505A086010030AC0108E8
:10D7B80070B5084615461E460B4B32462946FCF7FF
:10D7C800CBFD38B9094CFCF7E7FD18B1601E44B130
:10D7D8000446F8E732462946054801F083FE002052
:10D7E80070BD0220FCE700BF00E1F505A08601003E
:10D7F8005CAC010808B5044801F0D4FEFCF7E6FD6E
:10D8080000B908BD0220FCE788AC0108022805D849
:10D81800DFE800F00504020001207047022070478D
:10D8280002680E4B9A4200D0704700B583B003F5EA
:10D83800DA33DA6942F40002DA61DB6903F40003DF
:10D848000193019B002203211420F7F71FF91420EC
:10D85800F7F72CF903B05DF804FB00BF005C00404B
:10D8680008B500F52C71D0F8EC02FDF79AFB08BD5D
:10D8780008B501EB810300EBC303D3F87C21D0F892
:10D88800EC02FDF7BBFB08BD08B501EB810300EB1B
:10D89800C303DA6BD0F8EC02FDF7F6FB08BD08B558
:10D8A800D0F8EC02FDF797FC08BD10B50446836874
:10D8B800022B09D10121D4F8EC02FDF775FCD4F84C
:10D8C800EC02FDF749FC10BDF3F7A6FFF2E70000F4
:10D8D80010B50446D0F8EC02FDF769FCA36923B142
:10D8E800024A136943F00603136110BD00ED00E01E
:10D8F80008B5D0F8EC02FDF763FC08BD10B5044686
:10D908001948C0F8EC42C4F8C002184B0360082359
:10D9180043600223836000238361C3610362F7F7D6
:10D9280097FDE8B9182300221146D4F8C002F8F789
:10D9380017FD582300228021D4F8C002F8F710FD03
:10D94800982300228121D4F8C002F8F709FDD823D2
:10D9580000220121D4F8C002F8F702FD002010BD12
:10D96800F3F75AFFDEE700BFFC1B0020005C004015
:10D9780008B5D0F8C002F7F7F3FDFFF747FF08BD79
:10D9880008B594461A466346D0F8C002F8F79EFBDD
:10D99800FFF73CFF08BD08B5D0F8C002F8F7D4FB84
:10D9A800FFF734FF08BD08B5D0F8C002F8F7BDFC92
:10D9B800FFF72CFF08BD08B5D0F8C002F8F73EFC09
:10D9C800FFF724FF08BD08B5D0F8C002F8F772FCCD
:10D9D800FFF71CFF08BDD0F8C03211F0800F08D146
:10D9E80001F07F0101EB810103EBC10393F86A01A8
:10D9F800704701F07F01013101EB810103EBC103A5
:10DA08009878704708B5D0F8C002F8F773FAFFF7AE
:10DA1800FDFE08BD08B5D0F8C002F8F7EDFBFFF72A
:10DA2800F5FE08BD08B5D0F8C002F8F7BFFBFFF750
:10DA3800EDFE08BD08B5D0F8C002F8F7D4FB08BD64
:10DA4800004870478C19002070477047024B014608
:10DA5800186800F00BB800BFC8060020024B01464A
:10DA6800186802F095BB00BFC80600202DE9F04FEA
:10DA780001F10B05162D064683B024D8102900F2B3
:10DA8800AD8000F0A7FA102518234FF0020CB84F0C
:10DA98003B445C68A3F10802944200F01D813046C3
:10DAA8006368E268A16823F00303CA6023449160B5
:10DAB8005A68083442F001025A6000F091FA204690
:10DAC80003B0BDE8F08F35F0070500F18780A94263
:10DAD80000F2848000F07EFAB5F5FC7FC0F06F811B
:10DAE8006B0A7FD0042B00F21E81AB0903F1390CBD
:10DAF80003F1380E4FEACC009D4F3844446808388B
:10DB0800A04207D10DE0002AE16880F2DF80884258
:10DB180007D00C46636823F003035A1B0F2AF2DD73
:10DB2800F446DFF850823C69444500F0BC806368E5
:10DB380023F00309A9EB05030F2B00F34581002B04
:10DB4800C7E9048880F22F81B9F5007FD7F804E08F
:10DB580080F0C98001234FEAD9014FEA59191944C5
:10DB680003FA09F357F831204EEA030E07EBC10315
:10DB7800083BA260E360C7F804E047F83140D4608E
:10DB880001204FEAAC039840704532D810EA0E0FD6
:10DB980007D12CF0030C400010EA0E0F0CF1040C16
:10DBA800F9D007EBCC0AD646E146DEF80C300BE09C
:10DBB80059681C4621F003014A1B0F2ADB6800F351
:10DBC800BF80002A80F2E2809E45F1D109F1010967
:10DBD80019F0030F0EF1080EE7D11FE10C23336093
:10DBE80000246CE74FF400704FF0400C4FF03F0EEC
:10DBF80082E7BC68636823F00309A94503D3A9EB4E
:10DC080005030F2B52DC5C4B08201B6803F110083E
:10DC180004EB0903009302F009FA584A8346136893
:10DC2800A844013305D008F1FF388044434203EA91
:10DC380008084146304602F09BF9B0F1FF3F8246A2
:10DC48004E4A00F0DC8004EB0903834200F2D580E1
:10DC58004B4B0BF1FF31186840448446186040F084
:10DC6800FB801AEA010F40F0F780D7F808A0C844F3
:10DC780048F00102CAF804205446424B1968814210
:10DC880038BF1860404B1968814238BF186022F0CD
:10DC98000308A845A8EB050301D30F2B06DC304683
:10DCA80000F09EF99CE7D7F804E069E7621943F0B1
:10DCB800010345F0010565603046BA6008345360D9
:10DCC80000F08EF9204603B0BDE8F08FA268304618
:10DCD800D16023448A60EBE6DC68A3427FF4DFAEC0
:10DCE8000CF1020C1DE7B9F5206F4FEA59227DD3DC
:10DCF800142A00F2118102F15C03DB005B32F9188F
:10DD0800FB580839994203D1ECE09B68994204D04A
:10DD18005A6822F003024A45F7D8D968C4E90231A3
:10DD28008C60DC602CE7142B6CD9542B00F2FD803E
:10DD38002B0B03F16F0C03F16E0E4FEACC00DBE600
:10DD4800D4F808C03046661945F001056560CCF87E
:10DD58000C30C3F808C042F00103C7E90466C6E9FD
:10DD680002887360625000F03BF90834A7E600BFF0
:10DD780048010020500100201C1F00203C01002009
:10DD8800EC1E0020181F0020141F002021444A68A0
:10DD9800304642F001024A6054F8082FD3609A6076
:10DDA80000F01EF98BE6A144D9F80430304643F060
:10DDB8000103C9F8043000F013F908347FE64FEA8C
:10DDC800D50C05F1080362E6621943F0010145F03C
:10DDD800010565603046C7E90422C2E9028851603E
:10DDE80044F8093000F0FCF8083468E64FEA991264
:10DDF80002F13903DB00383281E7BC4224D0BC6829
:10DE0800626844E703F15C0C03F15B0E4FEACC0057
:10DE180072E65AF80839534540F0D8801CF0030FD1
:10DE28000CF1FF3CF5D17B6823EA00037B604000DE
:10DE380098423FF6DEAE18B9DBE6400009F1040966
:10DE48001842FAD0CC46ACE6614B0BF1FF311868AA
:10DE580008EB000CC3F800C01068013070D004EB68
:10DE68000902AAEB020262441A601AF00702CDE91D
:10DE7800002340D0C2F108029244D04408EA0100CD
:10DE88005A44121A02EA010B5946304602F070F859
:10DE9800421C019B71D0A0EB0A0000EB0B0818682C
:10DEA80048F001025844BC42C7F808A01860CAF8F4
:10DEB80004203FF4E1AEB9F10F0F44D94FF0050C3F
:10DEC8006168A9F10C0222F0070201F00101114377
:10DED80061600F2A04EB0201C1E901CC55D8DAF8D8
:10DEE8000420C9E60120921000FA02F24EEA020E5E
:10DEF800C7F804E012E70AEB08020A40ABEB02029B
:10DF080002EA010B5946304602F032F8431C019BE5
:10DF1800C1D1DDF800B0C2E7542A18D84FEA193247
:10DF280002F16F03DB006E32E9E6B3F5AA7F18D879
:10DF3800EB0B03F1780C03F1770E4FEACC00DBE52D
:10DF4800C2F800A091E70123CAF80430A7E6B2F5A9
:10DF5800AA7F25D84FEAD93202F17803DB0077325D
:10DF6800CDE640F25452934225D8AB0C03F17D0C18
:10DF780003F17C0E4FEACC00BEE5009A4FF0000B8F
:10DF8800083A9044A8EB0A0889E7304604F10801EA
:10DF9800009302F0FDF8009BD7F808A018689EE7E8
:10DFA80040F254539A420DD84FEA994202F17D0348
:10DFB800DB007C32A3E64FF47E704FF07F0C4FF00D
:10DFC8007E0E99E54FF47E737E2298E67B682EE7F5
:10DFD800EC1E0020014802F025B800BF6020002098
:10DFE800014802F021B800BF6020002003460A461D
:10DFF80002490868194600F003B800BFC8060020A7
:10E008002DE9F84F1646002900F096800C46804608
:10E0180006F10B05FFF7DEFF54F8041C162DA4F1DA
:10E02800080921F0030758D81025AE4258D8AF4246
:10E0380060DABF4B09EB070C9A68DCF8040062450C
:10E0480000F0908020F0010363445B68DB0768D42C
:10E0580020F003003B189D4247DDCB0712D454F84B
:10E06800083CA9EB030BDBF8043023F0030210444F
:10E0780000EB070A554540F3F68007EB020A5545C1
:10E0880040F3CC8031464046FFF7F0FC06460028B6
:10E0980000F0218154F8043CA0F1080223F00103A8
:10E0A8004B44934200F0B4803A1F242A00F2D780F0
:10E0B800132A00F2A28003462246116819605168AB
:10E0C800596092689A602146404602F061F84046DD
:10E0D800FFF786FF3046BDE8F88F35F00705A4D571
:10E0E8000C23C8F80030002618E01F46DCE902239C
:10E0F800D3609A60D9F804307A1B0F2A03F0010321
:10E1080009EB07001DD83B43C9F80430436843F0C6
:10E11800010343604046FFF763FF26463046BDE8EB
:10E12800F88FC907AED454F8083CA9EB030BDBF809
:10E13800043023F00302A0E71146BDE8F84FFFF7CB
:10E1480095BC2B4309EB050142F00102C9F80430E4
:10E158004A604368083143F001034360404602F0D7
:10E1680017F8D7E720F00300C21905F1100C624533
:10E1780080F29280CA0785D454F8082CA9EB020BC8
:10E18800DBF8042022F00302104400EB070AD44510
:10E198003FF773AF5E46DBF80C1056F8080F3A1FCE
:10E1A800242AC160886000F2B080132A40F2AB8054
:10E1B80021681B2ACBF808106168CBF80C1000F214
:10E1C800AA8008340BF1100221681160616851605F
:10E1D800A1689160AAEB05020BEB050142F0010270
:10E1E80099604A60DBF80430404603F001032B4392
:10E1F800CBF80430FFF7F4FE90E723681B2A03608E
:10E20800636843603DD804F1080200F1080354E74D
:10E2180050F8043C23F003031F446BE75E463A1FA3
:10E22800DBF80C3056F8081F242ACB60996023D8F5
:10E23800132A1FD923681B2ACBF808306368CBF848
:10E248000C303CD808340BF1100322681A6062685D
:10E258005A60A2689A6034465746D9464AE721462A
:10E2680001F012FB2FE7DCE902135E46CB603A1F90
:10E278009960D5E73346E8E72146304601F004FBCC
:10E28800E9E7A368242A8360E368C36027D004F120
:10E29800100200F1100310E7521B09EB050142F0D0
:10E2A800010299604A6054F8043C404603F00103B7
:10E2B8002B4344F8043CFFF793FE26462EE7A36859
:10E2C800242ACBF81030E368CBF8143010D010347F
:10E2D8000BF11803B9E74046FFF782FE03E723690D
:10E2E80004F1180203616369436100F11803E4E66D
:10E2F80023691834CBF8183054F8043CCBF81C3098
:10E308000BF12003A1E732465EE72146304601F0D3
:10E31800BBFA074B5EE7A168242ACBF81010E16826
:10E32800CBF8141006D010340BF118024CE700BFDC
:10E338004801002022691834CBF8182054F8042C1E
:10E34800CBF81C200BF120023EE700BF00000000C4
:10E358002DE9F04F9FB08846079200210022002443
:10E36800CDE90412834641461A9419910F4611F8D3
:10E37800012B2D2A5ED801A050F822F05BE5000899
:10E388003DE400083DE400083DE400083DE40008E1
:10E398003DE400083DE400083DE400083DE40008D1
:10E3A80073E3000873E3000873E3000873E30008ED
:10E3B80073E300083DE400083DE400083DE400087C
:10E3C8003DE400083DE400083DE400083DE40008A1
:10E3D8003DE400083DE400083DE400083DE4000891
:10E3E8003DE400083DE400083DE400083DE4000881
:10E3F8003DE400083DE400083DE4000873E300083C
:10E408003DE400083DE400083DE400083DE4000860
:10E418003DE400083DE400083DE400083DE4000850
:10E428003DE400083DE40008DDEA00083DE400089A
:10E43800F1EA000800210891302A00F095800023B5
:10E4480009932F2A144640F2EF844FF0000938460A
:10E458004E464D4613E00130082D1990C8BF09EB10
:10E4680089090478C6BF02EB4902A2F13009A3F179
:10E4780030062F2C224605F1010540F3B48006EB47
:10E488008603392C02EB4303E5DD0122AB4901F099
:10E49800C9FA002879D1199A1346013219925C7881
:10E4A800002D40F08D85302C40F03B8513461846F2
:10E4B800013319931C78302CF9D0C2F101021044B1
:10E4C800A4F13103082B37D8199F012539464FF09D
:10E4D800000A431CA4F1300E0C93002006EB8606BC
:10E4E8000EEB46064B1C19934C78A4F13002092A0E
:10E4F80000F2E082964619990130002AF2D00128EC
:10E50800D8BF05F1010C40F3878400EB050C0CF132
:10E51800FF340A9703E07E00AC4200F07C84082DAB
:10E5280006EB860705F10105F5DD102DDCBF09EBCB
:10E5380089094FEA4909EFE7652C40F0D8824FF086
:10E54800000A0123CDF830A00A93099B034340F049
:10E55800BF82079B002600270BB1C3F80080304616
:10E5680039461FB0BDE8F08F7A7802F0DF02582AEA
:10E5780000F01284013719973A78302AFAD0002A25
:10E5880000F08182012309935BE70020AA460C90E2
:10E598000A90652C34D0452C32D000231093002DDE
:10E5A8007AD1099B034340F06E820A9B002BD0D19D
:10E5B800692C00F0898400F35F84492C00F084847E
:10E5C8004E2CC6D15E4919A802F004FA0028C0D022
:10E5D800199B1B78282B00F0A5855A4801F062FD8D
:10E5E80006460F4651E20122544901F01BFA002861
:10E5F800CBD1199BAA465A1C19925C780C9074E7E7
:10E60800002DA2D0DDF8648008F10103199398F871
:10E6180001402B2C00F059822D2C00F04E824FF037
:10E62800000CA4F13001092900F23F82302C199B1B
:10E638000AD1013319931C78302CFAD0A4F1310295
:10E64800082AAAD8A4F130015A1C19925C782F2CF8
:10E6580040F3FE8396460B9308E0013219929EF828
:10E668000140A3F130012F2C06DD964601EB810312
:10E67800392C04EB4303F0DD0B9BD21A082A40F334
:10E68800E78344F61F631093BCF1000F87D0109BFB
:10E698005B421093002D84D00C9A109BBAF1000FA6
:10E6A80008BFAA469B1A102D30460B932C46A8BFCC
:10E6B8001024F1F7D7FE02460B46092DCDE90423B5
:10E6C80016DD214B03EBC40353E91223F2F782FC56
:10E6D8000246484690468946F1F7C4FE02460B4674
:10E6E80040464946F1F782FD0F2DCDE904012DDCA6
:10E6F8000B9B002B00F020830B9B40F35282162BC0
:10E7080040F3AD830B9AC5F1250393421EDBDDE987
:10E7180004230D4CC5F10F0504EBC501D1E9000137
:10E72800F2F758FC0B9B5D1B04EBC504D4E90023EE
:10E73800F2F750FC06460F46A7E100BF98AC010867
:10E74800A8AC0108E8A9010870E401080B9B2C1B80
:10E758001C44002C40F3D18114F00F000AD0DDE9ED
:10E768000423354901EBC001D1E90001F2F732FC7D
:10E77800CDE9040134F00F0340D0B3F59A7F00F3DC
:10E78800B883102B4FEA231440F31E85DDE90401FA
:10E7980000232A4A0997904699461746E20704D566
:10E7A800D8E90023F2F716FC01236410012C09F1C3
:10E7B800010908F10808F1D13A46099F0BB1CDE9E2
:10E7C8000401059B02EBC901A3F154730593DDE92C
:10E7D8000423D1E90001F2F7FDFB194B194A0B405C
:10E7E8009342CDE9040100F28483174A934240F230
:10E7F80041844FF0FF33154CCDE9043400230A93CC
:10E808002B46524639465846009602F07DFA149037
:10E81800002800F06E83109A0C9B4FF0000A9B1A98
:10E828000B9ACDF824A0002AA8BF0023109322EA4F
:10E83800E2731593E5E000BF70E4010848E40108BD
:10E848000000F07F0000A07C0000907CFFFFEF7FBD
:10E85800D21A1F2AA4EB020400F332820123934048
:10E868001E4600250A9BA0444C44A14598444B46AB
:10E87800A8BF23464345A8BF4346002B04DDE41A3E
:10E88800A8EB0308A9EB0309109B002B00F3BE813A
:10E89800002C00F3D4810B9B002B00F30782B8F106
:10E8A800000F00F3F781B9F1000F08DD51464A4621
:10E8B800584602F00BFC8246002800F0F4813A46E4
:10E8C80058461A9902F098FC0990002800F0EB814C
:10E8D8000023099AD168D3601191514602F06CFC6B
:10E8E8000028C0F2EA83DDF8149000F076835146E0
:10E8F800099802F01DFE00224FF0804304460D46A1
:10E90800F1F794FE002800F07181119B002B40F074
:10E91800E381049B002B40F06B82C9F31303002BA7
:10E9280040F00D82002220462946A94BF1F774FEDB
:10E93800002840F049832046A64B29460022F2F7DA
:10E9480049FB03460C46CDE9123401F100430E9011
:10E958000F93DFF88482A14B09EA08089845DDE99E
:10E968000E4500F0C0810A9B1BB3B8F1D46F20D8C4
:10E9780095A3D3E90023DDE91201F1F757FEA0B111
:10E98800DDE91201F2F738FD012838BF0120F1F75F
:10E9980069FD119BCDE91201002B40F0BD8201F108
:10E9A800004316901793DDE9164505F1D663A3EBEE
:10E9B8000805DDE90C0102F0DBFC02460B462046A7
:10E9C8002946F2F707FBDDE90C23F1F70FFC0C46AB
:10E9D800CDE904010A9B23B97F4B2340984500F0F9
:10E9E800B78158461A9902F033F93946584602F069
:10E9F8002FF95146584602F02BF95846099902F06A
:10EA080027F9149C5846616802F0FCF8074600286C
:10EA180000F04981226904F10C01023292000C30A5
:10EA2800F2F762FA1CAB01931BAB00935846DDE981
:10EA380004341A46CDE90C34234602F01BFD1A9023
:10EA4800002800F005810121584602F005FA8246A7
:10EA5800002800F028811B9B002BC0F21581109A1A
:10EA6800DDF8548003EB02090A9A1C9C9B1A234484
:10EA78005B4A013B9342C4F13604FFF6E9AE012339
:10EA880000251E46EEE600260027079A0AB1199BC4
:10EA98001360089B002B3FF462AD07F100431F464B
:10EAA800304639461FB0BDE8F08F0023CDF86480AA
:10EAB800109374E501230A936BE54FF0010C08F1FC
:10EAC8000203199398F80240ABE54FF0000CF6E703
:10EAD800002597E500220892791C19917A78002A76
:10EAE8003FF437AD0F46A7E401220892F4E7452C1E
:10EAF8003FF425AD01230A9353E53FF47FAE64420A
:10EB080014F00F020AD0DDE90401364B03EBC2030F
:10EB1800D3E90023F2F788FBCDE9040124113FF47F
:10EB28006DAE1F2C37DCDDE9040114F0100318BFAB
:10EB38006A230A930023DFF8B080E20704D5D8E9F6
:10EB48000023F2F747FA0123641008F10808F4D10A
:10EB58000BB1CDE904010A9BA3B1DDE90401C1F3BE
:10EB68000A52C2F16B03002B0ADD1F2B40F33983D5
:10EB78000020342B049040F37C834FF05C730593A2
:10EB88006A230A930022DDE904010023F1F73AFD24
:10EB980000283FF435AE222300260027CBF80030AA
:10EBA80073E71633FFF6D2ADDDE904010C9B109A2A
:10EBB8009A1A0C4B03EBC203D3E90023F2F734FB98
:10EBC80006460F4661E700BF0000C0FFFFFFDF41B8
:10EBD8000000F03F0000E03F0000F07F0000E07F11
:10EBE80002FCFFFF70E4010810E20108AC4B20466C
:10EBF80029460022F2F7EEF9119BCDE91201002B0C
:10EC080065D101F100430E900F93A2E651461A46D2
:10EC1800584602F001FA8246002844D001461A9A62
:10EC2800584602F047F900283DD011901A995846E5
:10EC380002F00EF8119B002C1A937FF72CAE224697
:10EC480058461A9902F042FA1A9000287FF423AE27
:10EC5800B946054622230026924FCBF800302946B4
:10EC6800584601F0F5FF4946584601F0F1FF514674
:10EC7800584601F0EDFF5846149901F0E9FF58464F
:10EC8800099901F0E5FF00E7159ADDF84090A2EB3D
:10EC98000308E9E639464246584602F017FA07469D
:10ECA80000287FF400AEB9461A9DD3E73946584686
:10ECB800159A02F0B1F9074600287FF4F0ADF2E7A3
:10ECC800012279491646CB1A02FA03F5CAE5DDE9AD
:10ECD8001234CDE90E343CE60023744CCDE90E34F1
:10ECE800CDE9123435E6A9F154730593DDE90445FD
:10ECF8002046294602F03CFBDDE90E23F2F76AF9CB
:10ED08002B462246F1F772FADFF89891684B01EA30
:10ED180009099945CDE9040179D9DDE90C0103F127
:10ED28005473994202D106460136BCD04FF0FF33E6
:10ED3800604CCDE9043454E6DDE90467A5E6002318
:10ED48005D4CCDE90E340023584CCDE9123400E671
:10ED5800DDE91256284631460BF0D4FAF1F7CEFB1E
:10ED68000B46024631462846F1F73EFA119D049BB0
:10ED7800C4F313041D432C438046894626D142A37D
:10ED8800D3E90023F1F748FC00283FF42AAEB9463E
:10ED9800DDE904671A9D62E70293089B58460193D0
:10EDA8001AAB0093454A1BAB19A901F03FFB10F0C1
:10EDB8000F0504463FF467AE062D40F0B5800022EB
:10EDC8007B1C00260027089219935EE630A3D3E93E
:10EDD8000023F1F721FC0028D9D12FA3D3E9002380
:10EDE80040464946F1F736FC00283FF4FAADCEE735
:10EDF800049B012BA3D1B9F1000FA0D1B9461A9CED
:10EE08002223254600260027CBF8003027E701F10A
:10EE180054740594DEE50A9F0C9B082D03440C935B
:10EE28006DDC6546FFF759BB01223846244900F0DE
:10EE3800F9FD002800F0BB804FF000094E46484617
:10EE48004D46CA46CDF83090CDF82890FFF7A3BBC1
:10EE580044F61F639942A8BF1946109114E40B9811
:10EE68001849DDE9042301EBC001D1E90001F2F7FB
:10EE7800B1F806460F4608E66E2C3FF4A3ABFFF741
:10EE880068BB00BFAFF300809535A094FFFFCF3F6C
:10EE98009535A094FFFFDF3F35E5AF350000E03F33
:10EEA8000000E03F0000F07FE2FBFFFF0000F03FC2
:10EEB800FFFF9F7CFFFFEF7F0000F0BFFCE1010830
:10EEC80098AC010870E40108A04919A801F082FD76
:10EED80000283FF43EAB199B9D49013B19A81993A3
:10EEE80001F078FD10B9199B013319930026994F49
:10EEF800CBE522230026974FCBF80030C5E5BCF1BF
:10EF0800100FD8BF09EB890965464FF00000D8BF3C
:10EF180002EB4909FFF7E6BADDE91234CDE9163408
:10EF280041E50020FFF7CCBA1A9A3AB135211CA85E
:10EF380002F02CFB58461A9901F08AFE013D1B9BF2
:10EF4800042D00F2C481DFE805F0032C291E03001C
:10EF58001C9A049203F233421D9B23F4801343EA64
:10EF680002530593E10502D543F000430593794A1E
:10EF7800DDE904671A40002A7FF487AD01F020F824
:10EF88002223036081E54FF0FF326FF00043CDE9A3
:10EF98000423E3057FF5D0AE059BE5E76D4B0593AC
:10EFA800F7E7DDE91C121D9BCDE90412DAE7199A8F
:10EFB800064613460132199281465C78FFF773BA08
:10EFC800AA460C90FFF791BA0023634CCDE90E34A2
:10EFD8000023624CCDE91234BBE44B461198B44689
:10EFE800B946DDE90C67AE465D49C3F31302002854
:10EFF80045D08A4200F0FD80ADBB049A1CEA020F9E
:10F0080034D030463946049302F0B2F90A9B002BFB
:10F0180000F03781049BC3F30A53C3F16B03002B41
:10F0280040F352811C0504F17F53002203F540137D
:10F03800F1F7D0FF02460B4630463946F1F7D6F8CD
:10F0480006460F4630463946464B0022F1F7C2FFC6
:10F05800404B06460B400F46002B7FF49BAE222305
:10F06800CBF8003096E61EEA030FCAD10A9B002BA4
:10F07800E8D18FE601F154730593FFF7BFBB002A6F
:10F0880074D1DDE904452246002C40F0A2800A9A9A
:10F09800002A40F0CB8025F00044240D2405A4F577
:10F0A80080146FEA14536FEA035305934FF0FF334C
:10F0B80004931A9DDDE90467D1E5119BDDE904019C
:10F0C8000343B946DDE90C67D0D1C1F31303002B24
:10F0D800CCD121F00044240D2405B4F1D66F254687
:10F0E800C4D9099A536913B91369012BBEDD0122EA
:10F0F8000999584601F0EAFF5146099002F05CF878
:10F108000028B3DD0A9B002BC9D0A5F580136FEA50
:10F1180013536FEA035305934FF0FF330493DDE96C
:10F1280004678FE7104919A81CAA01F06DFC05288F
:10F138007FF453AA1D9B43F0FF4343F4E003059378
:10F148001C9B0493DDE904679FE400BF9CAC0108A5
:10F15800A0AC01080000F07F0000E0BF0000E03F25
:10F16800FFFF0F0000005039E8E10108A5BB049A31
:10F178001CEA020F3FF47AAF30463946049302F096
:10F18800F7F80A9B002B62D0049BC3F30A53C3F120
:10F198006B03002B40F38C801C0504F17F53002285
:10F1A80003F54013F1F716FF02460B463046394681
:10F1B800F1F71AF80022002306460F46F1F722FA63
:10F1C80000283FF43FAF1AE64FF00009414AFFF725
:10F1D800F8BABEF1000FCBD01EEA030F3FF446AFDA
:10F1E800CAE74FF0FF3202FA03F3049A1A40049276
:10F1F800C6E40A9A0499B2B1374A1A40B2F1D46FF8
:10F2080011D84FF0FF30120DC2F16B0200FA02F272
:10F21800914240D0BEF1000F7FF425AF11EA0C0FE8
:10F228003FF424AFEDE64FF0FF32F1E72A4D1D40E1
:10F23800B5F1D66F3FF669AFB5F15C7F3FF602AF27
:10F248002223002600271A9DCBF8003007E5024646
:10F258000B4630463946F0F7C7FF1A9C00220023B8
:10F2680006460F462546F1F7CDF900283FF4F7ACDE
:10F27800C6E54FF0FF33C2F14B0293400B400593B4
:10F288007EE402460B4630463946F0F7AFFF1A9D3A
:10F2980006460F46E3E4114A93420CD00E4A1A4040
:10F2A80002F58013059300230493DDE90467DDE686
:10F2B80002460B467AE70131F0D1222300261A9D37
:10F2C800054FCBF80030CAE402460B46B4E60023EB
:10F2D80048E600BF48E401080000F07FFFFFEF7F29
:10F2E800014BFFF735B800BF5C05002084460A468D
:10F2F8000249034B08686146FFF72AB8C806002090
:10F308005C050020024A0349034800F0C9B800BF61
:10F31800500500202D790108D00600200C4B4168CB
:10F3280010B59942044601D008F0FCFAA168094BCF
:10F33800994202D0204608F0F5FAE168064B994256
:10F3480004D02046BDE8104008F0ECBA10BD00BF5C
:10F35800201F0020881F0020F01F00202DE9F843FF
:10F3680000250423304C314A3149DFF8C890DFF8D2
:10F37800C880324F324E116004F15C0029460822E1
:10F38800C4E90335C4E90055C4E90555A5606566B7
:10F3980000F0F8FA04F15800C4E90749C4E90987FC
:10F3A800E66200F03BFE274B2946082204F1C40020
:10F3B8006367C4E91A55C4E91E552567C4F8CC50DB
:10F3C800C4F8805000F0DEFA04F1680304F1C000CC
:10F3D800C4F88430C4E92298C4E9247600F01EFEFB
:10F3E800194B294604F596700822C4F8DC30C4E9A4
:10F3F8003455C4E93855C4F8D850C4F83451C4F861
:10F40800E85000F0BFFA04F1D003C4E93D87C4F81E
:10F41800F09004F59470C4F8FC60C4F8EC30BDE8D2
:10F42800F84300F0FBBD00BF201F0020582000203B
:10F438000DF30008FDF7000825F8000865F8000836
:10F4480089F80008090001001200020010B50446FE
:10F458000A4800F0E7FD636B23B9094B094A1B68AA
:10F46800626323B1BDE81040044800F0DDBDFFF73A
:10F4780075FFBDE81040014800F0D6BD68200020A7
:10F488005820002025F30008014800F0CBBD00BF3C
:10F4980068200020014800F0C7BD00BF6820002098
:10F4A8002DE9F8434FF0000980460F461646D6E985
:10F4B8000154013D10D4A389012B08D9B4F90E30A9
:10F4C800013304D021464046B84749EA0009013DC6
:10F4D8006B1C04F16804EED13668002EE7D148466B
:10F4E800BDE8F8830FB400B5074A83B004AB1068D1
:10F4F80053F8042B8168019305F062FB03B05DF8B3
:10F5080004EB04B0704700BFC806002030B50546BC
:10F5180089B008460C4600F097FD012302222049D5
:10F5280007936B6B0691029204A9421C0494019103
:10F53800AC6805900392002B2ED0626EB4F90C30A3
:10F54800D20701D4980521D5990406D4626E43F4F4
:10F55800005322F40052A3816266284601AA21467C
:10F5680008F0FEFA636E00280CBF0A254FF0FF353D
:10F57800DA0702D4A3899B0502D5284609B030BD15
:10F58800A06D00F051FD284609B030BDA06D00F017
:10F5980049FDB4F90C30D7E72846FFF757FFCCE709
:10F5A800BCAA0108024B01461868FFF7AFBF00BFAD
:10F5B800C80600202DE9F043664C0E46D4F80080BA
:10F5C800174604461D4683B0B8F1000F04D0D8F89A
:10F5D8003430002B00F0A680022F05D0012F00F256
:10F5E800A580002DC0F2A280636EDA0751D52146AE
:10F5F800404608F08BFA216B41B104F1400399426F
:10F6080002D0404600F0C4FD002323630023B4F970
:10F618000CC0A3611CF0800F63605DD12CF44A6CB0
:10F628002CF0030C022FA4F80CC063D001AB2146C8
:10F6380040466A4608F078FCA3891843A081002D4B
:10F648002ED0002E2DD0D8F83430002B37D0009A89
:10F65800B4F90C30AA421CBF43F40063A381012F04
:10F6680004BF43F00103A38113F00802C4E9046551
:10F67800266028D0D90753D50022A260626E6D4259
:10F68800D207A56123D49B0521D4A06D00F0CCFC42
:10F698001DE0A3899B05AAD4A06D00F0C3FCA6E7D2
:10F6A800009D2846FEF7D2F90646002841D0A389D6
:10F6B80043F08003A381D8F83430002BC7D14046EB
:10F6C800FFF7C4FEC3E7A260626ED207DBD5002550
:10F6D800284603B0BDE8F0834046216900F058FD94
:10F6E800B4F90CC0022F2CF44A6C2CF0030CA4F8CB
:10F6F8000CC09BD100250021012204F143032360A3
:10F708002361636E4CF00200A081D807A16062619A
:10F71800DED41CF4007FDBD1A06D00F085FCD7E7B8
:10F72800A560D1E74046FFF791FE55E74FF0FF355A
:10F73800CEE7DDF80090A94506D04846FEF786F9E1
:10F74800064608B14D46B2E74FF0FF35B4F90CC094
:10F75800D1E700BFC80600200EB430B504466FF0EC
:10F7680000459CB00B4A1FAB0B49059253F8042B7C
:10F77800086802A9CDE9013404950795069402F0BA
:10F788000DF80022029B1A701CB0BDE8304003B08F
:10F79800704700BF0802FFFFC80600200EB44FF4F0
:10F7A800017270B59DB021AD55F8046BADF8142009
:10F7B8000290069000F048FC00234FF6FF710446C3
:10F7C8000E931393094A0A4B0A92ADF81610324663
:10F7D800186802A92B4601950394079403F074FD59
:10F7E8001DB0BDE8704003B0704700BF21F80008A5
:10F7F800C806002010B50C46B1F90E1000F0A2FBA7
:10F80800002803DB236D0344236510BDA38923F47B
:10F818008053A38110BD00BF002070472DE9F0413F
:10F828000C46B1F90C101F46CB05054616460BD4FD
:10F8380021F48051A1813B4632462846B4F90E1086
:10F84800BDE8F04100F0A6BBB4F90E100223002277
:10F8580000F062FBB4F90C10EAE700BF10B50C46E3
:10F86800B1F90E1000F058FBB4F90C30421C0EBF71
:10F8780023F4805343F480532065A38110BD00BF57
:10F88800B1F90E1000F036BB88420ED98B188342AE
:10F898000BD900EB020C002A6DD0624613F801CD9B
:10F8A800994202F801CDF9D170470F2A0FD80346C3
:10F8B80002F1FF3C002A5ED00CF1010C013B8C44A4
:10F8C80011F8012B614503F8012FF9D1704740EA7F
:10F8D80001039B0750D1A2F1100370B501F1200C70
:10F8E80023F00F0501F1100E00F11004AC441B09C0
:10F8F8005EF8105C0EF1100E44F8105C5EF81C5CAB
:10F90800103444F81C5C5EF8185C44F8185C5EF827
:10F91800145CE64544F8145CEAD1013312F00C0F8C
:10F9280001EB031102F00F0400EB031328D08E46FD
:10F93800043C24F003064FEA940C1E441C1F5EF896
:10F94800045B44F8045FB442F9D10CF1010402F0FD
:10F95800030203EB840301EB840102F1FF3C4AB18B
:10F968000CF1010C013B8C4411F8012B614503F8A3
:10F97800012FF9D170BD7047034602F1FF3C9BE7A8
:10F988002246EAE770B5860747D0541E002A3ED0C3
:10F998000346CAB201E0013C39D303F8012B9D07A5
:10F9A800F9D1032C2CD9CDB205EB05250F2C1A461D
:10F9B80005EB054534D9A4F1100C2CF00F0603F122
:10F9C800100EB6444FEA1C1CC2E90055C2E90255A4
:10F9D80010327245F8D10CF1010214F00C0F03EB50
:10F9E800021204F00F0C13D0ACF1040323F003034C
:10F9F8000433134442F8045B9342FBD10CF0030434
:10FA08002CB1C9B21C4403F8011BA342FBD170BD41
:10FA180064461346002CF4D1F9E703461446C0E7C0
:10FA2800A446E1E7002A3ED0844630B504460843A0
:10FA380080070B462ED1032A07D82BE0043A25D09D
:10FA48001EF0803F22D1032A22D919462068A446F5
:10FA5800A0F1013323EA000E0B4653F8045B04348B
:10FA6800A842EBD09CF800000C7884421DD1E646F1
:10FA780068B11EF8010F11F8014FA2EB0E03A04266
:10FA880003F1FF3311D11CEB0303F1D1002030BD8A
:10FA9800A44619469CF800000C78A04205D1012A1A
:10FAA800F4D0E646E4E710467047001B30BD00BFBF
:10FAB80001292DE9F0415AD901274FF0000E4FF0E6
:10FAC800FF34BC463B4607E09E464FF0010C1F1B27
:10FAD8000EEB0C0399420ED9051915F80C50C65CAB
:10FAE800AE42F1D333D00127BC467446BE440EEB78
:10FAF8000C039942F0D84FF001084FF0000E4FF078
:10FB0800FF35C4464346176008E09E464FF0010C97
:10FB1800A3EB05080EEB0C0399420FD9461916F80A
:10FB28000C60C75CB742F0D819D04FF00108C44642
:10FB38007546C6440EEB0C039942EFD80135601C9C
:10FB4800854202D32846C2F80080BDE8F081BC4552
:10FB58000ABFE6440CF1010C4FF0010CB8E7C445AC
:10FB68000ABFE6440CF1010C4FF0010CD2E74FF04C
:10FB780001080025E6E700BF2DE9F04F9346ADF2F6
:10FB88001C4D05AA80468A46584619461C46FFF76A
:10FB98008FFF814613460DF2144243F8044F9342F7
:10FBA800FBD16CB1601E58440BF1FF3206AD12F860
:10FBB800011FA31A013B5B44824245F82130F6D16C
:10FBC800059B4A4658460BEB0301019308F0FAFAE5
:10FBD800002879D10746054644F40063AAEB040ED1
:10FBE8000293661EAE4512D308EB050C1CF80630CE
:10FBF80006AA52F82330CBB127B1019A9A4284BFA2
:10FC08001346E31A1D44AE454FF00007ECD208EB4B
:10FC18000A00029908F0A2FB8244AAEB040EAE4542
:10FC2800E2D200200DF21C4DBDE8F08F4F453B4657
:10FC380038BF4B469E4218D9591EEA1859444244C7
:10FC4800009502E001339E420ED012F8010B11F824
:10FC5800015F8542F6D09E42009D06D9C9F1010296
:10FC68002A440027D518BDE7009D4F4509F1FF3309
:10FC780080F0828005EB090242440BEB09010095F4
:10FC8800CDF80C9002E09F4213D04B4611F8015D6D
:10FC980012F8010D03F1FF398542F4D0009DDDF81B
:10FCA8000C90013301379F4209D8019B1D44E71A84
:10FCB80098E701379F42009DDDF80C90F5D9604622
:10FCC8000DF21C4DBDE8F08FA4EB09034B4538BF7E
:10FCD8004B460025013344F40062AAEB040E00925F
:10FCE800661E01930593AE4509D308EB0500835DB5
:10FCF80006AA52F823306BB11D44AE45F5D208EB85
:10FD08000A00009908F02AFB8244AAEB040EAE45CB
:10FD1800EBD286E7B14517D209F1FF3105EB0902AD
:10FD28004B465944424402E00133B3420CD012F826
:10FD3800017B11F801CFBC45F6D09E4204D9C9F128
:10FD480001022A44D518CEE7B9F1000F3FF46AAF93
:10FD580005EB090141440BEB090203E0013B5B455C
:10FD68003FF460AF134611F8017D12F801CDBC4590
:10FD7800F4D0019B1D44C0E74B4693E72DE9F041C1
:10FD88000D460978044690B0002954D06A78002AB4
:10FD980000F08280AB78002B51D0E8782E680028DC
:10FDA80000F081802B79002B56D0284600F04CF9C2
:10FDB8000646204646F4007108F0D0FA86425AD822
:10FDC800FE2E00F28880801B271840226846711C8E
:10FDD800FFF7D8FD7EB16A1E5FFA86FC901912F80B
:10FDE800013F03F03F034033A91A6B44614490423A
:10FDF80003F8401CF3D1013CA35D03F03F034033FB
:10FE08006B4413F8403C1C44A74203D238E04444F6
:10FE1800A74235D314F806C032460CF03F0C0CF15B
:10FE280040030DEB030C294620461CF8408C08F0D3
:10FE3800C9F90028EBD1204610B0BDE8F081007860
:10FE480042EA0142B8B140EA03439A42214614F813
:10FE5800010FF7D14C1EEEE7227862B131BA01E00A
:10FE68008B421ED0204642EA032314F8012F002AB1
:10FE7800F6D18B4215D00024204610B0BDE8F081A1
:10FE8800BB5DB819002BF6D04FF4006108F066FA94
:10FE98000744A742AFD2EEE710B0BDE8F04108F042
:10FEA800BFB9C41EC7E7120442EA0162217842EAD8
:10FEB80003230029DFD0024601E00029DBD041EA14
:10FEC8000200B3EB002F25464FEA002214F8011F69
:10FED800F3D1AC1EAFE7014633462A46204610B0A0
:10FEE800BDE8F041FFF748BE014B93F82801704781
:10FEF8005C050020002238B5064D044608462A60F5
:10FF0800F1F766FD431C00D038BD2B68002BFBD0F1
:10FF1800236038BD5C20002038B50C46114600220D
:10FF28008446074D20462A601A466446F1F75CFD70
:10FF3800431C00D038BD2B68002BFBD0236038BD94
:10FF48005C20002038B50C46114600228446074D37
:10FF580020462A601A466446F1F74EFD431C00D03D
:10FF680038BD2B68002BFBD0236038BD5C200020F7
:10FF7800002238B5064D044608462A60F1F740FFCE
:10FF8800431C00D038BD2B68002BFBD0236038BD44
:10FF98005C20002038B50C46114600228446074DE7
:10FFA80020462A601A466446F1F7F8FC431C00D044
:10FFB80038BD2B68002BFBD0236038BD5C200020A7
:10FFC800014B1868704700BFC806002070B50F4B7A
:10FFD8000F4DAB42A3EB050607D00024B61055F829
:10FFE800043B01349847A642F9D80AF01BFB094D97
:08FFF800094B5E1BAB424FEA0E
:020000040801F1
:10000000A60606D0002455F8043B01349847A642C2
:10001000F9D870BD70500208705002087050020884
:1000200078500208704700BF704700BF704700BF9C
:10003000704700BF082802D14FF48050704708B5C0
:10004000FFF7C2FF162203464FF0FF301A6008BDCB
:1000500020F0030110F00300C0F1000051F8043B50
:1000600000F1040C4FEACC0C6FF000021CBF22FA26
:100070000CF213434FF0010C4CEA0C2C4CEA0C4CE4
:10008000A3EB0C0222EA030212EACC1204BF51F8DD
:10009000043B0430F4D0C2F1000102EA0102B2FADA
:1000A00082F2C2F11F0200EBD2007047002001492A
:1000B000704700BF0000F87F004870470000C07F15
:1000C000024B13B1024800F005B870470000000071
:1000D00059840108002301461A46184608F052BA0E
:1000E0002DE9F843064608208946FFF7A3FF054699
:1000F000DFF898803046FDF771FFD8F808305F6868
:1001000027F00307A7F11104A4EB09042C44B4FB66
:10011000F5F4013C05FB04F4A54208DC002130465F
:10012000FFF72AFFD8F808303B44984205D0304604
:10013000FDF75AFF0020BDE8F88330466142FFF723
:100140001BFF01300FD0124AD8F808303F1B47F090
:1001500001075F60136830461B1B1360FDF744FF07
:100160000120BDE8F88300213046FFF705FFD8F8ED
:100170000820831A0F2BDADD43F001035360054B8F
:1001800003491B68C01A0860D1E700BF480100207E
:10019000EC1E00203C01002000297CD0F8B50C4664
:1001A0000646FDF71BFF54F8043C764FA4F1080502
:1001B00023F001016818D7F808C04268844522F08E
:1001C000030200F08380DB07426000EB020C33D4B3
:1001D00054F8084CDCF804302D1B2144AC6807F1BE
:1001E000080C644503F0010364D0D5F80CE0C4F8B2
:1001F0000CE0CEF80840002B00F0818041F00103B4
:100200006B600160B1F5007F22D20122CB08490961
:100210008A40796801330A437A6057F8331007EB54
:10022000C302083AC5E9021247F83350CD603046A0
:10023000BDE8F840FDF7D8BEDCF80430DB072BD56D
:1002400041F00103B1F5007F44F8043C0160DCD3C8
:10025000B1F5206F4FEA512353D28B0903F13900D6
:1002600003F13802C300F818FB580838984203D14C
:1002700061E09B68984204D05A6822F003028A42E7
:10028000F7D8D868C5E9023085603046DD60BDE842
:10029000F840FDF7A9BE7047114407F1080C8368C8
:1002A00063453FD0C268DA60936041F001036B6040
:1002B0006950A7E7002B5FD10A44D0E90213CB6055
:1002C000996042F001036B60AA50B0E70A44D90775
:1002D00007D454F8083CED1A1A44D5E90213CB6050
:1002E000996042F001036B60274BBD601B6893422D
:1002F0009DD8264B30461968FFF7F2FE97E7114468
:10030000CDE7142B08D9542B1DD80B0B03F16F002C
:1003100003F16E02C300A6E703F15C0003F15B0288
:10032000C300A0E741F00103C7E90455C5E902CCC9
:100330006B6069507BE70121921001FA02F2796843
:100340000A437A609EE7B3F5AA7F06D8CB0B03F188
:10035000780003F17702C30085E740F254529342DC
:1003600006D88B0C03F17D0003F17C02C3007AE711
:100370004FF47E737E2276E741F001036B600160EB
:1003800055E700BF48010020400100201C1F00204D
:100390002DE9F0410469B4EB611F05DC0023036122
:1003A00000234361BDE8F08100F114054E1111F006
:1003B0001F0C05EB840E05EB860321D055F82610A3
:1003C00004339E4521FA0CF1CCF120082DD92F469B
:1003D0001A6802FA08F20A4347F8042B53F8041B80
:1003E0009E4521FA0CF1F3D8A31B9B00053B9B080B
:1003F000013305EB830445F8231079B104340DE093
:100400009E4588BF00F11002C8D953F8041B9E45D1
:1004100042F8041FF9D8A41B05EB8404631B9B104E
:10042000AC420361BCD0BDE8F08141610029B5D088
:100430002C46E3E72DE9F04F1C4685B00090086894
:10044000934682780B46302A029440F0F381C11C17
:100450000A780C46302A01F10101F9D0A4EB000919
:10046000A9F10209DFF8C08218F80220002A00F082
:10047000EF80002722783D4618F80220002A00F07D
:100480007781264616F8012F18F80220002AF9D1A4
:1004900001223046A5490193FFF7C8FA019B824625
:1004A00000284DD03278002D00F0A581A5EB060A7A
:1004B0004FEA8A0A02F0DF02502A35464DD01E600C
:1004C000002F74D12B1B013B072B394604DD5B1039
:1004D000072B01F10101FADC009800F097FB0346BD
:1004E000002800F06A8200F11406A542019640F24D
:1004F000CA8100270390B9460DE0202F1AD0394653
:1005000004372A7818F8022002F00F028A4049EADC
:100510000209A54254D015F8012D2E2AEDD1A5428D
:10052000EBD3012228468149FFF780FA0028F0D05A
:10053000202FE4D1002146F8049B04278946E0E7F8
:10054000002D00F068813278A5EB060A02F0DF0288
:10055000502A35464FEA8A0AB1D16A782B2A00F030
:1005600048812D2A40F0D5800120AA78AE1C18F8C9
:1005700002104A1E182A00F2D5807278103918F835
:10058000022001365AB90CE001EB810102EB410275
:10059000A2F1100116F8012F18F802200AB1192A49
:1005A000F2DD00B149428A441E60002F8AD0B9F1C1
:1005B000000F0CBF06250025284605B0BDE8F08FCA
:1005C000039B019A46F8049BB61AB6101E61484672
:1005D000039300F0F5FB7601DBF80040361AA642E3
:1005E000039B76DCC0F209810027DBF80820524526
:1005F000C0F23E81DBF8042052454EDDA2EB0A0A30
:10060000544500F39580DBF80C10022900F0E180DE
:10061000032900F05381012940F0DF80544540F068
:10062000DC80012C0AD01846611E039300F0E2FF23
:10063000039B002800F0D180DBF804200121029800
:1006400062250260019A196111600E9A1360B3E786
:100650000122204635490193FFF7E8F9019B07463F
:10066000002840F087806278651C18F80210002985
:1006700000F08280302A2C4640F02B8114F8012FA4
:10068000302AFBD018F802204FF00109B2FA82F7A5
:100690007F09002A7FF4F5AE6AE0012587B1DBF817
:1006A0000C20022A6FD0032A71D0012A06D1B90783
:1006B00004D5019A12681743FA076BD445F0100568
:1006C00028460E9A1360029BC3F800A005B0BDE84F
:1006D000F08F361B1846314600F08CFF039B07460F
:1006E00078B10127711E01984A1150F8220001F0DB
:1006F0001F0207FA02F2024203D0B94200F3CF8090
:100700000227184631460393B244FFF741FE039B8C
:100710006BE718F8021000204A1E182A05F101069E
:100720007FF62BAF2E46CAE63CE3010898AC0108E1
:100730000AF1FF35002F40F0A480002D40F0A78083
:1007400001220198691150F8211005F01F05AA40F7
:100750000A4218465146039318BF47F00207A4EB1C
:100760000A04FFF715FE0225DBF804A0039B95E7BA
:1007700026468DE62546227802F0DF02502A00F058
:1007800099801D6013E70F9AC2F101020F920F9A30
:10079000002A93D001991E6988460A4600274FEA2D
:1007A000860901EB860003E0904242F8047C45D9BB
:1007B000944652F8041BB1F1FF3FF5D00131022DF0
:1007C000CCF800107ED014F01F0440F0AE8021253C
:1007D00076E70F9900293FF431AF5025194600986C
:1007E00000F03AFA002328460E9A136005B0BDE8DF
:1007F000F08F0020B9E6AA465CE6A61B19463246F1
:10080000009800F067FC00F1140203460027AAEBF1
:10081000060A0192E9E67278751C18F802102E4655
:1008200000293FF447AE16F8012F18F802100029EE
:10083000F9D13BE64FF00009841C13E69A68964212
:100840004ADA0121022D06EB010003EB860618614E
:10085000DDF80480716135D0002874DC00221A6153
:1008600000225A61DBF808200AF1010A5245AEDA8B
:100870001946009800F0F0F900230E9AA3251360A2
:100880009AE601275CE74FF00009019E99E61846B9
:100890002946039300F0AEFE039B074650E7184637
:1008A000B11E039300F0A6FE039B00283FF428AF7F
:1008B000032726E74FF0000A01274EE60F9900298B
:1008C0008BD0BBE6DBF80020013AA24262D02225A1
:1008D000F6E64FF00109D4E559680098013101931B
:1008E00000F094F9019B074600286CD01A6903F1C7
:1008F0000C01023292000C300193F0F7F9FA019BDF
:100900000098194600F0A8F901213B69022D03EB7C
:10091000010007EB8303386107F1140859613B4676
:10092000D0D08642BFF64FAF96E7C14459F8040CC9
:10093000019300F045FAC4F12004A042019BBFF6E8
:1009400046AF186988E75A6908EB800003F118047C
:10095000A0424FEA520229D94546216842EAC172B3
:1009600045F8042B54F8042BA0424FEA5202F4D865
:10097000C11A19398908013148F8212008EB810191
:1009800002B10431A1EB0802921041451A617FF4D3
:1009900069AF65E70122611158F8211004F01F04C6
:1009A000A2400A4214BF2125222589E6C8F800206A
:1009B0000AB14146E5E71A6152E70246E421054BD8
:1009C000054807F01FFE02468421024B024807F04B
:1009D00019FE00BFF0AC010804AD010810B50468B1
:1009E0008646013409E014F8013BA3F1410CBCF147
:1009F000190F98BF2033934207D111F8012B002A19
:100A0000F1D10120CEF8004010BD002010BD00BF84
:100A10000B682DE9F04F591102EB810113F01F0310
:100A200006464FF000050DBF0846081D8E46A1F191
:100A3000040E316840F8045C4C1C497885B00029EC
:100A400000F0AF807746F4460093AA460B46A946CD
:100A50007146AB469646DFF884810246019610E067
:100A6000202B00F296804D4508DD674502D9BAF18A
:100A7000070F67DDE6455CD34FF0080A14F8013F25
:100A8000B3B118F80360002EEAD00AF1010ABAF1F6
:100A9000080F05F1010542DCDCF800301B0106F00F
:100AA0000F061E43CCF8006014F8013F002BE8D17C
:100AB000104672468E46009B002D72D0BC4502D275
:100AC000BAF1070F74DD624555D26346111F53F822
:100AD000044B734541F8044FF9D9AEEB0C0323F0F6
:100AE00003030EF1010104330CF1010C8C4588BFA6
:100AF00004230021134443F8041B7345FBD950F829
:100B0000041C19B107E05EF8043D23B97245FAD11F
:100B10000123CEF80030052005B0BDE8F08FE64592
:100B2000ACD24CF804BC00234FF0010AACF1040C29
:100B3000B5E7ACF104074CF804BCA946BC464FF03D
:100B4000000A9BE7CAF1080080006646CDE902C2B0
:100B5000DCF800308446C0F1200A706800FA0AF21E
:100B60001A4320FA0CF3326046F8043FB742F4D837
:100B7000DDE902C27EE750F8041C002BC1D04FF023
:100B8000FF34C3F1200324FA03F3194040F8041C96
:100B9000B7E7104672468E4619462929019E009BEA
:100BA00003D0042005B0BDE8F08F0134346083E742
:100BB000DCF80040CAF108018900664688462546EF
:100BC000C1F12009716801FA09F42C4321FA08F5F2
:100BD000346046F8045FB742F4D874E73CE3010898
:100BE00082B049B15AB16BB113780B601278101E04
:100BF00018BF012002B0704701A9002AF3D11046A6
:100C000002B070476FF00100F4E700BF38B5436CE5
:100C100005460C464BB153F8240080B1026843F8F6
:100C200024200023C0E9033338BD2122042107F02A
:100C300009FD034668640028EDD1002038BD01217C
:100C4000284601FA04F56A1D920007F0FBFC002813
:100C5000F3D0C0E90145E4E731B1436C4A6853F889
:100C60002200086043F82210704700BF2DE9F041D0
:100C70004FF0000E0E461C460D69074601F11400A8
:100C800001680EF1010E8BB202FB0343090C4FEA1F
:100C9000134C02FB01CC9BB203EB0C43754540F8AF
:100CA000043B4FEA1C44EBDC3CB1B368AB4207DDCC
:100CB00006EB850301355C6135613046BDE8F081A6
:100CC000716838460131FFF7A1FF8046A8B132694B
:100CD00006F10C01023292000C30F0F709F97B6C3E
:100CE000726853F82210316043F82260464606EBE2
:100CF000850301355C613561DFE70246BA21024BAD
:100D0000024807F07FFC00BFF0AC010868AD0108A5
:100D10002DE9F8431E460C4626490833174681FB49
:100D2000032C092E4FEAE3730546C3EB6C0339DD50
:100D30004FF0010C00214FEA4C0C634501F1010119
:100D4000F9DC2846FFF762FF014668B3089B092FCC
:100D500043614FF00103036112DC09270A34BE42EC
:100D60000BDDF61B264414F8013B0A222846303BD3
:100D7000FFF77CFFB4420146F5D10846BDE8F88391
:100D800004F10909C8463C4418F8013B0A222846E8
:100D9000303BFFF76BFFA0450146F5D1A7F10804F2
:100DA0004C44DCE70021CCE70246D321024B034848
:100DB00007F028FC398EE338F0AC010868AD010873
:100DC000B0F5803F03463ABF102083400020B3F1C6
:100DD000807F3CBF1B020830B3F1805F3CBF1B012A
:100DE0000430B3F1804F03D3002B06DB0130704792
:100DF0009B0003D45B0003D420207047023070476F
:100E0000033070470368014613F0070209D0DA0780
:100E100021D498074BBF5B089B08012002200B6080
:100E2000704798B2A0B11046DAB20AB908301B0A6E
:100E30001A0704BF1B0904309A0704BF9B0802303D
:100E4000DA0703D45B0800F1010006D00B6070479D
:100E50001020C340E8E7002070472020704700BF03
:100E600038B5436C04460D464BB15868B0B10268C2
:100E70005A60002201234561C0E9032338BD2122C5
:100E8000042107F0DFFB034660640028EDD1002257
:100E900040F24511074B084807F0B4FB1C22012122
:100EA000204607F0CFFB0028F1D001220223C0E941
:100EB0000123DEE7F0AC010868AD01082DE9F04F31
:100EC000D1F8108015690E46A845924685B005DB1D
:100ED0002A46534645468A4690461E46DAF808306A
:100EE000DAF8041005EB0804A342B8BF0131FFF79C
:100EF0008DFE002800F0898000F1140707EB840EB6
:100F0000774505D23B46002243F8042B9E45FBD88B
:100F1000143606EB88080AF11409464509EB8505E5
:100F200066D2A5EB0A03153B23F003030AF1150A69
:100F3000043355452CBF9B464FF0040BCDF808E019
:100F40008246AE46039405E0090C2AD1B04507F16C
:100F500004074AD956F8041B8DB2002DF4D0CC46B4
:100F60003C46002301965CF8040B216886B28AB2E5
:100F700005FB0622000C090C05FB00111A4401EBCD
:100F8000124192B242EA0142E64544F8042B4FEA8C
:100F90001143E8D8019E47F80B3056F8041C090CA1
:100FA000D4D000223B6848461D463C469446028801
:100FB0009BB201FB02C202EB154243EA024344F832
:100FC000043B50F8043B25684FEA134CABB201FBDD
:100FD0000C33704503EB12434FEA134CE7D3B04593
:100FE00047F80B3007F10407B4D8DDE902E45046B6
:100FF000002C02DC05E0013C03D05EF8043D002B30
:10100000F9D0046105B0BDE8F08F02464FF4B1712C
:10101000014B024807F0F6FAF0AC010868AD010890
:1010200012F003032DE9F041144607462CD10E4679
:10103000A4101CD03D6C85B3E3074FF0000806D424
:10104000641014D02868A8B10546E307F8D52A46ED
:1010500031463846FFF732FF36B17B6C716853F882
:101060002120326043F8216064100646EAD1304600
:10107000BDE8F0812A4629463846FFF71FFF286061
:101080000546C0F80080E0E70F4A013B52F82320F4
:101090000023FFF7EBFD0646CAE701213846FFF7BC
:1010A000B5FD054640B140F271230122C0E9042399
:1010B000002338640360BFE7024640F24511034B4A
:1010C000034807F09FFA00BF3CE40108F0AC0108B8
:1010D00068AD01082DE9F0470C462769A36807EBC6
:1010E00062177D1C9D429046064649684FEA621988
:1010F00004DD5B009D4201F10101FADC3046FFF79F
:1011000085FD002851D0B9F1000F00F114010FDD69
:101110000B464FF0000C09F105024FEA820E00EB7E
:10112000820243F804CB9342FBD1AEF1140319447D
:10113000226904F1140318F01F0803EB820C2CD071
:101140008E464FF0000AC8F120091A6802FA08F228
:1011500042EA0A024EF8042B53F8042B9C4522FA6B
:1011600009FAF2D8ACEB0403153B23F00303043374
:1011700004F11502944538BF042341F803A0BAF1E5
:10118000000F00D13D46736C6268056153F8221070
:10119000216043F82240BDE8F087043953F8042B5E
:1011A0009C4541F8042FF9D8ECE702464FF4EF7163
:1011B000014B024807F026FAF0AC010868AD0108BF
:1011C00084460B690069C01A15D10CF1140C143156
:1011D0000CEB830210B401EB830301E0944508D2C9
:1011E00052F8044D53F8041D8C42F7D004D24FF04E
:1011F000FF3010BC70477047012010BC704700BF23
:101200002DE9F04F14460A6923698846D21A002A4C
:1012100083B040F0888001F1140604F1140202EB5F
:10122000830206EB830301E09E427FD253F8045D04
:1012300052F8041D8D42F7D076D32346002544464C
:1012400098466168FFF7E2FC002800F0898000F111
:10125000140949464FF0000C2769D8F8106004F1D2
:10126000140B08F1140EC56004F110020EEB860693
:101270000BEB870ACDF804B05EF8044B52F8045F1C
:101280001FFA84FBABB2A3EB0B03240C6344C4EB47
:10129000154404EB23449BB243EA0443764541F8EA
:1012A000043B4FEA244CE7D808F115018E4234BFC5
:1012B00000210121A6EB0806153EB608002906F11B
:1012C00001024FEA820208BF0422DDF804B00BEBF2
:1012D0000204A2454A4434D915462146E04651F855
:1012E000046BB3B263444FEA164E0EEB234E06EB8B
:1012F00008039BB243EA0E438A454FEA2E4C45F859
:10130000043BEBD80AF1FF3AAAEB040A2AF0030ADD
:10131000524423B952F8043D013F002BFAD0076133
:1013200003B0BDE8F08F88DA01258AE70021FFF7D6
:101330006DFC70B101220023C0E9042303B0BDE8B5
:10134000F08F00294FEA860608BF002609EB060247
:10135000DFE7024640F23721054B064807F052F915
:10136000024640F24521024B024807F04BF900BF0C
:10137000F0AC010868AD0108124B0A460B40A3F11E
:101380005073002B03DD00221946104670475B4264
:10139000B3F1A07F4FEA235106DA4FF40023002275
:1013A0000B4119461046704714391E29D4BF4FF01F
:1013B000004201224FF00003D8BFCA401046194630
:1013C000704700BF0000F07FF8B5046900F1140217
:1013D00002EB840454F8045C261F2846FFF7F0FC57
:1013E0000346C0F120000A2B086030DDB242A3F1B1
:1013F0000B071AD254F8083C1FB3C7F1200C23FA8C
:101400000CF1BD4045EA0106A4F1080546F07F5104
:10141000AA4203FA07F341F4401116D254F80C2CF7
:1014200022FA0CF213431846F8BD0B2B08D0002308
:1014300005FA07F747F07F51184641F44011F8BD0F
:10144000002345F07F5141F440111846F8BDB242E7
:101450002CBF002254F8082CC3F10B0703F115032D
:1014600025FA07FC38BFFA4005FA03F34CF07F5128
:101470001343184641F44011F8BD00BFF0B50121F7
:1014800083B016461F46FFF7C1FB0546002847D02C
:10149000C7F30A54C7F313030CB143F48013002EAF
:1014A000019314D101A8FFF7ADFC0122019B20306C
:1014B0006B612A6114B3089BA4F2334404441C609A
:1014C000099BC0F135001860284603B0F0BD68469E
:1014D0000096FFF797FC019B00B30099C0F1200232
:1014E00003FA02F2C34001930A43002B6A610CBF66
:1014F00001220222AB612A61002CDCD105EB8201C2
:10150000A0F23243086908990B60FFF759FC099B68
:10151000C0EB42101860284603B0F0BD009AE4E723
:10152000024640F20F31024B024807F06BF800BF51
:10153000F0AC010868AD01082DE9F04383B088469E
:1015400069468146FFF740FF04460D46404601A923
:10155000FFF73AFFD9F81030D8F81020A3EB020CAF
:10156000DDE900329B1A03EB4C13002B0BDD05EB7E
:1015700003573D4602460B4620462946EFF758FEE4
:1015800003B0BDE8F083C3EB033301EB03594946D5
:10159000F0E700BF01F1FF3C116902F114034FEACB
:1015A0006C1C03EB81010CF1010C8B4200EB8C0CE9
:1015B00016D210B5A0F1040E53F8044B99424EF820
:1015C000044FF9D88B1A153B23F003030433184456
:1015D000844504D9002340F8043B8445FBD810BD62
:1015E000844505D9002340F8043B8445FBD8704767
:1015F000704700BF03694A11934200F1140009DAF1
:1016000000EB830302E053F8042DA2B98342FAD819
:101610000020704700EB8203F8DD11F01F01F5D0C8
:1016200010B450F8224024FA01F28A40944208D0C3
:10163000012010BC70470120704753F8042D002A88
:10164000F6D18342F9D8002010BC7047242B2DE935
:10165000F84F42D8012B40D01F468E46804648485E
:1016600075461EF801BB10F80B4014F00804F7D1C2
:10167000BBF12D0F6FD06FF00049BBF12B0F04BFF2
:101680009EF800B005F1020E7BBBBBF1300F4CD0D1
:101690000A273B460025B9FBF7F6284607FB169AB2
:1016A00005E03BD0012507FB00C01EF801BBABF1F4
:1016B000300CBCF1090F06D9ABF1410CBCF1190F8C
:1016C0001AD8ABF1370C63451FDDB5F1FF3FECD005
:1016D0008642E6D24FF0FF35E7E7FEF775FC1622AB
:1016E000034600201A60BDE8F88F102BD2D1BBF161
:1016F000300F23D01F46CDE7ABF1610CBCF1190FC1
:1017000003D8ABF1570C6345DFDC6B1C2BD054B90D
:10171000002AE8D085BB1160BDE8F88FE245C1DA48
:101720004FF0FF35C1E74042F2E79EF8003003F08A
:10173000DF03582B08D008273B46ABE79EF8000094
:1017400000F0DF005828D5D110279EF801B03B46A5
:101750000EF1020E9EE79EF800B04FF00049012402
:1017600005F1020E90E72223C8F8003032B10EF1E5
:10177000FF3148461160CFE78146F8E74846B2E7B7
:1017800039E20108FFF762BF034649B1FF2A02D8D8
:1017900001200A7070478A224FF0FF301A607047AC
:1017A000084670472DE9F04FDDB00C4691460D918B
:1017B0000F93834606F026FE036818461A93FEF739
:1017C00047FC0822189000212CA8FEF7DFF8A38917
:1017D000180603D52369002B00F015870023002489
:1017E0009E46CDE93133002333AACDE91634DA46DB
:1017F00014464D46CDE91BEE3092CDF864E0CDF8AD
:1018000080E0CDF874E0CDF828E0CDF848E02F4630
:101810006E4BD3F8E460FEF76BFB0DF1B00C0346A2
:101820003A46504628A9CDF800C0B047002800F03D
:101830009F80C0F29580289B252B01D00744E7E7C5
:10184000B7EB0508064640F0978000224FF0FF33C3
:10185000934609937B787E1C8DF897200B929946CE
:101860000136A9F120035A2B00F2B280DFE813F011
:10187000F302B000B000EF02B000B000B000FD0213
:10188000B000B0006A003502B0002702D202B000FA
:10189000CE025B005B005B005B005B005B005B00FB
:1018A0005B005B00B000B000B000B000B000B00062
:1018B000B0002801B000AA013E0228012801280139
:1018C000B000B000B000B0003A02B000B000A80212
:1018D000B000B000B000D001B000BC02B000B00059
:1018E0008A06B000B000B000B000B000B000B00098
:1018F000B0002801B000AA01010228012801280136
:101900002B0201027400B0006402B0005502AF0661
:101910006E027400B000D0017200AC06B000B000DE
:10192000B206B00072000022A9F1300316F8019B44
:1019300002EB820203EB4202A9F13003092BF5D935
:101940000B928EE70F9B53F8042B002A0B920F93F8
:10195000C0F2B281337882E733784BF0200B7EE718
:10196000082200212CA8FEF711F8012007444FE7B8
:10197000B7EB0508064610D0329BC4E90058434433
:101980003293319B0133072B319315DC08340A9BCA
:1019900043440A93002E7FF458AF329B002B41F052
:1019A0005E810D9B9B8903F04003002B41F08083F7
:1019B0000A985DB0BDE8F08F50460D9930AA08F046
:1019C000D7F90028EDD133ACE1E700BF5C0500207A
:1019D0001096B9F1000FE0D0012300228DF80C9190
:1019E000069343AD8DF897200C93CDE913220E9208
:1019F000099211921BF0020302D00699023106915E
:101A00001BF08408329E05D10B9906980F1A002FFF
:101A100000F39B806AB101226260319A0136013283
:101A20000DF19701072A32963192216000F3D88395
:101A3000083463B102236360319B0236013326AA66
:101A4000072B32963193226000F3BF830834B8F13C
:101A5000800F00F0BF82099B0C9A9F1A002F00F3A1
:101A6000F9821BF4807F40F01E820C9B25601E448F
:101A70006360319B32960133072B319300F33F8330
:101A800008341BF0040F05D00B9B069A9D1A002DFD
:101A900000F3B383DDE90A3206998A42ACBF9B1892
:101AA0005B180A93002E40F00883002331930E9BAD
:101AB0001BB150460E99FEF76FFB33AC109DA6E6A6
:101AC0000F9B1096073323F00703F3E802670F9389
:101AD00027F000431F931E964FF0FF32DDE91E01F1
:101AE000B24BCDE91667EEF7C3FD002840F0F48451
:101AF000DDE91E014FF0FF32AC4BEEF79BFD0028F5
:101B000040F0EA840022002330463946EEF788FD93
:101B1000002840F0B2879DF8972000210320A44DB3
:101B2000A44B2BF0800B0E910690B9F1470FD8BF54
:101B30001D46CDE9131109910C901191002A3FF433
:101B400059AF069B0133069354E7102F319A41F3A6
:101B50000D82DFF864C2214630460D9C2E46CDF83A
:101B600054C06546219304E0103F102F01F1080195
:101B700016DD102301321030072ACDE931200D6027
:101B80004B60F1DD2146504630AA08F0F1F80028FC
:101B900040F09B82DDE93120103F102F33A9E8DCB3
:101BA00035460C460646219B013215993E44072ACC
:101BB000CDE931262160676000F381869DF897208A
:101BC000083427E70F9BB9F1430F109603F1040681
:101BD00003D01BF0100F00F00185082200212EA871
:101BE000FDF7D4FE0F9A43AD2EAB2946504612683E
:101BF00007F09AFF034601330C9001F054820C9BCE
